:020000040800F2
:1050000000C0002091740008E1740008E1740008F9
:10501000E1740008E1740008E17400080000000079
:10502000000000000000000000000000E174000823
:10503000E174000800000000E1740008E174000859
:10504000E1740008E1740008E1740008E1740008EC
:10505000E1740008E1740008315C0008E1740008A4
:10506000E1740008E1740008E1740008E1740008CC
:10507000E1740008E1740008E1740008E1740008BC
:10508000E1740008E1740008E1740008E1740008AC
:10509000E1740008E1740008E1740008E17400089C
:1050A000E1740008E1740008E1740008E17400088C
:1050B000E17400080000000000000000E174000836
:1050C000E17400080000000000000000E174000826
:1050D00000000000E1740008E17400080000000016
:1050E000E1740008E1740008000000000000000006
:1050F00000000000000000000000000000000000B0
:10510000000000000000000000000000E174000842
:105110000000000000000000755C0008E174000859
:10512000E1740008E1740008E1740008E17400080B
:10513000E174000800000000000000000000000012
:10514000E1740008E1740008E17400080D5C0008D7
:10515000E1740008E1740008E1740008E1740008DB
:10516000E1740008E1740008E17400080000000028
:10517000E1740008E1740008000000000000000075
:10518000E1740008E1740008E17400080000000008
:1051900010B590B000F05CFE4022002168460DF092
:1051A000D5F8002400F038FD001B962804D900F043
:1051B0003FFF00F031FD044601F050F8684600F072
:1051C000E1FE002807DD684605F03EF94022002197
:1051D00068460DF0BBF805F09DF8E3E7024BD86890
:1051E000C0F30220704700BF00ED00E0034AD2F890
:1051F000943043F00103C2F894307047001002402D
:10520000024BD3F89400C0F34000704700100240F6
:10521000024A136843F00103136070470010024014
:10522000024B1868C0F34000704700BF00100240F6
:10523000024A136843F008031360704700100240ED
:10524000034A136823F0F00318431060704700BF4F
:1052500000100240034A936823F003031843906050
:10526000704700BF00100240034A936823F4605364
:1052700018439060704700BF00100240044AD2F803
:10528000883023F040631843C2F88800704700BF9D
:1052900000100240034A136823F00703184310600C
:1052A000704700BF00200240034A136823F4C06324
:1052B00018431060704700BF00700040054AD16C71
:1052C0000143D164D36C82B003400193019B02B0CF
:1052D000704700BF00100240054A916D014391657F
:1052E000936D82B003400193019B02B0704700BFF1
:1052F00000100240054A116E01431166136E82B020
:1053000003400193019B02B0704700BF00100240B0
:10531000024A136843F004031360704710E000E092
:10532000024A536823F47F435360704700100240E1
:1053300000207047034AD2F8883023F00303C2F8F4
:105340008830704700100240024A936823F4E063FB
:105350009360704700100240024A936823F0F00304
:10536000936070470010024038B5444CA36D43F081
:105370008053A3650220FFF78DFF414B1B6803F0AC
:105380000703022B03D0AC213E4801F055F84FF43F
:105390000070FFF789FFD4F8983043F00103C4F898
:1053A0009830D4F898309B07FBD5FFF71FFFFFF725
:1053B00027FF0128FBD1FFF72BFFFFF731FF012863
:1053C000FBD1FFF735FFB020FFF73AFFFFF7A8FF4B
:1053D0000020FFF73FFFA56815F00C05FBD1FFF794
:1053E000BBFFFFF7B1FF4FF46050FFF73DFF2648CA
:1053F00003F094FAFFF78CFF234803F09DFAFFF7C0
:1054000099FF2846FFF73AFF4FF08070FFF764FFDF
:10541000A36B43F08073A363A36B23F08073A36338
:105420001A4B5A6822F0E0625A605A6822F0004231
:105430005A605A6822F0405242F000525A605A684C
:10544000120C120442F43B4242F07F025A605A6846
:1054500022F47F0242F408125A601A6822F47C5245
:1054600042F400521A60FFF7B9FEFFF761FF084BE4
:105470000001C0B283F8230038BD00BF0010024015
:1054800000200240D0360108006CDC0200600040C1
:1054900000ED00E028498B6D43F0805310B54FF4C8
:1054A00080608B65FFF700FFFFF7A0FEFFF7A8FE07
:1054B0000128FBD1FFF7ACFEFFF7B2FE0128FBD1BC
:1054C000FFF7B6FE8020FFF7BBFEFFF729FF0020A5
:1054D000FFF7C0FE8C6814F00C04FBD1FFF73CFF13
:1054E000FFF732FF4FF44050FFF7BEFE134803F0C2
:1054F00015FAFFF70DFF114803F01EFAFFF71AFF28
:105500004FF04060FFF7BAFEFFF768FEFFF710FFAD
:105510000B4B0001C0B283F823002046FFF7BAFE10
:10552000084B1B685B0706D040F2AB110648BDE88C
:10553000104000F081BF10BD001002400024F400B4
:1055400000ED00E000200240D036010810B5284CE4
:10555000A36D43F08053A3650120FFF79BFE254B0D
:105560001B6803F00703012B04D040F2BB11224853
:1055700000F062FF4FF48060FFF796FEFFF736FE03
:10558000FFF73EFE0128FBD1FFF742FEFFF748FE82
:105590000128FBD1FFF74CFE9020FFF751FEFFF7EB
:1055A000BFFE0020FFF756FEA36813F00C0FFBD1DF
:1055B000FFF7D2FEFFF7C8FE4FF44050FFF754FE4E
:1055C0000E4803F0ABF9FFF7A3FE0C4803F0B4F963
:1055D000FFF7B0FE4FF04060FFF750FEFFF7FEFD13
:1055E000FFF7A6FE064B0001C0B283F8230010BDF2
:1055F0000010024000200240D036010800366E0143
:1056000000ED00E0012805D010B1022804D0704759
:10561000FFF740BFFFF79ABFFFF7A6BE144A154930
:105620005368154843F4806310B5536002F5D032D7
:10563000124C936D43F080639365114A03F010FCA4
:10564000104B1149012000228861186102204A6034
:10565000886098600D495A60204603F034FD20466A
:105660000B4903F045FD2046BDE8104003F047BD5F
:1056700000700040A80100202C0100209449002067
:1056800044000020304C0020704C0020EC00002032
:10569000A8000020F0B54FF0804495B0002501200F
:1056A000FFF71AFE4FF47A77256101A92046CDE96C
:1056B0000375ADF80450029502F0E2FB236843F055
:1056C00080032360A36823F4A03323F0070301269B
:1056D000A3600CAA602310212046CDE90C36CDE949
:1056E0000E67109502F006FCA369214F23F4806336
:1056F000A3610CAA4FF480712046CDE90D6602F03B
:10570000F9FB7B6823F004037B600CAA4FF4805103
:105710002046CDE90D6602F0EDFB7B6823F4806343
:105720007B60A36823F00803A360A36823F480438D
:10573000A360A36823F43F43A360636823F070036E
:105740006360A36823F08003A3600E22022306A9EE
:105750004FF09040CDE90623CDE90855CDE90A5632
:1057600002F0EFFA23683343236015B0F0BD00BFA9
:105770001800004030B5012085B04FF09044FFF78D
:105780009DFD0220FFF79AFD2268012393FAA3F101
:10579000B1FA81F19940032505FA01F122EA0101EC
:1057A00093FAA3F22160E16893FAA3F0B0FA80F0D3
:1057B00093FAA3F29840B2FA82F205FA00F09A4006
:1057C00021EA000103FA02F20A430C49E2608A6806
:1057D0000F2022F00F0290FAA0F08A6001A80022A8
:1057E00001930292ADF80C308DF80E3003F0D8F82A
:1057F000034B40221A6005B030BD00BF00000140DD
:1058000000E100E030B5044687B01020FFF764FDEA
:1058100045F6C0534BF68030002C18BF1846134C89
:10582000ADF8040000255A2301A92046CDE9025312
:1058300002F026FB236823F080032360636823F0D3
:1058400070036360A36823F08003A360E36843F000
:105850000103E360236843F001032360256162B61E
:10586000034B4FF480025A6007B030BD0010004077
:1058700000E100E008B54FF48020FFF71FFD034A68
:10588000136843F00403136008BD00BF000806500E
:1058900010B54FF4805090B0FFF72CFDE0220223AA
:1058A0000024CDE900230323CDE902346946052312
:1058B0004FF090400494059302F043FA4FF4827144
:1058C0004FF4E063CDE9071301204FF40073CDE9F5
:1058D0000A031023CDE90C34069409940E94064C67
:1058E000072306A920460F9303F02CF8636823F0E2
:1058F0001003636010B010BD0030014010B50446C5
:105900000120FFF7F7FC4FF08050FFF7E5FC2D4A30
:10591000D36823F4E0631B041B0C43F0BF6343F420
:105920000133D360FFF75AFCFFF702FD0001C0B25C
:105930001076FFF753FCFFF7FBFC0001C0B2507676
:10594000FFF74CFCFFF7F4FC0001C0B29076FFF7C4
:1059500045FCFFF7EDFC0001C0B2D077FFF73EFC3D
:10596000FFF7E6FC0001C0B282F82000FFF736FC2A
:10597000FFF7DEFC0001C0B282F82200FFF72EFC28
:10598000FFF7D6FC0001C0B282F82300FFF7F2FE59
:1059900094B14FF48060FFF787FCFFF77BFD4FF475
:1059A0008060FFF781FC2046FFF72CFFFFF762FFC6
:1059B000BDE81040FFF76CBFFFF7D6FCFFF76AFEAB
:1059C000F1E700BF00ED00E0044B5A69002ABFBFB9
:1059D000034A9A6002F188329A60704700200240C0
:1059E0002301674508B500282AD100F0F9F9154BC5
:1059F000154A00280CBF1846104614490B6A20F0BF
:105A0000E06083421BD072B60B69DA03FCD4FFF767
:105A1000DBFF4B695B0041BF0D4BCB6003F14433AF
:105A2000CB600A4B18625A6942F400325A611A6913
:105A3000D203FCD45A6942F000425A6162B608BDF2
:105A40000448DAE7AAF8FFFFCCF8FFFF0020024085
:105A50003B2A1908AAF8FFF708B572B611490B6975
:105A6000DB03FCD4FFF7B0FF0B690B614A6922F43A
:105A7000FF6222F007024A614B6943EAC00343F028
:105A800002034B614B6943F480334B61054B1A6948
:105A9000D203FCD41A695A6922F007025A6162B62D
:105AA00008BD00BF0020024030B572B60C490C465C
:105AB0000D69ED03FCD40D690D614D6945F00105DB
:105AC0004D61026043602369DB03FCD42369012339
:105AD0002361636923F00103636162B630BD00BFD7
:105AE000002002402DE9F3411546164A1369DB03F5
:105AF000FCD4FFF769FF20F007002C4646194F1928
:105B00002B1B9D42A6EB040802D802B0BDE8F08131
:105B1000082C2246A7EB040128BF082268460CF097
:105B2000FBFB072C06D8C4F10802FF210DEB040093
:105B30000CF00CFCDDE900234046FFF7B5FF083C04
:105B4000DEE700BF00200240F7B56FF00306104CFF
:105B5000031D361A0844F218914201D803B0F0BD73
:105B60006268D207FCD5A2680192626812F0660FE3
:105B700002D001200CF06AFB01AD1A1F8242EDD069
:105B800015F8017B02F8017B9A42F7D10433E2E772
:105B9000000806501D2893BF024B00EB8000400018
:105BA000185C704700000020014610B5C0F30740A4
:105BB000FFF7F0FF0246C1F30720FFF7EBFF0446B3
:105BC000C8B2FFF7E7FF642358434FF080415A43C0
:105BD000000A6343C0F57A701B0A8863C3F57A73C1
:105BE0004FF4C060B2FBF0F2C2F57A72CA630B6484
:105BF00010BD4FF090431869C04300F0010070479A
:105C0000014B1870704700BF68020020014801F086
:105C1000B9BD00BFB04C0020034B044A5B6A126858
:105C20005A2000FB02307047001000405402002050
:105C300008B50B4B5A695A610A4B1A680A4B9A42CB
:105C40000DD1FFF7E9FF09490A68801A192803D91D
:105C5000FFF7E2FF064B1860FFF7DEFF086008BDA4
:105C60000004014020000020F35B00085C020020DB
:105C70006002002038B5204B00221A611F4A1368C9
:105C800001331360FFF7C8FF1D4B1B68C01A5A2869
:105C900005D91C4B186810B140B204F06FFB1A4BC9
:105CA0001A681A4B9A421CD1002001F095FB00BBE8
:105CB000012001F091FB051C18BF0125144CFFF7D2
:105CC000ABFF2268801A19280BD912490A7822B929
:105CD0001DB1FFF7A1FF104B1860FFF79DFF20607B
:105CE0000D700E4B1B68012B05D1BDE8384000F04C
:105CF0004FBD0125E2E738BD0010004054020020EE
:105D0000640200205802002020000020635D00088B
:105D10005C020020AA020020600200205002002045
:105D200038B5044672B6FFF777FF064B186062B6C7
:105D3000054D2CB12B68A34202D060B204F01EFBCB
:105D40002C6038BD640200205802002010B50146C6
:105D5000FFF762FF0446FFF75FFF001B8842FAD39C
:105D600010BD08B5002001F037FB68B15F20FFF7D8
:105D7000EDFF002001F030FB60B9012001F02CFBA9
:105D8000003018BF012004E0012001F025FB0028AD
:105D9000ECD108BD0120FCE7BFF34F8F0549064B4E
:105DA000CA6802F4E0621343CB60BFF34F8F00BFB9
:105DB000FDE700BF00ED00E00400FA0510B501F0BA
:105DC00021FB044C20B101F0B3FA034B236010BD5A
:105DD000024BFBE720000020635D0008F35B000836
:105DE000044BD3E90802044B9A420CBFC0F34000B5
:105DF0000020704700880308791E55AA10B50C4C86
:105E0000ADF5006D21464FF4006268460CF084FA4F
:105E1000089B712043F002030893FFF71DFE4FF427
:105E2000006269462046FFF75DFE0DF5006D10BD6E
:105E300000880308014B1868704700BF500200201B
:105E4000024B1B780BB9FFF7E9BB7047A902002092
:105E5000F0B5012091B0FFF751FD01F0D3FA3A4CB3
:105E600010B901F0EFF820602368384C012B50D1B5
:105E70002370374B374A1A60FFF7E2FF04F048FA05
:105E800006F0BEF8344B5A6A344B9A423CD0344B3D
:105E900031491B6ADBB2AA2B4FF02002684619BFBA
:105EA00025A7D7E9006726A7D7E900670CF034FAE1
:105EB0007120FFF7D1FD202269462748FFF712FE27
:105EC000284B08AA03F1200C154618685968144697
:105ED00003C4083363452246F7D120226946284689
:105EE0000CF0FEF9E8B9204B20481C88002322461C
:105EF000FFF7DAFD1E4922461E48FFF7F3FD324642
:105F00003B461D48FFF7D0FD0020FFF76BFD11B0A9
:105F1000F0BD0020FFF7F2FC00232370FFF74EFFD7
:105F2000AAE7164B11481C8800232246FFF7BCFD48
:105F300022461349E0E700BF02000000791E55AA7F
:105F400000000000791E55AA50020020A90200207E
:105F500020000020F35B000800880308791E55AA82
:105F600000200240DB360108FC39010828880308BC
:105F70000D3701083088030820880308063D010812
:105F8000FE39010810B5044600F09CFA18B120460D
:105F900000F078FA402010BD08B5402200210948E1
:105FA0000CF0D4F90748FFF7EDFF002808DD05489D
:105FB00004F04AFA91284FF0FF3018BF002008BDC6
:105FC0000020FCE76902002038B50446FFF724FEF4
:105FD000084D0444FFF720FE844209D30120FFF757
:105FE000B5FEFFF7D9FF20B92B6898470028F1D1FB
:105FF000002038BD20000020054902460B8803F030
:106000003003302BFAD040238121024803F047B8F7
:106010000468004094490020034B0A221A60034B95
:1060200000221A60704700BFB4020020B8020020AE
:1060300038B5204B204C1B689847204A21681368CC
:1060400039B3013B9D1E0C2D136007D9B1FA81F1C4
:1060500049090F2B21601ED90F231360184C2368A8
:10606000EBB1FFF7D9FD17490B68C01A78280FD993
:10607000FFF7D2FD144B08601868421C10F00100B5
:1060800018BF70201A60FFF78FFD2368013B236063
:1060900038BD0133D6E7002BE0D10123DDE71368DB
:1060A000DA0020B11046BDE83840FFF77DBDD802C8
:1060B000F9E700BF20000020B002002024000020EB
:1060C000B4020020B8020020BC02002010B5044633
:1060D0007F20FFF7C1FC2146D0220648FFF702FDD2
:1060E0007E20FFF7B9FC2146D0220348BDE81040CE
:1060F000FFF7F8BC00F8030800F003081FB50446DA
:10610000D0220E490CF008F92378A52B10D01022CC
:106110000B4968460CF000F99DF80030A52B0AD118
:10612000D022074920460CF0F7F82046FFF7CEFFB3
:10613000012004B010BD0020FBE700BF00F80308F9
:1061400000F0030830B5424D2B685A1C85B0044658
:1061500035D002930023039344B9012101A8FFF72E
:10616000F3FC9DF8044004F00F0401340021039A6D
:106170000D46AB0003F1006303F57A331B68581C2E
:1061800028D101B10392DDE902325ABB1B0201336F
:106190007D200393FFF760FC042203A92D48FFF73D
:1061A000A1FC029B7C2001330293FFF755FC284899
:1061B000042202A9FFF796FC039805B030BD012325
:1061C0007C200293FFF748FC042202A92846FFF72F
:1061D00089FCBFE70235B5F5007F1A464FF0010193
:1061E000C7D1CFE7B4F5807F98BFA4180394240AE1
:1061F0009C4208D97C200294FFF72EFC042202A9BD
:106200001348FFF76FFCB5F5007F0FD1039B1B0A06
:1062100001337C200293FFF71FFC042202A90C48E3
:10622000FFF760FC7D20FFF717FC002505F10070EB
:1062300000F57A400422800003A9FFF753FC064BC7
:1062400003981A68904200D1FEE71860B5E700BFD6
:1062500000E0030800E80308AC020020024B1B68C2
:106260000BB100F09FBE704750020020F8B5214BE3
:1062700019680129054638D01F4B1B78002B36D1F1
:106280001E4C236823BB1E481E4EFFF78DFCFFF7F4
:10629000C3FC2F18FFF7C0FC87420AD30120FFF789
:1062A00055FDFFF779FE0146F8B933689847002895
:1062B000F0D02846FFF788FE0146B0B92368A3B1A5
:1062C000FFF7AAFC2368C01AB0F5FA6F0DD206E0FA
:1062D000FFF7A2FC2368C01AB0F5FA6FD3D22846A4
:1062E000FFF772FE0023236001210846F8BD02215A
:1062F000FBE700BF5002002068020020600200207F
:106300002035FF002000002008B5FFF71DFC01200C
:1063100008BD10B5722420460134E4B2FFF79CFB9F
:106320007C2CF8D110BD322070474FF4B47250432A
:10633000C30A092B08D803F58033723300F4FF60D9
:1063400000EBC320FFF7CEBB70474FF4B47250434D
:10635000C30A092B10B40C460BD803F5803300F4A4
:10636000FF617233204601EBC3215DF8044B0BF053
:10637000D3BF5DF8044B70472DE9F0414FF4B4777B
:1063800007FB00F6F50A092DADF5006D88461BD810
:1063900005F580307230C4024FF400622146684631
:1063A0000BF0ACFF06F4FF603A46414668440BF040
:1063B000A5FF05F17200C0B2FFF74EFB4FF400627B
:1063C00069462046FFF78EFB0DF5006DBDE8F081B4
:1063D0000A4B4CF6CC421A6045F255521A60002224
:1063E0005A6040F6FF721A614FF4FA629A60DA68F6
:1063F0005207FCD14AF6AA221A60704700300040CA
:106400000B4B10B50246044603F1100153F8040B80
:1064100042F8040B8B42F9D1064B1B6813B1892358
:10642000237010BD00F0EEFF0028FAD09823F7E7A4
:10643000FC36010850020020FEE70000F8B50E4DC2
:106440002E68632E014613DC0C4F0D483C68402239
:1064500000EB84100BF060FF0134632CC8BF0023F5
:1064600006F10106D4BF3C603B602E600020F8BD01
:106470004FF0FF30FBE700BFC4020020C81B002024
:10648000C802002010B50C4C0C4B2168402203EBD5
:1064900081110BF041FF0A4B1A68002A09DD2168BF
:1064A00001316329C8BF0021013A21601A60002030
:1064B00010BD4FF0FF30FBE7C0020020C8020020F3
:1064C000C4020020014B1868704700BFC4020020BE
:1064D0000048704700880308014B188D704700BFC3
:1064E000008803081D4B1E491A8D10B504460BF099
:1064F00013FF0A221B4904F2C6200BF0F1FE60BB19
:10650000FFF798FCA8B1892384F8A232164B04F156
:10651000AC0203F1140153F8040B42F8040B8B4254
:10652000F9D11249422204F2C520BDE810400BF017
:10653000E5BE00F067FF80B1982384F8A2320C4BCF
:1065400004F1AC0203F1140153F8040B42F8040BFC
:106550008B42F9D142220749E5E710BD00880308C4
:1065600030880308083D0108133D0108283D010853
:106570006B3D0108803D010810F0040F0CBF0123A2
:106580000223020748BF013318467047034B00221D
:106590001A6020221A7001229A707047CC1B0020CA
:1065A00070B5114D2B7813F0020F04462E4605D01E
:1065B0000A2000F081FD2870012070BDFFF72CFB40
:1065C0000444FFF729FB844201D80020F5E70A20A4
:1065D00000F072FD10F0060F30704FF00100ECD1AA
:1065E000FFF7B4FBEDE700BFDE2300202DE9F04309
:1065F0001F46002389B03B60064688469146FFF758
:106600000BFB174C0644FFF707FB864201D800201E
:106610001FE025786A0704D40A2000F04DFD0546E6
:1066200020700C2000F048FD43B2002B14DD6B07F6
:1066300012D500F01F042146684600F06DFD4C4560
:106640002246A8BF4A463A60694640460BF056FECD
:10665000012009B0BDE8F0830120FFF777FBD2E706
:10666000DE23002038B50D460446042000F0C0FDAE
:10667000202D2946204628BF202100F063FD082058
:10668000BDE8384000F0B4BD70B588B01E4600F0DB
:106690000F038DF80030124B1B788DF8013000236A
:1066A00014468DF80230FFF767FF054624B119B193
:1066B000224668440BF022FE631908AA02341344F0
:1066C0002C44320AE1B2684603F8202C03F81F6C10
:1066D000FFF7C8FF0120FFF763FF08B070BD00BFE0
:1066E000DD2300201D2A01D8FFF7CEBF0020704710
:1066F00000220B461146FFF7C7BF6123FF29037035
:1067000086BF00234370417070470000034A002396
:106710001370034A1370034A13607047D11B0020A3
:10672000D01B0020D41B002070B5164D2C788AB0E9
:1067300034BB154E337863B9144B02211B88ADF876
:10674000083002A80124FFF78DFF347020460AB0FC
:1067500070BD01AB202202A9FFF748FF10B9012349
:106760002B70F3E7019B022BF9D19DF80830F22B37
:10677000F5D19DF80930012BF1D134700446E5E7DD
:106780000024E3E7D01B0020D11B0020C33D0108FB
:1067900038B5084D2C685CB1FFF73EFA04F59674E5
:1067A000844205D80A20FFF7BFFFFFF735FA2860BB
:1067B00038BD00BFD41B00201FB5194B00F00F02DD
:1067C00000095A7024D110221A7042F20E23ADF83B
:1067D0000030C0238DF80230124B1A68CDF8032028
:1067E0005A68CDF8072068461A899B7AADF80B20C5
:1067F0000E218DF80D30FFF735FF0A20FFF7D0FE90
:1068000058B9022000F0F4FC012005B05DF804FB4B
:1068100001280CBF18222022D6E70020F5E700BF90
:10682000CC1B0020E73D010830B589B004461E228C
:106830000D460DF1020000210BF088FD2046FFF708
:106840009BFE0D4A9378B3FA83F35B0993700B4B6D
:1068500004F00F0444F0A0041B788DF800400146BA
:106860008DF801301DB944F010048DF800406846E1
:10687000FFF7F8FE09B030BDCC1B0020DD2300205F
:106880002DE9F04F95B01446884600F00F07FFF74A
:1068900073FE1F2C0646DFF810911DDC99F800509E
:1068A0001E2200210DF12E000BF050FD8DF82C70F2
:1068B0008DF82D5044B1B8F1000F05D00BAB224636
:1068C000414698190BF01AFD3119C9B20BA8FFF710
:1068D000C9FE15B0BDE8F08FC0F12003002500937C
:1068E0000BABAA4603EB000B009A8DF82C70631BD0
:1068F0009342A8BF134699F800208DF82D2008EB8D
:1069000005011A46584601938DF82EA00BF0F6FCAF
:10691000019B1D44A542B8BF9DF82C2006EB030146
:10692000B8BF42F010020BA8C9B2B8BF8DF82C2036
:10693000FFF798FE0520FFF733FE0028C9D09DF829
:106940002C30D8062AD52022002103A80BF0FEFC0B
:1069500002AB202203A96420FFF748FE0028B8D02C
:106960009DF80C3003F0E202A22AB2D1D90604D578
:1069700001211846FFF758FFABE718460193FFF7D0
:10698000FBFD029A9042A4D19DF82C20019B5A4015
:10699000D20703D403F0F603A22B9AD0A54287F0C6
:1069A0000107A1DB95E700BFDD230020F8B5144DFA
:1069B00007460020286013480124FF2A0E46047071
:1069C00000DD2BB131463846BDE8F840FFF758BF2F
:1069D000A2F1FD040C482C60FD220BF09DFC214629
:1069E0000A48FFF78AFE3846FF220749FFF748FFAB
:1069F0002A68054806F1FD01BDE8F8400BF08CBCA3
:106A0000D8230020DC230020D81B0020D51C002028
:106A100010B40C469C42114612DC127802F0F002CF
:106A2000A02A09D1042C0FDD9C422246A8BF1A4699
:106A30005DF8044B0BF054BC9C4205D12246F7E7AD
:106A40000A205DF8044B70470B20FAE738B5144A6A
:106A5000082304460D46FFF7DBFF18B90520114B4C
:106A6000D87038BD0723104A29462046FFF7D0FFCB
:106A700008B90120F3E702230C4A29462046FFF714
:106A8000C7FF08B90320EAE70223094A294620463E
:106A9000FFF7BEFF08B90420E1E70020E1E700BFEF
:106AA000C53D0108CC1B0020CE3D0108FF3D01087B
:106AB000023E01082DE9F0411378ADF5805D13F039
:106AC0007F0782B005460E46144604D04FF4DC41E1
:106AD000FFF70EFE8EE05378102B00F0D78012D80F
:106AE000022B00F0BE80032B00F09080012B10D110
:106AF000944BDB78052B0CD19388402B00F09480CD
:106B00004FF4CE41E4E7B02B00F0F68004D8A42B7C
:106B100062D04FF4DA411EE0C02B16D0EE2BF8D134
:106B20009288042AF5D18849D4F806000BF0D8FBE6
:106B30000028EED14FF410412846FFF7D9FD14206C
:106B4000FFF704F9FFF728F9FEE793780BB9D3783C
:106B50001BB146F686212846BAE7D2F80A607B4B7D
:106B600036F480721C68984608D0A64206D9FF2CDD
:106B700000F2868004F5CE4189B2ECE7FF220021C5
:106B800001A80BF0E3FB002E08BFFD26A642374606
:106B900028BF27463A466E4901A80BF0AFFBA64234
:106BA00018D201ABE11BD819FFF7A7FD02223A4426
:106BB00001A92846FFF764FED8F800206448D21BDC
:106BC000C119C8F800200DF5805D02B0BDE8F041A4
:106BD0000BF0A2BB0022EAE79188D2F80600FFF78B
:106BE00035FF05280BD14FF410430622594928469A
:106BF000FFF778FD0DF5805D02B0BDE8F08110B1C2
:106C00004FF41041A7E746F68221A4E74D4BDB780D
:106C1000052B7FF47EAF9288D4F8061002AF01AB4B
:106C2000304603F071FA14E0FFF704F9012801D1AE
:106C3000FEF7E8FC01ABA288D4F80610304603F05A
:106C400063FAFFF7F7F8012802AF02D10020FEF740
:106C5000D9FCA37BB7F8FE2F01A92846FFF7A6FEB3
:106C6000C8E7384BD87805287FF453AFD4F806101E
:106C7000928891F8403041339A4204D0FFF766F889
:106C80004FF4CE4167E702AF01ABC9E72D4BDB788C
:106C9000052B02D04FF4DA411AE70120FEF7B0FFCE
:106CA00001A805F0A1F901AAA188D4F8060005F011
:106CB000CDFC8046384602AEFEF7A2FFB8F1000FC9
:106CC00018D1B6F8FE2F01A9F01E0BF025FBB6F87F
:106CD000FE3F0333A6F8FE3FB6F8FE2F06F8048CFD
:106CE00001AB1344902103F8021C002103F8011C9E
:106CF000A37BB1E70323EDE7124BD2F80A20DB7840
:106D0000032B92B204D0042B11D046F68221DFE689
:106D1000531E9BB20F2B28BF0F220F494FF4104375
:106D2000D2B2FFF7DFFC0A20FFF73AFC62E7531EFE
:106D30009BB2142B28BF14224FF41043D2B2074940
:106D4000EFE700BFCC1B0020FA3D0108D82300204C
:106D5000D81B0020F33D0108D83D01082800002081
:106D60002DE9F043054685B000782B4C0E46FFF721
:106D700003FC237880462F1833B17B78C02B1FBFCC
:106D8000264A002313602370A6EB08016A463846A2
:106D900002F014FF014628B12878FFF7A9FC05B0DE
:106DA000BDE8F083237883BB15F80830DFF86C90DA
:106DB000DB06D9F8004015D53119B1F5006F02D9BD
:106DC0004FF4CE41E8E7BDF804601548DDF8061041
:106DD0002044324634440BF09FFAC9F800404FF487
:106DE0001041D9E78CB1DDF80610BDF80420081970
:106DF0000BF092FA22460A49DDF806000BF08CFAF5
:106E0000BDF804301C44ADF804406A463946287881
:106E1000FFF750FEC3E700BFDC230020D82300208B
:106E2000D81B0020034B044800214FF480621960F6
:106E30000BF08CBAE0270020DF2300202DE9F0477B
:106E400006460C46002900F0A280057805F0F00304
:106E5000D02B0DD14378112B4FF0010106D183784F
:106E60001C0703D1BDE8F047FFF7FCBB4948F9E731
:106E700005F0C203022B5CD12846FFF77DFB2907F2
:106E800044BF454B7278DFF818A148BF1A7015F05F
:106E9000100F0746DAF80080D1461DD004EB080336
:106EA000B3F5806F06D94FF4DE412846BDE8F047C0
:106EB000FFF71EBC844209D9241A311837482246EC
:106EC000404444440BF01AFACAF8004030780121DB
:106ED000BDE8F047FFF7A8BCB8F1000F22D084420C
:106EE0002E4D09D9241A22463118444405EB0800D6
:106EF0000BF004FACAF80040D9F8004027492246AE
:106F0000E8190BF009FA31463A4624480BF004FA26
:106F10003919C9F800102148FFF722FFBDE8F047F2
:106F2000FFF780BF314622461C480BF0E7F92146A7
:106F3000F1E705F0E202A22A07D12A0742BF164B69
:106F400042781A7001212846C2E7C22B1FD115F0E2
:106F5000300F19D12846FFF70FFB2B0742BF0E4B0E
:106F600072781A7001463046FFF77CFB0220FFF76B
:106F700017FB102000F03CF9FFF708FBFFF752FF6A
:106F8000BDE8F047FFF7C2BB46F685118DE7BDE8C7
:106F9000F08700BFD63D0108DD230020DF2300205D
:106FA000E027002010B590B008A800F097F8234B18
:106FB0009DF82A2019781A709DF8243003F03803C0
:106FC000302B03D00024204610B010BD100601D491
:106FD0000A0601D5FFF7DAFA9DF82A3019434B0764
:106FE000F0D59DF82C4063B2002BEBDD04F01F04BC
:106FF0002146684600F090F8002CE3D09DF8003060
:10700000502B17D006D8262BDDD021466846FFF737
:1070100015FFD8E7522BD6D0E02BF6D19DF8010012
:10702000FFF7CAFB064B01229A70FFF7FBFEFFF742
:107030006DFBC8E7102000F0DBF8C4E7DE2300207A
:10704000CC1B002038B5FFF7A1FA00F0DDF80446AC
:10705000FEF7E2FD0546FEF7DFFD401B092806D9D5
:1070600000F00AF9002C18BF0224204638BDFFF7B3
:1070700099FF0028EFDD0124F7E70000064B1A46D0
:10708000996811F4C05FFBD118739368DB07FCD5D6
:10709000D068C0B2704700BF0030014010B50C4648
:1070A000FFF7ECFF2046FFF7E9FF024B01229A6150
:1070B0009A6210BD0004004808B500F01F0040F0BF
:1070C0002000FFF7DBFF0020FFF7D8FF024B012273
:1070D0009A619A6208BD00BF0004004838B50C4BA5
:1070E00004469A68D20701D5DA68FAE72420FFF748
:1070F000C5FF251D0D340020FFF7C0FF05F8010B6B
:10710000A542F8D1034B01229A619A6238BD00BFB3
:10711000003001400004004838B50446A0200D4668
:10712000FFF7ACFF2544AC4204D1054B01229A6124
:107130009A6238BD0020FFF7A1FF04F8010BF2E7C7
:107140000004004838B5044680200D46FFF796FF3E
:107150002544AC4204D1054B01229A619A6238BDA4
:1071600014F8010BFFF78AFFF3E700BF00040048A3
:1071700038B505467F200C46FFF780FF680000F019
:10718000FE00FFF77BFF0020FFF778FF2070002054
:10719000FFF774FF60700020FFF770FFA070002001
:1071A000FFF76CFF024BE07001229A619A6238BDD2
:1071B0000004004838B5054640200C46FFF75EFF46
:1071C000680000F0FE00FFF759FF2078FFF756FF38
:1071D0006078FFF753FFA078FFF750FFE078FFF7E4
:1071E0004DFF024B01229A619A6238BD00040048AB
:1071F00008B540F0C000FFF741FF024B01229A6141
:107200009A6208BD0004004838B5194C0120226874
:1072100090FAA0F1B1FA81F190FAA0F30325814030
:10722000B3FA83F305FA01F1834022EA010200FA7E
:1072300003F3134323600F4BA0611A6822F002028C
:107240001A601A6802431A605A6842F480525A60FF
:107250001A6842F040021A60A062FEF777FD1C2017
:10726000FFF72AFFA0F114035842584138BD00BF70
:10727000000400480030014037B51C20FFF71CFF18
:1072800001A90020FFF774FF01A97E20FFF770FF1E
:107290009DF80430442B06D19DF805301BB99DF8AC
:1072A0000630202B13D01F4C1F4B019301A97E20C9
:1072B0000125FFF77FFF0A20A561FEF747FD0A20A1
:1072C000A562FEF743FD01A97E20FFF751FF01A94A
:1072D0007F20FFF74DFF9DF80430052B03D19DF86B
:1072E0000530402B1BD005210220FFF7D7FE0D4CA7
:1072F00040210320FFF7D2FE01250C4B019301A989
:107300007F20FFF757FF0A20A561FEF71FFD0A2027
:10731000A562FEF71BFD01A97F20FFF729FF03B03F
:1073200030BD00BF0004004844002000054080003C
:10733000F0B5184A184F936C43F4803387B09364C8
:1073400002243023CDE900340023CDE90233049335
:107350006946092338460593402500F0F2FC0126D2
:10736000694638460095039600F0EBFC0B4B0C4A3F
:107370001E6019680A431A606FF070021A611D627C
:107380001C635A6822F003025A6003229A6007B015
:10739000F0BD00BF00100240000400480040024061
:1073A000C0400279074B1A6822F002021A600322D9
:1073B0009A601A6822F010021A601A6842F00202FB
:1073C0001A60704700400240024BDA68D207FCD5D1
:1073D000DB6870470040024008B5094958B10128F0
:1073E0000CD0FFF7DFFFFFF7EFFF886B2C288CBF77
:1073F0000020012008BD10238B62F2E72023FBE769
:107400000040024070B5204D2B78002B3AD11F4A26
:107410000223106893FAA3F1B1FA81F10324490021
:1074200004FA01F120EA010193FAA3F01160D06897
:1074300093FAA3F1B1FA81F193FAA3F3B3FA83F3C8
:10744000490004FA01F101265B0020EA010106FA75
:1074500003F30B43D36000BF00BF00BF00BF106940
:1074600080F00200C0F340002870D16896FAA6F3BD
:10747000B3FA83F3B3409C4021EA040496FAA6F6DB
:10748000D46070BD0120FCE7E42700200004004820
:10749000DFF834D000F026F8002103E00B4B5B58F6
:1074A000435004310A480B4B42189A42F6D30A4A19
:1074B00002E0002342F8043B084B9A42F9D30AF059
:1074C000EBFEFDF765FEFEE700C000201C4A010848
:1074D0000000002050020020500200201071002007
:1074E000FEE700000E4AD2F8883043F47003C2F879
:1074F00088300C4B1A68002042F001021A60986034
:107500001A6822F0A85222F410221A604FF4805216
:10751000DA601A6822F480221A609861FEF772B865
:1075200000ED00E0001002402DE9F041044686B075
:10753000002869D090F8293403F0FF021BB980F8C5
:10754000282401F097FC2546032355F8100B84F8F6
:10755000293400F030FE0FCD6E460FC62B68336025
:1075600004F1040898E80E00206800F013FE0021E2
:10757000206800F02AFE00212246234604F110056F
:107580000126084683F82810D98601310F2983F88F
:10759000296083F82B00C3E90E00186403F120036F
:1075A000F0D100231F4682F8283201330F2B82F8D6
:1075B000297282F82B72C2E98E77C2F8407202F10A
:1075C0002002F0D10FCD6E460FC62B68336098E8CD
:1075D0000E00206800F0FBFD012384F8247084F87D
:1075E0002934E369012B02D1204600F095FB236A80
:1075F000012B02D1204600F07DFB206801F08AF8C3
:10760000002006B0BDE8F0810120FAE790F82834A8
:10761000012B10B504460CD0012380F828340068F3
:1076200001F070F8206800F0BCFD002084F8280408
:1076300010BD0220FCE790F82824012A10B504466A
:107640000BD0012280F8282484F82410006801F06F
:1076500053F8002084F8280410BD0220FCE770B520
:1076600001F00F06044611F0800F4FEA4610054660
:107670001ED0254400F128010120214485F829006D
:107680000A614A780E70CB7002B1CE81022B04BF22
:1076900000230B7194F82834012B11D0012384F8B6
:1076A0002834206800F0B0FD002084F8280470BD64
:1076B000254400F50A710020214485F82902DFE7FE
:1076C0000220F4E710B5044601F00F00430111F069
:1076D000800F1A4615D0224403F1280101232144CA
:1076E00082F82930087094F82834012B11D0012336
:1076F00084F82834206800F0DFFE002084F8280495
:1077000010BD224403F50A710023214482F8293276
:10771000E8E70220F4E770B501F00F0100EB411635
:107720004C01002586F8281204F50A710144C6F8B8
:107730003C22C6F84032C6F8445286F82952006806
:1077400001F004F8284670BD01F00F0100EB411173
:10775000B1F84402704770B501F00F0100EB41151C
:107760004C012B640026012385F8281004F1280120
:107770000144EA636E6485F82930006800F0E6FF92
:10778000304670BD2DE9F84F0446006800F0CAFF8E
:10779000000409D5DFF854A4DFF854B42068B0F829
:1077A00044301A0400F1CB80206800F0BBFF410593
:1077B0000FD52268B2F8443023F480631B041B0CFD
:1077C0002046A2F8443001F0A8FB00212046FFF734
:1077D00032FF206800F0A6FF430408D52268B2F803
:1077E000443023F480431B041B0CA2F8443020686F
:1077F00000F098FF870408D52268B2F8443023F4DB
:1078000000531B041B0CA2F84430206800F08AFFD0
:10781000C60426D52268B2F8403023F004031B04C6
:107820001B0CA2F84030B2F8403023F008031B04D0
:107830001B0CA2F8403094F86034012B05D10021D4
:1078400084F86014204600F07BFA204601F073FBB8
:107850002268B2F8443023F480531B041B0CA2F8B6
:107860004430206800F05EFF05051BD52068B0F8A5
:10787000403043F00803A0F84030B0F8443023F41F
:1078800000631B041B0CA0F84430B0F8403043F0F8
:107890000403A0F8403000F045FFC00402D42046A5
:1078A00001F048FB206800F03DFF010626D5236863
:1078B000B3F8442022F080021204120CA3F84420F2
:1078C00094F86024002A40F08A81B3F8402042F006
:1078D0000402A3F84020B3F8402042F00802A3F8C5
:1078E0004020B3F854309B08012103F03C0384F896
:1078F0006014C4F86434204600F022FA206800F0D6
:1079000011FF82050BD52268B2F8443023F40073CE
:107910001B041B0CA2F84430204601F0FAFA206840
:1079200000F000FFC30508D52268B2F8443023F404
:1079300080731B041B0CA2F84430BDE8F88FB0F82C
:10794000441089B211F00F0740F0A18011F010012E
:10795000038827D10AEA03030380B0F8502094F883
:10796000283000F202401044E26B30F83330C3F3A9
:10797000090363641344E363204601F0C3FA94F8F7
:107980002430002B3FF40AAF226C002A7FF406AFAC
:1079900094F82430216843F08003A1F84C3084F837
:1079A0002420FBE69BB21A051DD5B0F8501094F8C0
:1079B000282200F206430B4404F5866133F8323086
:1079C000B4F82E22C3F30903C4F8443200F08CFF4C
:1079D0002268138823F070031B051B0D13802046BB
:1079E00001F078FADAE61F047FF5D8AE038823F0B9
:1079F00070031B051B0D0380B0F8501094F828226B
:107A000000F206430B4433F83230C3F30903C4F8E1
:107A1000443263B1B4F82E22D4F83C1200F064FF73
:107A2000D4F83C32D4F844221344C4F83C32002148
:107A3000204601F055FA2268D4F83832B2F85010D6
:107A400002F2064589B253B96B5A23F440639B0492
:107A50009B0C6FEA43436FEA53436B5207E03D2BA5
:107A600010D85808DE0748BF0130800268521388DA
:107A70000BEA030383F4405343F4004343F08003D1
:107A800013808BE658485B0940EA8323E5E73EB262
:107A900030F826901FFA89F919F4004F3DD030F8DC
:107AA000263023F070031B051B0D4FEA471820F802
:107AB000263004EB080191F83432002B53D1B0F892
:107AC000505091F8282200F206432B4433F83250EC
:107AD000C5F3090535B1B1F82E22D1F83C122B4679
:107AE00000F002FF04EB461304EB0801D3F8442234
:107AF0002A44C3F84422D1F83C222A44C1F83C224B
:107B0000D3F840321BB1D1F8380285425ED2A0448E
:107B1000204698F8281201F0E3F919F0800F3FF49D
:107B20003DAE236833F826200AEA020223F8262015
:107B300004EB4717B3F8501097F8282003F20243DC
:107B40000B4404EB461633F83220C2F30902726488
:107B5000FB6B97F828101A44FA63336C2046DBBBA2
:107B600001F0D0F91AE691F8283230F82350DA0003
:107B7000B0F850306D04034413441DD5B3F80254DB
:107B8000C5F3090535B1B1F830222B46D1F83C12C6
:107B900000F0AAFE04EB0803226893F8281232F8DA
:107BA000213023F4E04323F0700343F4004343F017
:107BB000C00322F8213095E7B3F80654C5F3090550
:107BC000002DE7D02B46B1F83222DFE791F82812DA
:107BD0002046FFF7A0FDA0E7FFF7BDFDDEE520464C
:107BE00001F0A8F98AE600BF0080FFFF0F8FFFFFBA
:107BF0008FBFFFFF38B5436801F00F059D42044673
:107C00002DD811F0800F4FF020031ED000EB45124D
:107C100003FB05030121283382F8291001229A7001
:107C20001D7094F8281491421BD084F8282419461A
:107C3000206800F007FD25B904F58661206800F092
:107C400074FD002084F8280438BD03FB010300EB19
:107C50004111002203F50A7381F82922DEE7012091
:107C6000F2E70220F0E738B5044601F00F00636840
:107C7000984224D8430111F0800F1A4617D02244AD
:107C800003F128010123214482F8293000258D7059
:107C9000087094F82834012B13D0012384F8283479
:107CA000206800F0EBFC84F82854284638BD2244B4
:107CB00003F50A710023214482F82932E6E7012006
:107CC000F4E70220F2E711F0800F1BBF01F00F0173
:107CD00000EB411000EB4110283008BF00F50A709E
:107CE00099B21AB90273C180002070470122027351
:107CF0008360F9E703680122C0F86C24B3F85820C8
:107D000042F00102A3F85820B3F8582042F00202D2
:107D1000A3F8582000207047036802460121C0F8EC
:107D20006814002082F86004B3F854200A43A3F8D2
:107D30005420B3F8542042F00202A3F854207047B4
:107D400070472DE9F04F0A6892FAA2F44D68B4FA30
:107D500084F405F1FF3C4FF0010803264FF00F0EAD
:107D600032FA04F30CD1BCF1010F06D84368C9689C
:107D700023EA02034A43134343600120BDE8F08F26
:107D800008FA04F3134062D0D0F800A093FAA3F9E4
:107D9000B9FA89F993FAA3F7B7FA87F74FEA4909CD
:107DA00006FA09F97F002AEA090905FA07F749EAFC
:107DB0000707BCF1010F076016D8876893FAA3F98B
:107DC000B9FA89F993FAA3FA4FEA490906FA09F9C7
:107DD00027EA0909BAFA8AFA8F684FEA4A0A07FAC3
:107DE0000AF749EA07078760C76893FAA3F9B9FA5F
:107DF00089F993FAA3FA4FEA490906FA09F927EA39
:107E00000909BAFA8AFA0F694FEA4A0A07FA0AF721
:107E100049EA0707022DC76019D1FF2BD1F814904A
:107E200017D8D0F820A093FAA3FBBBFA8BFB93FAE8
:107E3000A3F7B7FA87F74FEA8B030EFA03F3BF00F5
:107E40002AEA030309FA07F943EA09030362013442
:107E500086E7476A1B0A93FAA3FABAFA8AFA93FAF0
:107E6000A3F3B3FA83F34FEA8A0A0EFA0AFA9B00E5
:107E700027EA0A0709FA03F947EA09074762E6E72A
:107E80001A4A0368904210B502D0B0F1804F09D170
:107E90004C6823F07003904243EA040309D0B0F128
:107EA000804F06D0124A904203D002F58062904281
:107EB00003D1CA6823F44073134303608B68C36221
:107EC0000B888362094B984207D003F5A053984270
:107ED00003D003F58063984201D10B7C03634369AF
:107EE00043F001034361012010BD00BF002C01409D
:107EF00000400140B1F5807F30B500F0B58005D875
:107F000001293BD0102973D0002030BDB1F5803F4E
:107F100000F0E580B1F5801F00F00D81B1F5805FC4
:107F2000F2D1036A156823F480530362036A44683C
:107F3000C16921F0807121F4E64141EA052115690A
:107F400023F4005343EA0533556823F4805343EA8E
:107F500005338F4DA84207D005F5A055A84203D0A0
:107F600005F58065A84204D1956924F4804444EA6B
:107F70008514D2684460C161026436E0036A156802
:107F800023F001030362036A4168846924F48034A6
:107F900024F073042C43156923F002032B43556826
:107FA00023F001032B437A4DA84207D005F5A055D5
:107FB000A84203D005F58065A84212D1556923F087
:107FC000080343EA8503956823F0040343EA850325
:107FD000956921F480712943D56921F4007141EA42
:107FE0004501D268416084614263036201208CE7ED
:107FF000036A156823F010030362036A4168846909
:1080000024F0807424F4E64444EA0524156923F03E
:10801000200343EA0513556823F0100343EA0513D0
:108020005B4DA84207D005F5A055A84203D005F541
:108030008065A84213D1556923F0800343EA851374
:10804000956823F0400343EA8513956921F4806124
:1080500041EA8501D56921F4006141EAC501D26890
:10806000416084618263C0E7036A156823F480730A
:108070000362036A4168C46924F4803424F0730401
:108080002C43156923F4007343EA0523556823F450
:10809000807343EA05233E4DA84207D005F5A0555D
:1080A000A84203D005F58065A84213D1556923F491
:1080B000006343EA8523956823F4806343EA8523BC
:1080C000956921F4805141EA0511D56921F40051E7
:1080D00041EA4511D2684160C461C26385E7036A21
:1080E000146823F480330362036A416D21F4803104
:1080F00021F070010C43116923F4003343EA01437A
:10810000516823F4803343EA01432149884207D070
:1081100001F5A051884203D001F58061884206D163
:108120004168956921F4803141EA05214160D268B6
:108130004465826559E7036A146823F48013036277
:10814000036A416D21F0807121F4E04141EA042489
:10815000116923F4001343EA0153516823F4801397
:1081600043EA01530A49884207D001F5A0518842E9
:1081700003D001F58061884206D14168956921F4F8
:10818000802141EA85214160D2684465C2652CE7BF
:10819000002C014084B001A880E80E0004B000204B
:1081A0007047B0F8403043F43F4343F08003A0F8F9
:1081B000403000207047B0F8403023F47E535B0419
:1081C0005B0CA0F84030002070470020704784B05E
:1081D00010B503AC84E80E0000220123A0F8403063
:1081E000BDE81040A0F84020A0F84420A0F850209E
:1081F000B0F8403043F43F4343F08003A0F84030F0
:1082000004B0104670470000F0B50C7830F8242018
:108210000346C87822F4EC4222F0700203284CD8BE
:10822000DFE800F00248464442F4007223F82420BC
:108230000E789E4C35B233F825202240324342F46A
:10824000004242F0800223F825200D7B0A78002DA1
:108250007DD1CE884F7876080825760015FB02324E
:108260006FB3B3F850502A44A2F800640D7833F885
:108270002520560608D533F82520144044F4004440
:1082800044F0C00423F82540CA780C78012A33F85A
:108290002410874A02EA010218BF82F0200242F449
:1082A000004242F0800223F82420F0BD42F4C06274
:1082B0000020BBE742F48062FAE70120B6E7B3F89A
:1082C000504022440C69A2F804640A78B3F8506064
:1082D00015FB0232B6B202F2064254B9945B24F4A2
:1082E0004064A404A40C6FEA44446FEA54449453D9
:1082F00007E03D2C26D86508E40748BF0135AD02EC
:1083000095530C7833F8242052040BD533F82420ED
:1083100022F4E04222F0700242F4404242F0800235
:1083200023F82420097833F8212022F4804222F017
:10833000700282F4405242F4004242F0800223F87C
:108340002120B2E75B4D640945EA8424CFE712B2ED
:1083500033F82250254045F4014545F0800523F8C7
:1083600022500D78B3F85060082212FB05353544D1
:108370000E8926F00106A5F800640E78B3F8505077
:1083800012FB06322A444D8925F00105A2F8045457
:108390000A784D7812B2002D43D133F822506F0481
:1083A00008D533F822502C4044F4404444F0800473
:1083B00023F822400C7833F8242056060BD533F8E6
:1083C000242022F4E04222F0700242F4004242F003
:1083D000C00223F824200C7833F8242022F4E04251
:1083E00022F0700242F4004242F0C00223F824203E
:1083F0000D7833F8252022F4804222F0700248F2F2
:10840000800482F44052224323F82520097833F86F
:10841000212022F4E04222F04002144323F82140BC
:1084200043E733F822506D0408D533F822502C402E
:1084300044F4404444F0800423F822400C7833F89C
:10844000242052060BD533F8242022F4E04222F0F7
:10845000700242F4004242F0C00223F824200C785B
:1084600033F8242022F4E04222F0700242F4404229
:1084700042F0800223F824200C78CA7824B2012A22
:1084800033F824500A4A02EA050218BF82F020029B
:1084900042F4004242F0800223F82420097833F8A5
:1084A000212022F4804222F0700244E78F8FFFFFE8
:1084B000BF8FFFFF0080FFFF10B50C7B4A780B7861
:1084C000BCBBF2B130F8232052060BD530F8232084
:1084D00022F4E04222F0700242F4004242F0C00274
:1084E00020F823200A7830F8223023F4E04323F0E8
:1084F000400343F4004343F0800320F8223000207F
:1085000010BD30F8232054040BD530F8232022F47A
:10851000E04222F0700242F4404242F0800220F831
:1085200023200A7830F8223023F4804323F07003AC
:10853000DFE7002A44D130F8232052040BD530F86D
:10854000232022F4E04222F0700242F4404242F042
:10855000800220F823200A7830F822305C060BD500
:1085600030F8223023F4E04323F0700343F4004357
:1085700043F0C00320F822300A7830F8223023F488
:10858000E04323F0700343F4004343F0C00320F8BA
:1085900022300C7830F8243023F4804323F0700329
:1085A00048F28002134320F82430097830F8213053
:1085B00023F4E04323F040031A4320F821209EE7F0
:1085C00030F8232052040BD530F8232022F4E04267
:1085D00022F0700242F4404242F0800220F8232050
:1085E0000A7830F822305B060BD530F8223023F4BD
:1085F000E04323F0700343F4004343F0C00320F84A
:1086000022300A7830F8223023F4E04323F070035C
:1086100043F4404343F0800320F822300C7830F8D4
:10862000243023F4E04323F0400348F28002134354
:1086300020F82430097830F8213023F4804323F0E7
:108640007003B9E74B780A787BB130F8223023F415
:10865000E04323F0400383F0100343F4004343F06E
:10866000800320F822300020704730F8223023F4B5
:10867000804323F0700383F48053EEE74B780A784D
:1086800003B330F822305B060BD530F8223023F4E8
:10869000E04323F0700343F4004343F0C00320F8A9
:1086A00022300A7830F8223023F4E04323F04003EC
:1086B00083F0300343F4004343F0800320F822307A
:1086C0000020704730F822305B040BD530F82230A0
:1086D00023F4E04323F0700343F4404343F080036A
:1086E00020F822300A7830F8223023F4804323F037
:1086F000700383F44053DDE711B98023A0F84C30B8
:1087000000207047B0F8583043F40043A0F85830C8
:1087100000207047B0F85830C3F30E03A0F858306B
:1087200000207047B0F8440070470020704702F501
:108730008062013302445B0801EB4303521A994201
:1087400000D17047088850520231F8E7F8B5044666
:1087500048788E690A690F7B01280D4659D19642E7
:108760008ABFB11A00211646A961B6B26969EFB98C
:108770003346EA882046FFF7DAFFB4F850102A782B
:1087800004F202430B4423F832602A7834F8223092
:1087900023F4E04323F0400383F0300343F4004329
:1087A00043F0800324F822300020F8BD2B7834F801
:1087B0002300DA00B4F850302344134447064BBF7B
:1087C000A3F80664A3F802646A892A89334620461E
:1087D000FFF7ADFF6A782B786AB91BB234F8232013
:1087E00022F4E04222F0700242F4004242F0C00261
:1087F00024F82320C9E7012AC7D11BB234F823206B
:1088000022F4E04222F0700242F4404242F0800240
:10881000EEE796428CBFB11A0021A96188BF1646C7
:10882000297897B9B4F8500004F20642024402EBEA
:10883000C102AEBB138823F440639B049B0C6FEA18
:1088400043436FEA5343138032E088B9B4F85000D1
:1088500004F20242024402EBC102A6B9118821F4DB
:1088600040618904890C6FEA41416FEA51411180EE
:108870006A7828785ABBB4F8501004F206420A44C9
:1088800002EBC002D5E73D2E05D87108F00748BFBE
:1088900001318902EBE71348710940EA8121E6E7DB
:1088A0003D2E0FD87108F30748BF013189021180AE
:1088B0002A7834F8223023F4804323F0700383F4C1
:1088C00040536BE7074B710943EA8123BBE7012A59
:1088D00001BFB4F8502004F20641891821F8306035
:1088E000E6E700BF0080FFFF02F58062F0B51044AC
:1088F0005D080C462E46471A3A19023436B9DB0792
:1089000044BF30F8153001F81530F0BD128804F876
:10891000022C120A04F8012C013EEDE74FF47A73A1
:10892000B0FBF3F0034B0022013858609A60052237
:108930001A60704710E000E0014B1860704700BFFC
:108940004000002003685B0670B526D4D1E90036EC
:108950003343CE684D6904680A6A33430E69334372
:108960008E692B433343CE6924F47F44334324F090
:10897000BF0413432343036044688B6824F470648A
:1089800043EA154324F004042343B2F5005F436037
:1089900001D18B8C0361012000E0002070BD00003C
:1089A0000146D0E90032007A30B5002800F082801C
:1089B000002B4AD04C7A012C29D060B2F0B1022CA5
:1089C0002FD001208C7A6CB1022C2ED0032C35D004
:1089D000012C37D1404CE56825EA0305E560A56820
:1089E0002B43A360002A4AD04B7A012B48D0002B9E
:1089F0002DD0022B4DD040F0040030E0364C65689D
:108A000025EA0305656025681D432560DAE73248DD
:108A1000046824EA0304046044681C4344600020A2
:108A2000D0E72D4804681C43F5E72B4CA56825EAE0
:108A30000305A560E5682B43E360D3E7264CA568F2
:108A40001D43F6E740F00200CCE71846CAE7224B88
:108A50005C6A24EA02045C621C6A14431C628B7A1E
:108A60006BB1022B19D0032B20D0012B32D11A4B22
:108A7000D96A21EA0201D962996A0A439A6230BD31
:108A8000154B1C6A24EA02041C625C6A14435C6293
:108A9000E5E7114B1C6A1443F6E70F4B996A21EA8C
:108AA00002019962D96A0A43DA62E8E70A4B996AD5
:108AB0001143F6E708490C68DB431C400C604C6826
:108AC00023404B600B6AD24313400B624B6A1A403F
:108AD0004A62D4E70020D2E700040140D0F8943283
:108AE00010B56BB1D0F8904294F84000FF2807D041
:108AF0009B6894F8412021469847FF2384F8403032
:108B0000002010BD38B50546D0F8904200F0D5FAE7
:108B1000D5F89032E06443B1D5F89432606CDB68EC
:108B200004F14C019847002038BD0220FCE7F8B55D
:108B3000D0F89062C6B1142303FB0103DA6982B155
:108B4000D0F8984204EB4114A56BB2FBF5F405FB99
:108B5000142434B9DC612246234600F0A0FA2046F2
:108B6000F8BD00207065FBE70220F9E72DE9F74327
:108B70000A78D0F890724FF0000812F060040546B1
:108B80000E468DF80580ADF8068028D0202C5ED1E9
:108B9000CC884B78E4B1120611D5D0F8942239462E
:108BA000D2F8089018462246C847F2883946284627
:108BB00000F0B2FB4446204603B0BDE8F08387F8DE
:108BC000403087F841402246394600F0BAFBF1E7D1
:108BD000D0F89422184695682246A847EBE74F78CC
:108BE0000B2F34D801A353F827F000BF1D8C0008C9
:108BF0004F8C00084F8C00084F8C00084F8C0008E9
:108C00004F8C0008B78B00084F8C00084F8C000871
:108C10004F8C0008338C0008478C000890F87432A1
:108C2000032B14D102220DF1060100F075FB3C4626
:108C3000C1E790F87432032B09D101220DF105012F
:108C400000F06AFBB7E790F87432032BB3D03146DB
:108C5000284600F08AFD0224ADE700BF38B504467F
:108C60000025822100F0EFF902212564204600F062
:108C7000EAF9C4F86C518321204600F0E4F9D4F8F5
:108C8000903265652BB1D4F894325B689847C4F88C
:108C90009052002038BD000070B5402304460222E7
:108CA000822100F0C6F901250222256411464023E5
:108CB000204600F0BEF9C4F86C510322832108233A
:108CC000204600F0B6F9D4F894326565074DC4F833
:108CD00090521B689847002640236A6C6E650221FB
:108CE0002046AE6500F0E2F9304670BDE82700206E
:108CF000F8B50A4D06460F46002455F8043B23B943
:108D00000134032CF9D10020F8BD1B6839463046E8
:108D100098470028F4D00220F6E700BF442800203E
:108D2000F8B50A4D06460F46002455F8043B23B912
:108D30000134032CF9D10020F8BD5B683946304678
:108D400098470028F4D00220F6E700BF442800200E
:108D50000B792DE9F04106460D4663B9174B1B68A8
:108D60002C7814F0600408D0202C25D1F3B902240B
:108D70002046BDE8F0810023F2E76A78062A04D095
:108D8000F6D30A3A012AF1D9F2E7DFF83080274614
:108D900058F8043B1BB90137032FF9D1E8E79B686A
:108DA0002946304698470028F5D0E0E72946304666
:108DB0009B68BDE8F04118470024D9E7442800200B
:108DC000054B53F82120054B53F822300BB15B695A
:108DD00018470220704700BF704C00204428002034
:108DE000054B53F82120054B53F822300BB19B69FA
:108DF00018470220704700BF304C00204428002054
:108E000070B50A4D0646002455F8043B23B90134D9
:108E1000032CF9D1002070BD1B69002BF7D0304620
:108E200098470028F3D00220F5E700BF442800202F
:108E300029230380004870477C0000200A23038018
:108E400000487047E0000020292303800048704755
:108E50007C00002029230380004870477C0000200C
:108E6000034B0022C3E90122DA601860704700BF9B
:108E700044280020144A936D43F08063936583690E
:108E8000012B01BFA2F58632136843F480231360DF
:108E90000E4BDA68C2F30222C2F10701131D042946
:108EA00028BF0421062B4FF0FF3303FA01F38CBFD8
:108EB000033A0022DB4393401B01054ADBB282F8F0
:108EC00043330823936070470010024000ED00E038
:108ED00000E100E000F58661D0F8700400F026B9EA
:108EE00000EB411310B5D3F83C22D0F870040C46C7
:108EF00000F049F9012C04D12046BDE8104000F0F3
:108F000093BD10BD00EB4113D0F87004DA6B00F094
:108F100072B9D0F8700400F0F3B910B5044601211D
:108F2000D0F8700400F0E9F9D4F87004BDE81040FE
:108F300000F0BCB970477047364A536843F4806309
:108F400010B553600446344A34480823C0E900236E
:108F5000C0F8704400230222C4F89802C0E902233A
:108F6000C0E90423C0E906330362FEF7DDFA18B155
:108F7000FE212B48FDF760FA002211461823D4F891
:108F80009802FEF7A0FE582300228021D4F8980210
:108F9000FEF799FE982300220121D4F89802FEF7EB
:108FA00092FED82300228121D4F89802FEF78BFE8E
:108FB0004FF48C7300220421D4F89802FEF783FE4C
:108FC0004FF4AC7300228621D4F89802FEF77BFEA2
:108FD0004FF4CC7300228521D4F89802FEF773FE7B
:108FE0004FF4EC7300228321D4F89802FEF76BFE55
:108FF0004FF4067300220221D4F89802FEF763FEB4
:109000004FF4167300228221D4F89802FEF75BFE1B
:10901000002010BD0070004000680040B04C0020EF
:10902000053E010808B5D0F89802FEF7EFFA0020D7
:1090300008BD10B51C46D0F8980213462246FEF72C
:109040000EFB002010BD08B5D0F89802FEF73AFBE1
:10905000002008BD08B5D0F89802FEF7CBFD00202F
:1090600008BD08B5D0F89802FEF7FDFD002008BD48
:109070000A06D0F8983245BF01F07F0103EB411397
:1090800003EB411393F82A0058BF93F82A02704764
:1090900008B5D0F89802FEF7CEFA002008BD08B552
:1090A000D0F89802FEF757FB002008BD08B5D0F8AD
:1090B0009802FEF730FB002008BD08B5D0F89802F2
:1090C000FEF742FB08BD08B580B1D0F88C3213B171
:1090D0000023C0F88C3209B1C0F88812012380F84F
:1090E00074320270FFF728FF002008BD0220FCE761
:1090F00019B1C0F88C12002070470220704708B5E3
:10910000FFF790FF002008BD08B5D0F88C320BB9EE
:10911000022008BD1B6898470028FAD0F8E708B578
:10912000D0F88C325B689847002008BD38B50446FB
:1091300000F52075284600F004FB012394F8801206
:10914000C4F86C32B4F88632C4F8703201F01F03F0
:10915000012B0ED03BB1022B10D001F08001204634
:10916000FFF778FF03E02946204600F021F90020B0
:1091700038BD2946204600F037FAF8E72946204650
:1091800000F057FAF3E770B5044616460D4629BBC2
:10919000D0F86C32032B1CD1D0E9533293420BD957
:1091A0009B1A9A42C0F84C318CBF9AB292B23146A7
:1091B00000F0D4F8284670BDD0F88C321B6923B17A
:1091C00090F87422032A00D19847204600F0CEF888
:1091D000F0E7052BEED1FFF73DFFEBE7D0F88C323F
:1091E0009B6933B190F87422032A02D19847002575
:1091F000E0E70225DEE770B5044616460D46002975
:1092000047D1D0F86C32022B3CD1D0E908329342DE
:1092100014D99A1A0262314692B200F08AF82B46AB
:109220002A4629462046FFF741FF94F87832012B61
:1092300002D1002384F87832284670BDC369B3FB9D
:10924000F2F602FB16365EB99A4209D8D0F87022BF
:10925000934205D20A4600F06CF8C4F87052DEE77B
:10926000D4F88C32DB682BB194F87422032A01D134
:109270002046984780212046FFF7ECFE204600F06C
:1092800080F8D2E733F00403CFD18021FFF7E2FE6C
:10929000CBE7D0F88C325B6933B190F87422032AA3
:1092A00002D198470025C7E70225C5E770B500221F
:1092B00004461146012540264023FFF7BAFE3346F7
:1092C0008021C4F84451C4F8506100222046FFF7C1
:1092D000B0FED4F89032A5610021666284F8745221
:1092E000C4F86C126160C4F87C1223B1D4F88C32DB
:1092F00020465B689847002070BD017400207047CD
:1093000008B590F87422032A04D1D0F88C32DB69B6
:1093100003B19847002008BD10B513460222C0F8DB
:109320006C22C0E907330A460021FFF7B8FE00208F
:1093300010BD08B513460A460021FFF7B0FE002015
:1093400008BD10B513460322C0F86C22C0E95233A1
:109350000A460021FFF7AAFE002010BD08B51346FB
:109360000A460021FFF7A2FE002008BD08B504232D
:10937000C0F86C3200231A461946FFF790FE002011
:1093800008BD08B50523C0F86C3200231A461946FB
:10939000FFF78CFE002008BD10B580210446FFF7C2
:1093A00059FE20460021BDE81040FFF753BE0000E3
:1093B00037B50B7803F06003202B04460D4614D01C
:1093C000402B12D0002B40F08E804B78092B00F2FE
:1093D0008A80DFE813F0E300FC008800F5008800D5
:1093E0007D0013008800CE009B00D4F88C32294603
:1093F0009B6820469847002003B030BD4B881A0A6E
:10940000013A062A6FD8DFE802F00416236E6E4395
:109410004C00D0F888321B68207C0DF1060198477B
:10942000BDF80620002A4FD0EB88002B43D1204600
:10943000FFF79CFFDFE7027CD0F88C3232B99B6AE1
:109440000DF10600984702234370E9E7DB6AF7E76E
:10945000DBB2052B47D8DFE803F003070B0F131728
:10946000D0F888325B68D7E7D0F888329B68D3E7BA
:10947000D0F88832DB68CFE7D0F888321B69CBE7B9
:10948000D0F888325B69C7E7D0F888329B69C3E7B8
:10949000037C43BBD0F88C320DF106005B6B984720
:1094A000BEE7037CFBB9D0F88C320DF106001B6BD4
:1094B00098470723C8E79A4228BF1A460146204624
:1094C000ADF80620FFF728FFEB88002B93D1AEE71D
:1094D0008B8843B9CB8833B94D887F2D03D890F85A
:1094E0007432032B03D12046FFF756FF83E7E9B21E
:1094F00080F87612FFF7CCFD2046FFF737FF1DB14D
:10950000022384F8743276E70123FAE78978354D2F
:1095100001292970E7D890F87432022B08D0032B68
:1095200015D0FFF739FF29782046FFF7F8FD62E7ED
:1095300000293FF47CAF01210323416080F874329D
:109540002046FFF7E1FD02287FF471AFCBE731B988
:10955000022380F874324160FFF7E1FD67E741685C
:1095600001293FF464AFC9B2FFF7D9FD29786160E2
:10957000E6E7CA88012AB6D190F87432002BB2D03F
:10958000022B03D9032BAED1011D03E001460023BA
:1095900041F8083F2046FFF7BFFE2CE790F87432F1
:1095A000013B022B9FD8CA88022A9CD1D0F87C327A
:1095B0000146002B14BF1346002341F80C3FE9E796
:1095C0004B88012B7FF417AFC4F87C322FE790F85B
:1095D0007432013B022B86D84B88012B7FF40BAFF2
:1095E0000023F1E75428002038B50B7803F060031E
:1095F000202B04460D4602D0402B00D0ABB994F886
:109600007432013B022B10D82B79012B0DD8D4F8E2
:109610008C3229469B6820469847EB881BB910B9C5
:109620002046FFF7A3FE002038BD2046FFF7B4FE1A
:10963000F9E738B50A7802F06002202A04460B46A2
:1096400015D0402A13D072B95A788D88012AE9B210
:1096500021D0002A36D0032A05D190F87422022A9C
:1096600027D0032A0BD02046FFF796FE05E0D4F85A
:109670008C221946926820469047002038BD5A88AF
:109680002AB94A0603D0DB880BB9FFF7E3FC204672
:10969000FFF76CFEF1E790F87422022A09D0032A42
:1096A000E1D15B88002BE8D14D06F0D0FFF7D9FC63
:1096B000EDE74B06D7D0FFF7CDFC80212046FFF722
:1096C000C9FCDAE790F87432022B18D0032BCAD108
:1096D00001F00F02142315F0800F03FB02021DD0CE
:1096E0009269002ABFD001F07F0505FB03350544D0
:1096F00011F07F031DD12B60022229460AE04A06A1
:10970000B1D12B064CBF00F1140100F5A07100236C
:109710000B6002222046FFF7FFFDAEE7D2F844219E
:10972000002AA0D001F07F0503FB050505F5A07513
:10973000DEE72046FFF79CFC08B10123DBE7286049
:10974000DAE70B7803704B784370CA788B7803EBB9
:10975000022343804A790B7903EB02238380CA7981
:109760008B7903EB0223C380704710B58021044638
:10977000FFF770FC20460021BDE81040FFF76ABCEF
:1097800030B588B1042A0FD900220138551C445D38
:109790005CB9D2B2013252001A8003234B700A70B6
:1097A000022310F8015F15B930BD2A46EEE75A1CB6
:1097B000D2B2CD540233DBB28C54F2E712230B80C9
:1097C000004870471A3E010804230B800048704788
:1097D0005C3E010810B5044C04480B46302221467B
:1097E000FFF7CEFF204610BD24510020353E010872
:1097F00010B5044C04480B4630222146FFF7C0FF49
:10980000204610BD245100202C3E010870B5254A89
:109810008CB00B4607AC02F1100610685168254663
:1098200003C50832B2422C46F7D112782A701E497D
:109830001E4C00228DF81820C87A8DF804001C48B0
:109840000078247820448DF80500487A8DF80600C9
:10985000184800780C7820448DF80700C8798DF8F6
:10986000080089798DF8091003AC01AD204615F880
:10987000011B0CAE06EB111601F00F0116F8146C6B
:1098800026700CAE3144013211F8141C6170062AA6
:1098900004F10204EBD130220749FFF771FF0648BB
:1098A0000CB070BD4B3E01089075FF1F9275FF1FF5
:1098B0009A75FF1F9875FF1F2451002029230380EC
:1098C000004870477C010020D0F8903200201873C7
:1098D000704700000A230380004870477001002091
:1098E00037B50022ADF806200C78CA88D0F890323F
:1098F00002F07F0214F06004CA801ED0202C32D106
:109900004A78023A092A2ED8DFE802F0140B2D2DEE
:109910002D2D2D2D10058A781A600024204603B0C5
:1099200030BD01221946FFF7F7FCF6E74A88120A14
:109930005A60F2E70122191DF5E74D780B2D12D878
:10994000DFE805F006111111111115111111272F62
:1099500090F87432032B06D102220DF10601FFF7B5
:10996000DBFC2C46DAE7FFF700FF0224D6E74B8842
:109970001B0A222B06D1222A0D4928BF2222FFF7DB
:10998000CBFCCBE7212BEED1092A28BF09220949BC
:10999000F5E790F87422032AE5D1012203F10801CA
:1099A000EDE790F87422032ADDD18A789A60B5E752
:1099B000080100206401002010B581210446FFF752
:1099C00042FB01212046FFF73EFB0020E062C4F885
:1099D000580110BD10B54023044603228121FFF732
:1099E00028FB4023032201212046FFF722FB01210F
:1099F000074BE162C4F85811C4F8903200241C737C
:109A0000044A05484023FFF751FB204610BD00BF24
:109A1000952800205528002094490020D0F8903245
:109A2000002018737047000070B5094C402520468F
:109A3000FCF704FD2A460021204608F087FC2B464F
:109A4000224601210348BDE87040FFF72FBB00BF4D
:109A5000552800209449002000207047D0F890320B
:109A6000002058657047002070470000F7B50F7858
:109A7000D0F89062002517F0600403468DF8055079
:109A8000ADF8065016D0202C48D1CA88002A4AD0FA
:109A90003B0603D53146FFF73FFC07E04B7886F8DD
:109AA000403086F841203146FFF74BFC2C462046DB
:109AB00003B0F0BD4D780B2D30D801A252F825F03F
:109AC000F19A00081D9B00081D9B00081D9B0008C3
:109AD0001D9B00081D9B0008AF9A00081D9B0008F5
:109AE0001D9B00081D9B0008019B0008159B00089A
:109AF00090F87422032A11D102220DF10601CAE75F
:109B000090F87422032A09D101220DF10501FFF713
:109B100003FCCCE790F87422032AC8D01846FFF75C
:109B200024FE0224C3E71446C1E700BF38B504464B
:109B300000258621FFF787FA0421C4F890502046BB
:109B4000FFF781FAC4F8945185212046FFF77BFA8C
:109B5000D4F89032E5670BB1C4F89052002038BDBC
:109B600038B50222044640238621FFF762FA012518
:109B70004023022204212046FFF75BFAC4F89050EC
:109B8000C4F894514023032285212046FFF751FA5F
:109B9000074BE567C4F8903200245C65054A9C6574
:109BA000042140230448FFF781FA204638BD00BF56
:109BB000E8280020A52800209449002070B503461D
:109BC000007820F0100010705878507098789070DD
:109BD000D878D0700020107150719071D0711072CF
:109BE00050729072D072107350739073D0730429B6
:109BF000187904D10124D473062947D117E0052927
:109C000019D0441D8C421FD0841D8C4222D10028C3
:109C10003CD00424D4735C18908014F8014C002CC0
:109C200040F0868001259472D572147354730539FF
:109C300081422BD21AE00224D47310B1C2F80A0078
:109C4000E2E70124D472DFE70028DDD00324D473D7
:109C50009080D9E70629D0D90028E8D15C79987995
:109C600000EB042080B2CC1F844202D24FF4CE40DD
:109C700070BD07291AD11224D4730124947358B1EA
:109C8000C2F80A0000F10A048C422BD0D17B0029D3
:109C900040D146F68510EBE79072D0721473507382
:109CA0001324D47301249473908002E0C41D8C4269
:109CB000F6D000F109048C42E4D11424D4730125B8
:109CC0005C189573908014F8026C14F8014C14EB36
:109CD000062411BFC2F80A409472D472157308BFEB
:109CE0005473CFE7194411F8034C002CCED124242F
:109CF000D47301249473908011F8020C11F8011CA4
:109D000011EB002111BFC2F80A109172D1721473C5
:109D100008BF517390880028AAD0907B20B10733E8
:109D2000C2F806300020A3E70533C2F806309FE7EB
:109D3000C2F80A407BE770B50D4688B000210646A0
:109D4000144608466A4603F00DFD202106F1100076
:109D500003F0FAFC2846202103F0F6FC00216A46B5
:109D6000084603F02FFD04AD6B4622461C4603CC8B
:109D7000AC4210605160234602F10802F6D108B0EF
:109D800070BD00000C4B70B51C6841F2020604F572
:109D90008052A35B12880D465918914202DD0120C2
:109DA00008F054FA2A460146E01808F0B5FAA35B19
:109DB0001D44A553002070BD44290020014B1868A4
:109DC00002F012B94429002070B504460E46103046
:109DD00020211546FCF798FA224631462046FFF727
:109DE000AAFF204605F120032A46302103F0E0FDBA
:109DF000002070BD70B5ADF59C6D4FF480630446D6
:109E0000ADF80430FCF768FBB0F5806F054603D968
:109E100030480DF59C6D70BD40F2EE20FCF726FA3F
:109E2000002854D004F1200616AA31460AA8FFF7EC
:109E3000CBFF0130ECD003F06BFC012101A803F053
:109E400083FC3046202103F07FFC2021204603F0D4
:109E50007BFC30210AA803F077FC01210DF10500FD
:109E600003F072FC402116A803F06EFC02A803F078
:109E700073FC03F0F1FC2246202102A803F0FAFC57
:109E80000523022101A88DF80430FFF77BFF402154
:109E900016A8FFF777FF3026012101A88DF804608E
:109EA000FFF770FF31460AA8FFF76CFF38A8FCF7F0
:109EB00019FB294638A8FFF765FF26A9204601F0BF
:109EC00033FA81B226A8FFF75DFF0348A1E746F603
:109ED00085109EE71092FFFF0090FFFF30B54629E6
:109EE00085B00446154617D120222946223008F0B5
:109EF000F7F9C0B96B46D4F8422004F110012846A6
:109F000001F0ECF810226946204608F0E9F9B0FAB1
:109F100080F0400905B030BD302904D16A46294699
:109F2000FFF709FFEEE70020F4E7000007B5084B54
:109F300018689A8800909B79ADF80420062168463D
:109F40008DF80630FFF71EFF024803B05DF804FBF2
:109F5000F33D01080090FFFF2DE9F04107469CB05A
:109F600018461C460D469046654E02F03DF83B787B
:109F70003460002B40F0BE8042462946384603F04C
:109F8000AFFE84B2B4F5104F0ED046F685139C4256
:109F90000AD07B78032B00F0A1801CD8012B24D0A1
:109FA000022B2AD04FF4DA440020FBF7B9FEB4F5B7
:109FB000104F40F0A180230A01210AA88DF8283013
:109FC000FFF7E0FE01210AA88DF82840FFF7DAFE2E
:109FD0001CB0BDE8F081C02B00F08680FF2B0CBFC9
:109FE0004FF410444FF4DA44DEE7B8F1400F7ED16D
:109FF0002846FFF7FFFE84B2D6E7BC780123072C82
:10A000008DF807300FD105F1200295F8401005F1C9
:10A010004100FFF763FF18B146F68514A4B2C3E709
:10A020004FF4D544FAE7032C01D0082CF8D105F100
:10A03000410805F120073A4695F840104046FFF7E1
:10A040004DFF0028ECD000231A4695F840104046FA
:10A0500003F09CFC082C36D100238DF8073000203B
:10A06000FCF770F804BA029403F052FB2021384642
:10A0700003F06AFB01210DF1070003F065FB0421E9
:10A0800002A803F061FB2021284603F05DFB02A833
:10A0900003F062FB2A46202102A803F0EBFB01211A
:10A0A0000DF10700FFF76EFE042102A80294FFF7EE
:10A0B00069FE0AA9284601F037F981B20AA8FFF71C
:10A0C00061FE104CAAE79DF80730002BC7D040F284
:10A0D000EE20FCF7CBF800289ED0C0E7B8F1000FC7
:10A0E00005D1FFF723FF86E74FF410445CE74FF4F8
:10A0F000CE4459E74FF4DC44306801F075FF5AE76D
:10A10000442900200090FFFFF8B50D4616461F4673
:10A11000044668B10120FBF773FD20463B463246FA
:10A120002946FFF719FF0020BDE8F840FBF768BD9E
:10A13000F8BD30B4027943798579120442EA0322EA
:10A140002A430B4630BCC11DFFF706BF094A30B594
:10A150000023182404FB03F18D58854203D10A44DF
:10A160000020107430BD0133092BF3D14FF0FF30C4
:10A17000F8E700BF48290020044A00231380044A5E
:10A180001360044A1360044A13607047F2470020CA
:10A19000FC47002000480020F4470020044B1888AA
:10A1A00028B1044B1B6898420CBF02200120704765
:10A1B000F2470020FC4700200C4A38B51146002326
:10A1C000147C5CB918225343CD18C85001232B745A
:10A1D000FBF722FDC5E90204204638BD0133092BF7
:10A1E00002F11802ECD14FF0FF30F6E748290020C9
:10A1F00038B50C4C0022182303FB02F52959814283
:10A2000009D1FBF709FD631900220121C3E902020C
:10A210001974104638BD0132092AEDD14FF0FF30D4
:10A22000F8E700BF482900202DE9F04704460F4613
:10A23000164600254FF004084FF005094FF0070AB5
:10A24000B54201DBBDE8F087D4E9032362B9626857
:10A25000C4F81520C4F80C80C3B92278627622892C
:10A26000C4F80CA052BA6283E068421CE260204449
:10A27000795D41750133402A236105D104F1150050
:10A28000FBF7BAFE0023E3600135D9E7227D627651
:10A29000511C2175C4F80C90E6E7C36810B55BB992
:10A2A00003694BB94368C0F81530037843760389D6
:10A2B0005BBA43830723C360C368002B0CDD00F146
:10A2C0001504E018C3F14002002108F03FF82046D1
:10A2D000BDE81040FBF790BE10BD10B598B0044625
:10A2E0008DF807105822002102A808F02FF8BF238C
:10A2F00001220DF1070102A88DF80830ADF81020F9
:10A300000394FFF791FF02A8FFF7C7FF18B010BD35
:10A31000FFF732BF2DE9F04DDFF85C80154D0024CA
:10A3200040F2ED2A4FF0000B98F81030D3B1FBF754
:10A3300073FCD8E902320021C61A61EB0207BB4563
:10A3400008BFB2450ED20521D8F80000FFF7C5FFBF
:10A35000002388F81030D8F800202B689A4201D1E9
:10A36000FFF70AFF01340A2C08F11808DCD1BDE818
:10A37000F08D00BFF44700204829002000B599B0B7
:10A3800058228DF80700002102A807F0DFFF0A4BD2
:10A390001B6803930122BB230DF1070102A88DF86E
:10A3A0000830ADF81020FFF73FFF02A8FFF775FF58
:10A3B00019B05DF804FB00BFF4470020F8B514465F
:10A3C000084601F011FE2378D12B18D005D8992B1F
:10A3D0004FF0000531D00020F8BDE02B18D0E12B64
:10A3E000F9D1184E04272781032301253370757096
:10A3F000B370FBF7F5FC3A46F070314617E0FBF717
:10A40000E7FF002323812046FFF747FF0120E3E712
:10A410000C4B1B787BB1238122890A48002107F06D
:10A4200095FF21890748FBF76FFF228905492046E0
:10A43000FFF7FAFEE7E73923EDE7FBF7DFFC2581BD
:10A44000E1E700BF382A00202DE9F04702790668CD
:10A45000862AADF5815D054659D1B0F80530B3F5D2
:10A46000006F03D0002403250327C9E0002E00F06D
:10A47000E080FFF74DFF0768781C12D1AF4B1C68D6
:10A480000134621E033204F1010108D820461C6029
:10A49000FFF792FE013014D100240625E4E70C46B4
:10A4A000EFE7A74A0023182101FB03F080588742F9
:10A4B00000F08A810133092BF6D13846FFF77CFE84
:10A4C00085E15822002107A807F040FF55F8070F43
:10A4D0000897862369688DF81C3002AB019303C38B
:10A4E000019B01999C6002231122CB6007A80523E0
:10A4F000ADF824200B74FFF797FE07A8FFF7CDFEF9
:10A500002046FFF723FE00242546042778E0711C2F
:10A5100000F08F808A49002318200C4600FB03F7C7
:10A520007F58BE420AD00133092BF7D1130605D557
:10A53000FFF734FE10B93046FFF73EFE29680023CE
:10A54000182202FB03F02058814200F042810133BF
:10A55000092BF6D195F90430002BD4DA9CE7002BB7
:10A5600022DAB5F805305BBA9AB241F6B954A24284
:10A570003FF678AF734C2380734B1860734B74486D
:10A580001960392A734B28BF39221A60724B4FF079
:10A59000FF311960E91D07F0BFFE2868FFF728FEAC
:10A5A00038B3012007F052FE002CADD0674B1B687A
:10A5B0009942A8D1634B684AB3F800801368654F8D
:10A5C000013383423C68136040F01381A8EB04021E
:10A5D0005F483B2A204405F1050104DC07F09CFE9E
:10A5E000C7F80080D9E73B223B3407F095FE3C607A
:10A5F000D3E7544B1C88544B1D78FFF7CFFD07461B
:10A60000564B58220021184607F0A0FE042F466042
:10A610000570804614D0032F0ED13046FFF796FD0B
:10A62000042D01D1FFF7A8FD29463046FFF755FE5E
:10A6300006E000240B2517E7012F03D1FBF7ECFA06
:10A6400000253BE0A5F18103102B00F2AE8001A2B2
:10A6500052F823F099A60008ABA7000865A70008E8
:10A66000ABA70008ABA70008A3A50008ABA700088C
:10A67000C7A60008ABA70008ABA70008ABA7000857
:10A68000ABA70008ABA70008ABA70008ABA7000862
:10A69000CDA60008B7A70008048122462C492F4800
:10A6A000FFF7C2FD2D48FFF7F8FD3046FFF74EFDDE
:10A6B000FFF762FD2A4B1B78002BC1D128460DF510
:10A6C000815DBDE8F087FBF7A7FCEBE70CB9032140
:10A6D000ABE7234F97F80090B9F1000F01D00621A6
:10A6E000A3E74FF0010A07A887F800A001F07CFC5F
:10A6F00007AA2146164801F0A9FF0DF580531E3325
:10A7000002901B881548C8F804605344A8F8083024
:10A710005246902302A988F80030FFF785FD0DF519
:10A7200080531E3307A91A880C48FFF77DFD0B489C
:10A73000FFF7B3FD87F80090B7E700BFE001002006
:10A7400048290020F2470020F8470020F447002065
:10A75000382A0020FC47002000480020084800203C
:10A7600004480020002CB2D0234C2778002FB6D10B
:10A77000012307A80DF12009237001F035FC07A97A
:10A780001E48FFF7D6FCB9F8FE2F1D48A8F8082090
:10A79000832307A988F80030C8F80460FFF744FD58
:10A7A0001748FFF77AFD27707FE7154A07A920466B
:10A7B000FFF704FE18B1104B00221A7075E7012153
:10A7C0003046FFF78AFD70E73846FFF711FD3C463B
:10A7D00060E6FFF7E3FC04462879012C43B27FF4DE
:10A7E000BEAE084A126891427FF4B6AE002BBFF6A7
:10A7F000DDAE0024042537E604480020382A002076
:10A8000008480020F4470020D1F84330D0F8430036
:10A81000181A7047F8B5202206460D46223022311C
:10A8200007F05EFD044680B996F8867005F1460192
:10A830003A4606F1460007F053FD20B995F88640E8
:10A84000E31B5C425C412046F8BD0024FBE738B5C1
:10A85000054608460C4608F02FFA214602462846CF
:10A86000BDE8384007F0B5B808B50220FBF758FA44
:10A8700047F24810FBF7FAFC012805DC06D0002857
:10A8800014BF2D203A2008BD2120FCE70020FAE764
:10A8900020210148FBF738BD6048002010B5044670
:10A8A0000020FBF74FFC034610B9FBF74BFC0346B7
:10A8B0001A0E84F821201A0C84F822201A0A84F82F
:10A8C000232084F82430184610BD00002DE9F04301
:10A8D0000678022EB1B004468846154640F0AA809C
:10A8E00008AA7149683002F0E1FF02F011FF20214F
:10A8F0000DEB010002F028FF08A802F02DFF202137
:10A9000010AA0DEB010004F1050902F02BFF2179DB
:10A91000484602F019FF20210DEB010010AA02F0B9
:10A9200051FF102210A904F1450007F0D9FC074699
:10A93000002840F0B68018AA0146304602F012FF07
:10A940004621D4F8B00002F0FFFE18AA394630467E
:10A9500002F038FF394608A802F0B6FF21794846D0
:10A9600002F0D8FF20AA202118A802F0FBFE202127
:10A97000484602F0E9FE20AA202118A802F022FF92
:10A980002379402B0ED128AA202118A802F0EAFE34
:10A99000202104F1250002F0D7FE28AA202118A8C2
:10A9A00002F010FF002108A802F08EFF217920A8F4
:10A9B00002F0B8FF00232A684146684606F0B8FF57
:10A9C000012204A9684607F01DF8384A064640F2FD
:10A9D000831101F089FF002E5ED1354904A8FFF7ED
:10A9E00036FF324A06464FF4C37101F07DFF002E58
:10A9F00052D1227920A904A806F0D6FF2B4A04469A
:10AA000040F2891101F070FF002C45D104A968467D
:10AA100007F00AF8254A04464FF4C67101F064FFB6
:10AA2000002C39D10099A1EB08012960204631B0F2
:10AA3000BDE8F083012E31D100231268684606F08C
:10AA400077FF324620A9684606F0DCFF174A044625
:10AA50004FF4CB7101F048FFF4B9154920A8FFF776
:10AA6000F6FE124A044640F2991101F03DFF9CB9EE
:10AA7000152120A806F083FF0C4A04464FF4CE713E
:10AA800001F032FF44B920A9684606F0CDFF074A1D
:10AA9000044640F29F11C1E71024C7E70024146068
:10AAA000C4E7E024C2E700BF60480020BA3E0108C6
:10AAB000CD3E010838B5114CD022FF21204607F0C9
:10AAC00045FC802104F14E00FBF71EFC082384F8AE
:10AAD0004830A523238001250023A4F84A3084F8B8
:10AAE000CE50FBF716FC202104F12200FBF70CFCF2
:10AAF000A84202D0284607F0A9FB38BD306F0020DD
:10AB00002DE9FF410E4615466946052204461F46BB
:10AB100006F078FF494A8046CD2101F0E5FEB8F104
:10AB2000000F40F0868001220023684606F015FFE2
:10AB3000424A8046D22101F0D7FEB8F1000F78D109
:10AB400002220023684606F008FF3C4A8046D421D2
:10AB500001F0CAFEB8F1000F6BD103220023684652
:10AB600006F0FBFE354A8046D92101F0BDFEB8F162
:10AB7000000F5ED13A46FB17684606F0EEFE2F4AFC
:10AB80000746DB2101F0B0FE002F52D14FF0FF321B
:10AB90004FF0FF33684606F0E0FE284A0746E02102
:10ABA00001F0A2FE002F44D101220023684606F0E6
:10ABB000D4FE224A0746E22101F096FECFBB6FF099
:10ABC00001024FF0FF33684606F0C7FE1B4A0746F6
:10ABD000E82101F089FE67BB31462022684606F075
:10ABE000E3FE164A0646EA2101F07EFE0EBB6FF038
:10ABF00002024FF0FF33684606F0AFFE0F4A0646EA
:10AC0000EF2101F071FEA6B929462022684606F020
:10AC1000CBFE0A4A0546F12101F066FE4DB96946B0
:10AC2000204606F001FF054A0446F52101F05CFECE
:10AC300004B11024204604B0BDE8F081BA3E0108FA
:10AC4000F0B5ADF2244D044608A80D461646FBF7B4
:10AC500049FC03220023204606F07FFE444A0746B3
:10AC600040F2872101F040FE002F7BD1032269468C
:10AC7000204606F0C7FE3E4A074640F2892101F011
:10AC800033FE002F6ED13B496846FFF7E0FD384A9E
:10AC900007464FF4237101F027FE002F62D16FF0B9
:10ACA00006024FF0FF33684606F057FE304A07466B
:10ACB00040F28E2101F018FE002F53D12E49684634
:10ACC000FFF7C5FD2A4A074640F2922101F00CFE2B
:10ACD000002F47D129463246684606F065FE244AD1
:10ACE00005464FF4257101F0FFFD002D3AD12349AF
:10ACF0006846FFF7ACFD1E4A05464FF4267101F089
:10AD0000F3FD7DBB012204A9684606F077FE184AD0
:10AD1000054640F29A2101F0E7FD1DBBFBF7DCFB85
:10AD200008A9024604A806F03FFE114A054640F273
:10AD30009D2101F0D9FDADB904A9684606F074FE65
:10AD40000B4A054640F29F2101F0CEFD55B96946F8
:10AD5000204606F069FE064A04464FF4297101F0C8
:10AD6000C3FD1CB110200DF2244DF0BD2046FAE7C2
:10AD7000BA3E0108603E0108643E0108683E0108D1
:10AD800030B589B06A4604460D460C48102102F0E1
:10AD9000E9FC2846202102F0D7FC6A46102107482A
:10ADA00002F010FD10226946204607F099FA0028AB
:10ADB00014BF3320002009B030BD00BFE06E00207A
:10ADC00030B595B0044610A8FBF71AFB062204A97B
:10ADD000204606F017FEB84A05464C2101F084FDD6
:10ADE000002D40F063810122002304A806F0A7FD96
:10ADF000B14A0546502101F077FD002D40F0568103
:10AE00000222694604A806F0F9FDAB4A0546532123
:10AE100001F06AFD002D40F04981A8496846FFF71E
:10AE200016FDA54A0546562101F05EFD002D40F0B5
:10AE30003D81A3496846FFF70AFD9F4A0546582110
:10AE400001F052FD002D40F03181694604A806F062
:10AE5000EBFD994A05465B2101F046FD002D40F0CF
:10AE600025810222002304A806F069FD924A0546C6
:10AE70005F2101F039FD002D40F018810122694663
:10AE800004A806F0BBFD8C4A0546622101F02CFDAA
:10AE9000002D40F00B818B496846FFF7D8FC864AAD
:10AEA0000546652101F020FD002D40F0FF80694638
:10AEB00004A806F0B9FD804A0546682101F014FD9A
:10AEC000002D40F0F3800322002304A806F037FD94
:10AED000794A05466C2101F007FD002D40F0E6801F
:10AEE000102210A90DEB020006F05EFD724A054625
:10AEF0006F2101F0F9FC002D40F0D88004220023DE
:10AF000004A806F01CFD6C4A0546732101F0ECFC18
:10AF1000002D40F0CB80042208A904A806F072FDA1
:10AF2000654A0546762101F0DFFC002D40F0BE8029
:10AF30000222654908A806F04CFD5F4A05467921C2
:10AF400001F0D2FC002D40F0B180152108A806F0D8
:10AF500016FD594A05467C2101F0C6FC002D40F043
:10AF6000A5800222594908A806F033FD524A054639
:10AF7000802101F0B9FC002D40F09880152108A82F
:10AF800006F0FDFC4C4A0546832101F0ADFC002D86
:10AF900040F08C8004224E4908A806F01AFD464A6B
:10AFA0000546912101F0A0FC002D7FD1142108A8B5
:10AFB00006F0E5FC404A0546942101F095FC002D81
:10AFC00074D10922434908A806F003FD3A4A054610
:10AFD000992101F089FC002D68D13F4B59784B1E17
:10AFE00059425941143108A806F0C9FC324A0546B5
:10AFF0009C2101F079FC002D58D108A904A806F085
:10B0000013FD2D4A0546A22101F06EFC002D4DD105
:10B010000522002304A806F092FC274A0546A62133
:10B0200001F062FC002D41D14FF49662002304A888
:10B0300006F093FC204A0546A92101F055FC002D9D
:10B0400034D10622002304A806F079FC1A4A0546EA
:10B05000AD2101F049FC4DBB01220CA904A806F06A
:10B06000CDFC154A0546B02101F03EFCF5B90122A0
:10B0700000230CA806F071FC0F4A0546B32101F02D
:10B0800033FC9DB90CA904A806F0CEFC0A4A05467B
:10B09000B62101F029FC4DB904A9204606F0C4FCF4
:10B0A000054A0446C02101F01FFC14B1102015B060
:10B0B00030BD0020FBE700BFBA3E0108F33D0108A8
:10B0C000953E0108CD3E01089E3E0108A13E0108C3
:10B0D000A43E0108A93E0108306F002070B58AB077
:10B0E0000D46064601920021202202A81C4607F0C8
:10B0F0002DF902AA0021012002F034FB2021304664
:10B1000002F022FB2846122102F01EFB04210DEB67
:10B11000010002F019FB02AA0021012002F052FBFB
:10B1200006AD02AA2346144603CCAC42186059600F
:10B13000224603F10803F6D10AB070BD0148FAF7C0
:10B14000C5BF00BF306F00202DE9F04FADF5497D40
:10B15000164605464FF4B4720C4614A800211F464B
:10B1600007F0F4F84FF4B47200216EA807F0EEF87F
:10B170003368242B02D8012007F068F802F0C8FADF
:10B18000D5F80011284602F0DFFA204602F0E4FA72
:10B190002046FFF783FB814647F24810FFF764FB28
:10B1A0002128054619D100235D4D84F82030012067
:10B1B000FAF7B6FD6B78013B5A425A4194F82030B9
:10B1C00043EA820397B984F82030252131600025B5
:10B1D00028460DF5497DBDE8F08F524A40F2ED1149
:10B1E00001F082FB002DF3D10123DDE743F04003A2
:10B1F00084F82030326804F17D0800237D3A41460E
:10B20000684606F095FB04F12500FBF7F9F804F118
:10B21000370A4622002184F8362084F8351050463B
:10B2200004F1470B07F092F812215846FBF76CF82F
:10B23000C4F87990A44604F1590204F1200E634643
:10B2400003CB7345106051609C4602F10802F6D1B1
:10B2500053464A4659462046FFF740FF97F82831A3
:10B260006BB34622514614A807F048F84FF4917288
:10B2700039460DF1960007F041F8B5F84A900024E0
:10B28000A1450FD8FBF74FF8814546D2B5F84A30B3
:10B290000133A5F84A30FFF751FF14A94846FBF7E0
:10B2A00044F80CE06EA92046FBF74FF86EA914A8ED
:10B2B000FFF7B0FA78B314A92046FBF75DF897F8CA
:10B2C0002221D7F82431012A20D107331ED1FAF7E1
:10B2D000B1FD012801D1FAF795F90CAB04AA46217A
:10B2E000504602F065FBFAF7A5FD012802D10020C7
:10B2F000FAF788F90CAA04A96FF006036846FFF76D
:10B30000FFFB084A4FF4877101F0EEFA0099A1EBB8
:10B3100008017D315AE70134B2E7282558E700BF1C
:10B32000306F0020BA3E01082DE9F84F81460D46E6
:10B33000002319F80320DEB21AB90133202BF8D10B
:10B340001E4609F11F02002312F8011F5FFA83F85D
:10B3500019B90133202BF7D1984619F8060009EBEB
:10B360000803C70948220021284693F8204006F028
:10B37000EDFF30232B70C6F144033B44E409A3EBFB
:10B3800008032344EA196B704FF0000B0223AB70E3
:10B3900082F803B0C6F12002B91809EB060A381D7D
:10B3A000E9702844514606F0B7FF07F12402921BCA
:10B3B0000223AB5407F125031A19921B9B1B05F8B6
:10B3C00002B0C6F12600C8F12002A1183844E954A1
:10B3D000204408F120014944284406F09DFF04F16F
:10B3E00046003844801BA0EB0800BDE8F88F2DE92B
:10B3F000F843804689461D461746DDE9084602F0B7
:10B4000087F94946404602F09FF92021384602F06C
:10B410009BF9284602F0A0F928462246202102F096
:10B4200029FA31462046BDE8F843FFF77DBF70B5E5
:10B4300004460D461646FBF74FF8B0F5806F06D868
:10B44000324629462046BDE87040FFF7F9BB21206F
:10B4500070BD000030B50B78412B8DB005460C4611
:10B4600026D0422B34D0012B3AD102F051F9D5F835
:10B470000011284602F068F904A802F06DF92022B4
:10B4800004A904F1230006F02BFF48BB6B46D4F857
:10B49000432004F1110104A8FFF720FE10226946A1
:10B4A000601C06F01DFFB0FA80F040090DB030BD01
:10B4B00002F02EF9D5F80011284602F045F904A84B
:10B4C00002F04AF904AA3021601CFEF707FDEDE7FF
:10B4D000044A054841F68953D15C02F061FBE5E777
:10B4E0000020E3E754510020DD6D0020F0B5ADF2FF
:10B4F000B44D134605460A46014657A801F0DAFE48
:10B500000446A8B99DF8F733EBB147F24810FFF7AE
:10B51000ABF9824A40F2E32101F0E6F947F2481024
:10B52000FFF7A2F940B147F24810FFF79DF9C4B206
:10B5300020460DF2B44DF0BD794B5B78012B0CBF6A
:10B5400033243524F4E7579B03F00F030F2B40F00F
:10B55000DF80734A9DF8F6335278012A03D1002B1D
:10B5600046D13624E4E7002B42D19DF8E533012B88
:10B5700040F2D080694F0026F89BB34246D80322A0
:10B5800005A9284606F03EFA644A04464FF446717F
:10B5900001F0AAF9002C5AD10122002305A806F0D7
:10B5A000DCF95E4A04464FF4477101F09DF9002C26
:10B5B0004DD15C4905A8FFF74AF9584A044640F2C4
:10B5C0001E3101F091F9002C41D14FF49B7303938C
:10B5D00003AA09A9A9AB60A8FFF7B6FD4F4A044624
:10B5E00040F2253101F080F9002C32D0E4B29FE71F
:10B5F00058A90DF2E630FFF7C3FB484A044640F273
:10B60000F62101F071F9002CAFD091E709A9F4A857
:10B6100001F0D6FB1128044601D10136ACE73A46C9
:10B6200040F2073101F060F9002C81D109A960A82E
:10B63000FFF710FF00286FD1F4A806F069FD3A4625
:10B64000044640F2123101F04FF9002CE5D01024ED
:10B650006EE70399C1F59B73049309AB04AA1944DF
:10B66000FFA8FFF733F92D4A04464FF44B7101F060
:10B670003BF9002CBAD1049941B19DF84420039BB9
:10B6800062F07F020B448DF84420039302220023D2
:10B6900005A806F062F9214A044640F2363101F06D
:10B6A00023F9002CD3D1039A09A905A806F07CF947
:10B6B0001A4A04464FF44E7101F016F9002CC6D117
:10B6C00002F0CAF811AB21AC009309AB019458AA5F
:10B6D00003991846FFF78BFE2146024605A8FFF79F
:10B6E000A6FE0E4A04464FF4507101F0FDF8002CFE
:10B6F0007FF41EAF05A9284606F096F9074A0546CD
:10B7000040F2433101F0F0F8002D3FF411AF9EE715
:10B7100014240DE72C240BE7192409E7BA3E01088D
:10B72000306F0020B33E0108F0B5042285B000233D
:10B730000C46054606F011F94F4A064640F27931AB
:10B7400001F0D2F8002E40F0958094F84130002BA3
:10B750003FD04A4A41F68843D35C002B39D00422BB
:10B760006946284606F04EF901260746424A40F24D
:10B770008131384601F0B8F8002F7BD102224049D0
:10B78000684606F026F93C4A074640F2853101F04A
:10B79000ABF8002F6ED194F840202146684606F0A1
:10B7A00003F9354A07464FF4627101F09DF8002F06
:10B7B00060D1AEB96946284606F036F92E4A0446ED
:10B7C00040F2A33101F090F8002C53D1204605B08F
:10B7D000F0BD01226946284606F014F90746C5E780
:10B7E00004222849684606F0F4F8234A064640F247
:10B7F0008F3101F079F8002E3CD104F1A2016846A6
:10B80000FFF725F81C4A064640F2923101F06CF829
:10B8100086BB04221C49684606F0DBF8164A064639
:10B8200040F2953101F060F826BB04F14101684611
:10B83000FFF70DF8104A06464FF4667101F054F810
:10B84000C6B90B221149684606F0C3F80A4A0646F3
:10B8500040F29B3101F048F866B904F18201684674
:10B86000FEF7F5FF044A044640F29E3101F03CF831
:10B87000002C9FD01020AAE7BA3E010854510020A6
:10B880006C3E01086F3E0108743E0108793E0108D4
:10B890002DE9F04F0024DFF80C81E3B00546274680
:10B8A000D5F84C61BE421FDC8EB901F031FFD5F8EE
:10B8B00028113C4F05F1280001F046FF684601F0D1
:10B8C0004BFFB7F84A30B3424EDCC5F84C41D5F8CF
:10B8D0006C01354BD5F84C1140F2691207F053F862
:10B8E000204663B0BDE8F08F40F26916D5F86C11C0
:10B8F00006FB07F9494405F12800FFF7ABFDD5F831
:10B900006C614E4498B94621701C02F049F908B1A7
:10B9100001340AE0D5F86C614E4486F8430086F89D
:10B92000440086F8450086F846000137B8E7B8F8C5
:10B930004AA04FF0000906F1010BCA45E8DD08A94D
:10B940004846FAF702FD594608A8FEF763FF40B1E2
:10B950004FF491720DF1660106F1470006F0CEFC3E
:10B96000D6E709F10109E8E708A93046FAF7EDFC46
:10B97000202269460DF1420006F0B2FC80B9132C7A
:10B98000D5F86C21A1D040F269136343D01801218E
:10B99000D15401304FF4B47208A906F0BDFC013453
:10B9A00001368EE7306F002009A800082DE9F0432A
:10B9B0009046A5B001221F4600230E46054605F01D
:10B9C000CCFF6C4A04464FF4567100F08DFF002CFA
:10B9D00051D1022212A9284606F014F8654A0446FD
:10B9E00040F25B3100F080FF002C44D1022262491A
:10B9F00012A805F0EEFF5F4A044640F25F3100F006
:10BA000073FF002C37D1314611F8013B412B55D043
:10BA1000422B55D1594A41F68953D25C12A805F000
:10BA2000C3FF544A044640F2633100F05DFF14BB8B
:10BA30000422534912A805F0CCFF4E4A04464FF4A5
:10BA40005A7100F051FFB4B90A224E4912A805F00C
:10BA5000C0FF484A044640F26B3100F045FF54B93C
:10BA600012A9284605F0E0FF424A04464FF45C71F3
:10BA700000F03AFF04B110243E4A40F22F41204624
:10BA800000F032FF002C5CD102220023284605F092
:10BA900064FF384A044640F2334100F025FF5CB9A8
:10BAA0003A464146284605F07FFF324A044640F2B6
:10BAB000354100F019FF2CB1102442E03022ADE7EF
:10BAC0004622ABE73378412B3FD0422B3FD12B4A64
:10BAD00041F68953D15C741C002320461A460DF1AF
:10BAE000480901F053FF4946204602F0E3F880BBC5
:10BAF00002AB0093CDF8049043462C9A3946404659
:10BB0000FFF775FC044603220023284605F025FFB5
:10BB1000184A07464FF4896100F0E6FE002FCBD1AA
:10BB200022464946284605F03FFF124A044640F2A5
:10BB30004A4100F0D9FE002CBED196F8873053B9A7
:10BB40000024204625B0BDE8F0833021C3E746211C
:10BB5000C1E74824D7E706F147012846FFF7E4FD8F
:10BB6000044A044640F2514100F0BEFE002CE7D0EA
:10BB7000E7E700BFBA3E01086C3E010854510020BF
:10BB8000853E01088A3E01082DE9F0412F4F3D46D0
:10BB900006460FCD90B006AC0FC40FCD0FC495E88C
:10BBA000030041F67C4344F8040BF85821703C46EE
:10BBB000002849D0013840F26915F850454306A8DD
:10BBC000FEF76CFE7B1905F1450893F8CC30B844BC
:10BBD00083B1042202A9304605F014FF1C4A07462F
:10BBE00040F2734100F080FE37B11024204610B0BF
:10BBF000BDE8F0810322EDE741F68843E35C33B909
:10BC000005F1CD0041223946204406F09FFB114B3F
:10BC1000009306AA4146252302A8FFF7C7FE0C4A57
:10BC2000044640F27D4100F05FFE002CDED102A907
:10BC3000304605F0F9FE064A05464FF4906100F0E3
:10BC400053FE002DD2D0D0E73024CFE7545100204E
:10BC5000BA3E010879510020F0B5ADF50B7D0546DF
:10BC600027A801F07DF9044658B947F24810FEF7BD
:10BC7000FBFD2E4A064640F2934100F035FE26B108
:10BC8000F4B220460DF50B7DF0BD012201A9284636
:10BC900005F0B8FE254A064640F2954100F024FE24
:10BCA000002E3DD19DF8BC30412B3BD0422B3BD1E7
:10BCB0001F4A41F68953D15C00231A460DF1BD009D
:10BCC00001F064FE05AA202127A801F0D3FD15A9E3
:10BCD00005A8FFF729FB01220646002301A805F06D
:10BCE0003CFE124A074640F29E4100F0FDFDBFB9FE
:10BCF000324615A901A805F057FE0C4A06464FF436
:10BD0000946100F0F1FD5EB901A9284605F08CFEB2
:10BD1000064A054640F2A34100F0E6FD002DB0D0F2
:10BD20001024AEE73021C7E74621C5E7BA3E010837
:10BD3000545100202DE9F04FADF5317D804626A805
:10BD400001F082FB0446A8B99DF8FC31F3B147F23B
:10BD50004810FEF789FDA04A40F2B64100F0C4FD4C
:10BD600047F24810FEF780FD48B147F24810FEF751
:10BD70007BFDC4B220460DF5317DBDE8F08F974BB9
:10BD80005B78012B0CBF33243524F3E79DF8FB319E
:10BD9000002B71D027A90DF2EB10FEF7F1FF8E4AB0
:10BDA000044640F2BC4100F09FFD002CE2D18C4AD9
:10BDB00041F688430121D154709B002B00F007818C
:10BDC0009DF8BC30002B00F0028126A8FFF760FD33
:10BDD0000646002800F0FD8040F269176FF4B47346
:10BDE00047431F44819B3B44022893F88730B4BFEC
:10BDF0000322042203B1013204A9404605F002FEE9
:10BE0000754A044640F2E44100F06EFD002C40F01B
:10BE1000C180012E04DD724A41F68843D35C2BB900
:10BE2000819841220021883006F090FA819B03EB33
:10BE3000070909F1010075234621AF90029301F033
:10BE4000AFFE0546E8B12523029301F061FC70992D
:10BE500030A801F079FC08A801F07EFC05238DF8DC
:10BE60004030B6F1010B0DF19C0A6ED0BBF1130FFF
:10BE70004CD9012006F0EAF9594941F688428B5421
:10BE80009AE79DF8EA01B0FA80F04009F9F7B8FEA8
:10BE900002AA08A92B4630A8FFF756F904462846FF
:10BEA000F9F7AEFE4C4A40F20C51204600F01CFD62
:10BEB0000CB1E4B25EE74A499DF8403041F6884251
:10BEC00023F004038A5C029943EA82038DF8403030
:10BED000C1F17503039308AB03AA194483A8FEF7C5
:10BEE000F5FC3D4A044640F2165100F0FDFC002CE2
:10BEF000DFD103990029B4D09DF84020029B62F065
:10BF00007F020B448DF840200293AAE7DDF804C2BB
:10BF1000344A54462FAD234603CBAB4210605160E8
:10BF20001C4602F10802F6D108AD0FCD2C4C0FC40F
:10BF30000FCD0FC495E8030044F8040B20463A46A1
:10BF400000F8211B614606F0E7F9254A41F67C43DB
:10BF5000494642F803B004A808AACDF800A0029B05
:10BF6000FFF724FD1C4A044640F2235100F0BCFCBC
:10BF7000002C7FF4FFAE012E0EDC04A9404605F034
:10BF800053FD154A044640F22E5100F0ADFC002C42
:10BF90003FF4F0AE1024EDE60522002304A805F0DE
:10BFA000DCFC0D4A04464FF4A56100F09DFC002C1A
:10BFB000F0D13246F31704A805F0CFFC064A044638
:10BFC00040F22A5100F090FC002CD6D0E2E7142475
:10BFD000D0E62E24CEE600BFBA3E0108306F002026
:10BFE000545100207951002008B541F2040200218B
:10BFF00006F0ACF900F580534FF480521A8008BD6A
:10C0000010B501F01BFC1048FAF778F80446002040
:10C01000F9F786FE24B9FEF74DFD0B48FAF756F8FE
:10C02000094801F093FD094801F078FB1021084808
:10C03000FAF76AF9012802D0012006F007F9BDE8F5
:10C040001040FEF725BC00BF306F00207E6F00203F
:10C05000E06E002030B50B1F3B2B89B005460C4627
:10C0600002D9012006F0F2F801F052FB21462846E1
:10C0700001F06AFB684601F06FFB01F049FB68467E
:10C08000102101F061FB20220021684606F05EF9D4
:10C090002021064801F058FB054801F05DFB0548EA
:10C0A00001234370FAF712F809B030BD526F002037
:10C0B000326F0020306F0020044B082283F84820A4
:10C0C000034B03221A70FFF739B800BF306F00200E
:10C0D000E401002041F68C520021014806F036B9F7
:10C0E0005451002008B5FEF7E5FC0A48F9F7EEFFC9
:10C0F00010210948FAF708F9012802D0012006F0BA
:10C10000A5F8FFF7E7FFFEF7C3FB0448BDE80840CA
:10C1100001F004BB306F0020E06E00207E6F002035
:10C1200008B510220021074806F010F9064B20221E
:10C130001846002106F00AF9BDE808400238F9F770
:10C14000C5BF00BFE06E0020326F002010B50E4A60
:10C150000E4C92F90030002BC4BF03F1FF33137073
:10C1600094F94830002B0CDD013B84F84830FEF791
:10C17000E5FF94F94830002B01DCFFF7D1FF0020E8
:10C1800000E0FF2010BD00BFE4010020306F002060
:10C190002DE9F04198B03F2905460C4610469846D7
:10C1A0001E9E40F391804A4B5A78012A1F4609D1BE
:10C1B00093F94830002B40F38980464B93F90030C7
:10C1C000002B4FDD6A46444901F070FB01F0A0FAF4
:10C1D0002021684601F0B8FA684601F0BDFA202136
:10C1E000684608AA01F0BEFA2146284601F0ACFADA
:10C1F0001EB11021304601F0A7FA08AA2021684696
:10C2000001F0E0FA4146102208A806F069F801465C
:10C21000002857D1684601F057FB230711D121466A
:10C22000284601F077FB05F140031A46D41A13F8AB
:10C23000011D41B1C4F14004231F3B2B06D9372017
:10C2400035E00134E9E7AB42F0D1F3E77B78012B2D
:10C2500032D197F94830002B38DD1E4F97F9003066
:10C26000002B01DC342022E0002001F049FB1021EA
:10C27000304601F04FFB01F04BFA1021304601F03F
:10C2800063FA2021154801F05FFA10A801F064FA62
:10C290001022134910A806F023F858B1FEF7F8FA57
:10C2A000FFF754FF97F90030002BDBDD312018B089
:10C2B000BDE8F081FFF700FF28462146FFF7CAFEE0
:10C2C0000020F4E73320F2E77F20F0E73220EEE7AA
:10C2D000306F0020E401002060480020526F0020F1
:10C2E000326F002030B591B0144605466A460846C4
:10C2F000224901F0DBFA01F00BFA2021684601F037
:10C3000023FA684601F028FA0021684601F0DCFAB9
:10C310002046102101F0FEFA01F0FAF92046102122
:10C3200001F012FA2021164801F00EFA08A801F0D7
:10C3300013FA1022134908A805F0D2FF044660B191
:10C34000FEF7A6FAFFF702FF0F4B93F90030002B20
:10C35000D4BF3420312011B030BDFFF7ADFE2046F0
:10C3600001F0CEFA10220949284605F0D5FF2846EB
:10C37000102101F0D7FA2046EDE700BF6048002009
:10C38000526F0020326F0020E4010020E06E002098
:10C39000F0B5EBB006460BA801F004F90C9BDA1ED1
:10C3A000022A04460BD8A34A92F94820002A40F3F7
:10C3B0003281A14A92F90020002A40F32E81002CFC
:10C3C00040F096800B9A012A40F02981002B00F062
:10C3D0002681013B9DF8A651042B00F22081DFE865
:10C3E00013F0050049008A00AF00D000012203A924
:10C3F000304605F007FB914A074640F20B6100F01A
:10C4000073FA002F40F0CE8001238DF8A6319DF8FD
:10C41000A631002B00F009810322002303A805F0B8
:10C420009CFA864A074640F2656100F05DFA002FEB
:10C4300040F0B8807F4B93F9482003A8D31705F04C
:10C440008CFA7E4A074640F2676100F04DFA002FF1
:10C4500040F0A880002D00F0D88003A9304605F0F8
:10C46000E3FA764A054640F26D6100F03DFA002D90
:10C470003ED097E001352A4603A9304605F0C2FABE
:10C480006E4A074640F2146100F02EFA002F40F089
:10C4900089800122002303A805F05FFA674A074656
:10C4A00040F2176100F020FA002F7BD1F9F7C2FCAF
:10C4B000012801D1F9F7A6F86149624801F0F0F9C5
:10C4C000F9F7B8FC012802D10020F9F79BF85E4A81
:10C4D0006FF01803A2F1200103A8FEF711FB574AE1
:10C4E000074640F21E6100F0FFF9002F8FD0FCB22A
:10C4F00020466BB0F0BD4F4B5B78012B00F0918074
:10C50000649909B91424F3E79DF88D30002BF9D014
:10C510009DF87C30002BF5D0002300930DAA0DF17F
:10C520007D030DF18E00FFF733FE444A074640F2CB
:10C530002E6100F0D9F9002F3FF469AF3C46D7E7F0
:10C540003C4B5B78012B6ED164990029DAD09DF8C1
:10C550008D30002BD6D09DF87C30002BD2D09DF8AA
:10C56000A431002BCED065AB00930DAA0DF17D0355
:10C570000DF18E00FFF70CFE304A074640F23E6197
:10C58000D7E72C4B5B78012B4DD101352A4603A907
:10C59000304605F037FA294A074640F2476100F075
:10C5A000A3F90FB11024A3E79DF87C30002BA9D08C
:10C5B0009DF8A431002BA5D00222002303A805F08A
:10C5C000CCF91E4A07464FF4CA6100F08DF9002FDE
:10C5D000E8D165AA0DA907A8FFF784FE174A074608
:10C5E00040F2546100F080F9002FA7D1102207A972
:10C5F00003A805F0D9F9114A074640F2576100F047
:10C6000073F9002F3FF403AFCCE79DF8A631002B60
:10C610007FF423AF6CE732246AE7342468E77F2491
:10C6200066E7302464E7352462E7002D7FF415AF18
:10C630005EE700BF306F0020E4010020BA3E010831
:10C64000F06E002060480020106F00202DE9FF41AF
:10C65000154604460F4610220021684605F076FE76
:10C6600005F5805214F8016B1288DFF8048100236D
:10C6700029466846013F05F05BF96EB1022E01D9EB
:10C68000502E09D1384B93F94830002B64DD374BDD
:10C6900093F90030002B61DD042E3DD015D8022E19
:10C6A00034D05DD8012E25D001240020F9F738FBC5
:10C6B00041F6794308F803601CB141F202030022FD
:10C6C000EA52204604B0BDE8F081072E28D007D8F2
:10C6D000062EE9D13A4621466846FFF759FE0EE09C
:10C6E000082E27D0502EDFD13A4621466846FFF764
:10C6F000B3FA04E03A4621466846FEF7F7FE009B8F
:10C7000041F202025B1B0446AB52CEE73A46214699
:10C710006846FFF70FFBF2E76846FEF751FBEEE7CE
:10C7200047F24810FEF7A0F8C4B2002CBDD1FFF7C5
:10C73000D9FCBAE741F6794318F80330022B11D13E
:10C740006846FFF721FA009B41F202025B1B041EC0
:10C75000AB5208BF0226A8E73224A6E73424A4E798
:10C760000024A2E73024A0E7306F0020E40100207D
:10C770005451002008B5837BF52B06D0064B074AA1
:10C7800007484FF4A67105F043FD8389003318BFB5
:10C7900001230B70002008BDB73F0108D93E0108F6
:10C7A000D43F0108C27BD20701D505F039BB80898F
:10C7B0000021704738B5827BA02A0D4606D00C4B6D
:10C7C0000C4A0D484FF4F07105F022FDC37B13F0C5
:10C7D00004040AD1FFF7E6FF8C4208BF80422860BC
:10C7E0000CBF00204FF4806038BD0220FCE700BF82
:10C7F000EE3F0108613F0108D43F010838B5827B54
:10C80000802A0D4606D00C4B0C4A0D4840F2D3113D
:10C8100005F0FEFCC37B13F004040AD1FFF7C2FF4E
:10C820008C4208BF804228600CBF00204FF480601B
:10C8300038BD0220FCE700BF9C3F0108453F0108CE
:10C84000D43F010838B5837B03F0DF03402B0D464E
:10C8500006D00C4B0C4A0D4840F29D1105F0D8FC57
:10C86000C37B13F004040AD1FFF79CFFA14208BF69
:10C87000804228600CBF00204FF4806038BD022049
:10C88000FCE700BF07400108F03E0108D43F010863
:10C8900010B5837B402B06D0054B064A064840F274
:10C8A000B71105F0B5FC0023BDE8104005F0E0BB72
:10C8B0007B3F0108293F0108D43F010810B5837B65
:10C8C000602B06D0054B064A064840F2B11105F030
:10C8D0009FFC0023BDE8104005F0CABB2B400108B7
:10C8E0000D3F0108D43F0108704700002DE9F041D9
:10C8F0008B7BA02B8CB004460D4620D102A9284684
:10C9000005F010FB18B110200CB0BDE8F08101A9B2
:10C910002846FFF74FFF0028F5D1484E484FDFF873
:10C9200028810546019B9D4205D3236843F00403FB
:10C9300023600020E8E79DF81630602B01D013201B
:10C94000E2E718236A460DEB030102A80093FFF704
:10C95000B5FFB0F1004F01D11520D5E70028D2D1A5
:10C960008DF82F0002A805F0D3FB0028CBD131466B
:10C9700006A806F097F9C8B99DF81630402BDED10D
:10C980006A4604F5A47102A80093FFF781FFB0F195
:10C99000004FE1D0009B84F888310028B3D102A871
:10C9A00005F0B6FB0028AED10135BBE7394606A835
:10C9B00006F078F988B99DF81630602BBFD1412375
:10C9C0006A4604F2891102A80093FFF777FF30F05E
:10C9D000004098D184F8C901E1E7414606A806F075
:10C9E00061F990B99DF81630602BA8D120236A46D2
:10C9F00004F5E57102A80093FFF760FF30F00043F3
:10CA000081D1002384F8E931C9E70E4906A806F070
:10CA100049F90028C3D19DF81630602B8FD18023AF
:10CA20006A4604F5F57102A80093FFF747FF30F05E
:10CA300000407FF468AF84F86902B0E76C3E0108FB
:10CA4000743E01086F3E0108793E010870B58EB052
:10CA500010230193837BA02B04460E4615462BD151
:10CA600002AA174905F076FB10BB06AA1549204615
:10CA700005F070FBE0B99DF81630602B1ED19DF8D3
:10CA80002640DCB901AA0AA902A8FFF717FF78B966
:10CA90000D498DF837400AA806F004F900280CBFAC
:10CAA00001233F233370294606A805F0AFFA00B1F1
:10CAB000102420460EB070BD1324FAE71424F8E7C2
:10CAC000853E0108603E01088A3E010870B58B7BF7
:10CAD000802B88B005460E464AD104A9304605F0A1
:10CAE00021FA10B1102008B070BD02A93046FFF73E
:10CAF00085FE0028F6D10446029B9C420BD304A974
:10CB0000304605F00FFA0028ECD10446029B9C4207
:10CB100010D32620E7E703AA0DF1070104A8FFF7C9
:10CB200095FF0028DFD104A805F0F2FA0028D9D13A
:10CB30000134E1E703AA0DF1070104A8FFF786FF1E
:10CB400078B99DF80720012A0BD1039BD91D08D184
:10CB5000C5F86C322B6885F86A2243F008032B6015
:10CB6000C1E704A805F0D4FA0028BBD10134CDE711
:10CB70001320B8E713B5837B402B14460DD10192E7
:10CB800001AAFFF785FE30B90198844214BF032043
:10CB9000002002B010BD1020FBE71320F9E713B509
:10CBA000FD2301938B7B602B044608460ED101AA1E
:10CBB0002146FFF783FEB0F1004F09D050B9019B29
:10CBC00084F8FD00C4F8003102B010BD1320FBE76B
:10CBD0001520F9E71020F7E72DE9F0418B7BA02B1A
:10CBE00088B005460C4623D104A9204605F09AF9E1
:10CBF00018B1102008B0BDE8F08101A92046FFF768
:10CC0000D9FD0028F5D12A4FDFF8A880C5F800012A
:10CC100004460826019B9C4206D3D5F80031002B20
:10CC200014BF00201420E5E79DF81E30602B01D0D2
:10CC30001320DFE76A4602A904A80096FFF73EFE2C
:10CC4000B0F1004F32D00028D3D18DF80F0004A8E6
:10CC500005F05EFA0028CCD19DF81E30602BE7D19C
:10CC6000394602A806F01EF860B904A92846FFF765
:10CC700096FF0028BED104A805F04AFA0028B8D1D2
:10CC80000134C7E7414602A806F00CF80028F2D1AB
:10CC900020236A4605F5827104A80093FFF70EFE73
:10CCA00030F00040A5D185F82301E4E71520A1E785
:10CCB0006C3E0108743E01082DE9F0471F46837B56
:10CCC000A02B8AB004460D4616461DD106A905F0D4
:10CCD00029F918B110200AB0BDE8F08703A9204651
:10CCE000FFF768FD0028F5D1DFF8C880DFF8C890AD
:10CCF000DFF8C8A00446039B9C4201D30020EAE76A
:10CD00009DF82630602B01D01320E4E708230DEBBB
:10CD1000030204A906A80293FFF7D0FDB0F1004F6B
:10CD200046D00028D6D18DF8170006A805F0F0F9F6
:10CD30000028CFD19DF82630F52BE5D102224146BF
:10CD400004A805F0C1FF80B90DF1070106A8FFF79F
:10CD500011FD0028BED19DF807302B7006A805F004
:10CD6000D7F90028B6D10134C5E70222494604A804
:10CD700005F0AAFF50B90DF1070106A8FFF7FAFC6C
:10CD80000028A7D19DF807303370E7E7022251460B
:10CD900004A805F099FF0028E0D10DF1070106A8CD
:10CDA000FFF7E8FC002895D19DF807303B70D5E7E8
:10CDB000152090E79E3E01084C400108A13E010865
:10CDC00030B500230B70837BA02B89B005460C4641
:10CDD00056D104AA2B4905F0BDF918B11023184605
:10CDE00009B030BD9DF81E30402B01D01423F6E76A
:10CDF00046236A46611C04A80093FFF749FD009B87
:10CE0000302B24D1412323700028E7D104AA1E49E6
:10CE1000284605F09FF90028E0D19DF81E30602BD0
:10CE2000E4D10C236A4601A904A80093FFF746FD4C
:10CE3000B0F1004F1DD13F232370144901A805F024
:10CE400031FFC8B92378CBB901222270C7E7462B3E
:10CE5000DAD0422323706A464FF480730C49009362
:10CE600004A8FFF715FD0B4A009941F68953D154E8
:10CE7000CAE70028E1D0B1E73F2323700023AEE7E3
:10CE80001323ACE76C3E0108853E01088A3E010889
:10CE9000DD6D00205451002010B5E0B06946044615
:10CEA000FFF7ACFC10B1102060B010BD01A9204606
:10CEB00005F038F80028F6D10446009B9C4201D3C7
:10CEC0000020F1E705A901A8FFF77AFF0028EAD1C1
:10CED00001A805F01DF90028E5D10134EDE7837BB9
:10CEE000802B01D1FFF7D8BF1320704770B58B7B23
:10CEF000802B86B005460C4630D102A9204605F0AD
:10CF000011F810B1102006B070BD01A92046FFF73E
:10CF100075FC0028F6D1C5F84C01044640F26916AC
:10CF2000019B9C4201D30020EDE7142C14D0D5F8CE
:10CF30004C31D5F86C110133C5F84C3106FB0411A6
:10CF400002A8FFF73DFF0028DDD102A805F0E0F8B8
:10CF50000028D7D10134E3E71720D4E71320D2E724
:10CF6000F0B58FB00E461746002140F2891206AC8C
:10CF7000054605F0EBF9009404AB40F6FF72394624
:10CF8000304604F08DFF10B110200FB0F0BD9DF8B9
:10CF90002630A02B01D01320F7E70AA9204604F081
:10CFA000C1FF0028F0D103A92046FFF703FC0028A9
:10CFB000EAD1044605F12006039BA34201D80020D4
:10CFC000E3E79DF83630002BE5D102A90AA805F069
:10CFD0001DF80028D8D10AA805F09AF80028D3D166
:10CFE000029B012B08D0022B0ED00AA805F090F866
:10CFF0000028C9D10134DFE7202229460AA8FFF71B
:10D00000B9FD0028F1D0C0E731460AA8FFF7D8FEE5
:10D010000028EAD0B8E72DE9F0410023C1E9103338
:10D02000837BA02B86B005460C4625D102A904F0CF
:10D0300079FF18B1102006B0BDE8F0812846694696
:10D04000FFF7B8FB05460028F4D10746064604F171
:10D050002008009B9E420CD3002D4ED0002F4CD0B8
:10D06000236C002B49D0636C002B0CBF14200020D4
:10D07000E1E79DF816300BB11320DCE701A902A807
:10D0800004F0C4FF0028D5D102A805F041F800281B
:10D09000D0D1019B0333042B0FD8DFE803F0251C0C
:10D0A000150E03009DF81630002BE5D104F1400168
:10D0B00002A804F0ABFF0028BCD102A805F028F8B4
:10D0C0000028B7D10136C4E79DF81630002BD3D124
:10D0D00004F14401ECE72022214602A8FFF74AFDB3
:10D0E0000028A8D10125E8E72022414602A8FFF741
:10D0F00041FD00289FD10127DFE714209BE72DE9A0
:10D10000F043837BA02B87B004460F4663D102A96E
:10D1100004F008FF18B1102007B0BDE8F08369469D
:10D120002046FFF747FB0028F5D1054604464FF09F
:10D13000400807F10109009B9D4204D3032C0CBF5A
:10D1400000201420E8E79DF81630002B43D102A8F8
:10D15000FFF728FB9DF817309B07064648BFC643DC
:10D1600002A804F0D5FF0028D5D1022E13D0032E3B
:10D1700024D0012E08D107F1640102A8FFF74BFF6C
:10D180000028C9D10134E4B202A804F0C1FF00288C
:10D19000C1D10135CFE701AA494602A8CDF80480E4
:10D1A000FFF776FB019B202B01D0402B11D1B0F172
:10D1B000004F0ED00028AED13B70E3E7202301AA38
:10D1C00007F1410102A80193FFF762FB0028D9D0C3
:10D1D000A1E70320A0E713209EE70000F0B5837BC2
:10D1E000A02B8DB004460D465FD104A904F09AFE31
:10D1F00010B110200DB0F0BD03A92046FFF7DAFAF8
:10D200000028F6D12A4F04461026039B9C4201D3E6
:10D210000020EFE79DF81E30602B46D102AA08A936
:10D2200004A80296FFF74AFBB0F1004F11D104A801
:10D2300004F06EFF04A804F06BFF0028D9D104A805
:10D2400004F066FF04A804F063FF0028D1D1013484
:10D25000DBE70028CDD18DF82F0004A804F058FF9B
:10D260000028C6D10B22394608A805F02DFD00285C
:10D27000E8D19DF81E30F52B0DD10DF1070104A862
:10D28000FFF778FA0028B4D19DF80730002BD9D0E9
:10D2900001232B70D6E7A02BD4D1291D04A8FFF7BA
:10D2A0002EFF0028A6D10223F3E71320A2E700BF38
:10D2B000CD3E0108F0B5002191B0044616464FF46A
:10D2C00055721F4608AD05F041F8FF2384F88932F6
:10D2D000009506AB40F6FF723946304604F0E0FD9B
:10D2E00008B1C0B204E09DF82E30A02B02D011206E
:10D2F00011B0F0BD0CA9284604F014FE08B11020AE
:10D30000F6E704A92846FFF755FA0028F7D10546A5
:10D3100004F5277604F28A27049BAB4201D800204B
:10D32000E6E79DF83E30002BE1D103A90CA804F0FC
:10D330006DFE0028E3D10CA804F0EAFE0028DED13F
:10D34000039B013B082B11D8DFE803F005152027CC
:10D350002C404C5673002022211D0CA8FFF70AFC1C
:10D360000028BED1236843F0010323600CA804F019
:10D37000CFFE0135D0E70CA904F12400FFF72CFC07
:10D380000028AED1236843F00203EEE70CA9204643
:10D39000FFF7ACFA0028E9D0A3E70CA92046FFF775
:10D3A00095FBF7E70CA8FFF79AFD0028A7D104F535
:10D3B0001D710CA804F0B6FD0028A0D104F5217160
:10D3C0000CA8FFF71BFA0028D0D098E79DF83E3054
:10D3D000A02B36D104F528710CA8FFF7FFFE00281A
:10D3E000C4D085E704F2892304F5227204F51C7188
:10D3F0000CA8FFF761FCF2E79DF83E30402B0AD104
:10D4000005A90CA8FFF71EFA059B034303D10123CE
:10D4100084F89B32AAE7102239460CA8FFF7AAFB32
:10D42000032802D000287FF463AF012384F89A32E6
:10D430009CE79DF83E3023B931460CA804F0E6FD88
:10D44000C1E7132054E70000F0B5044691B00E4642
:10D45000174600214FF40A7204F078FF504BC4F8CD
:10D460006C3108ADFF2384F85231009506AB40F6CD
:10D47000FF723946304604F013FD10B1102011B090
:10D48000F0BD9DF82E30A02B01D01320F7E70CA99A
:10D49000284604F047FD0028F0D104A92846FFF7EC
:10D4A00089F90028EAD1054604F5B47604F2531749
:10D4B000049BAB4201D80020E1E79DF83E30002BF1
:10D4C000E3D103A90CA804F0A1FD0028D6D10CA833
:10D4D00004F01EFE0028D1D1039B013B062B0FD880
:10D4E000DFE803F013041B252B3552002022211DF9
:10D4F0000CA8FFF73FFB0028C1D1012384F824309A
:10D500000CA804F005FE0135D2E70CA904F12800AF
:10D51000FFF745FB0028F3D0B1E70CA92046FFF741
:10D52000E5FC0028AAD1012384F87031E8E704F56E
:10D53000BA710CA8FFF752FEECE704F5A97304F2E8
:10D54000511204F5A8710CA8FFF7B6FBE2E79DF8AD
:10D550003E30402B0AD105A90CA8FFF773F9059BB3
:10D56000034303D1012384F86431C9E7102239460B
:10D570000CA8FFF7FFFA032802D000287FF47FAF42
:10D58000012384F86331BBE79DF83E30002B7FF424
:10D590007CAF31460CA804F039FD0028B0D06DE70F
:10D5A00099510020F0B591B00E46174600214FF476
:10D5B000BE7208AD044604F0C9FE009506AB40F605
:10D5C000FF723946304604F06BFC10B1102011B0E8
:10D5D000F0BD9DF82E30A02B01D01320F7E70CA949
:10D5E000284604F09FFC0028F0D104A92846FFF744
:10D5F000E1F80028EAD1054604F5BD7604F2791772
:10D60000049BAB4201D80020E1E79DF83E30002B9F
:10D61000E3D103A90CA804F0F9FC0028D6D10CA88A
:10D6200004F076FD0028D1D1039B013B072B0DD8D8
:10D63000DFE803F004131924304D5A649DF83E309E
:10D64000002BCAD121460CA804F0E0FC0CA804F081
:10D650005FFD0028BAD10135D2E79DF83E30002B9E
:10D66000BBD1211DEFE704F108010CA8FFF7D3FCA3
:10D670000028ACD1012384F85030E7E7102204F1F0
:10D6800051010CA8FFF776FA0028A0D1012384F8F5
:10D690006130DBE79DF83E30402B9ED105A90CA8F8
:10D6A00004F050FD002891D1059BA3F14002C02A4F
:10D6B0002BD8C4F8643105AA4FF4807304F16201D9
:10D6C0000CA80593FFF7E4F80028BFD07EE71022EE
:10D6D00004F5B4710CA8FFF74DFA00287FF477AF7A
:10D6E000012384F87831B1E79DF83E30F52B7FF4C3
:10D6F00074AF39460CA8FFF73DF8E5E79DF83E30DA
:10D70000F52B7FF46AAF3146F4E737205FE700007E
:10D71000014800F0D5BB00BFF048002010B5402202
:10D7200004460146064804F0F7FD064A04F14003AA
:10D73000603453F8041B42F8041BA342F9D110BD16
:10D740008C480020604900200A460146014800F04C
:10D75000E3BB00BFF04800200146014800F0FABBDF
:10D76000F048002030B591B004460D46402200211B
:10D77000684604F0EBFD34B1012C1CD0402D04D9D7
:10D78000012004F063FD0D4C20252A462146684601
:10D7900004F0B4FD6A4640231178013B81F0360164
:10D7A00002F8011BF8D1FFF7B3FF40216846FFF7ED
:10D7B000CBFF11B030BD2025014CE6E78C4800209E
:10D7C0006049002070B5044690B010460D461646DC
:10D7D000FFF7C2FF40220021684604F0B7FD34B1D4
:10D7E000022C23D0402D04D9012004F02FFD114C30
:10D7F00020252A462146684604F080FD6A464023DB
:10D800001178013B81F05C0102F8011BF8D1FFF7B0
:10D810007FFF68464021FFF797FF20213046FFF742
:10D8200093FF3046FFF798FF10B070BD2025024CE3
:10D83000DFE700BF8C4800206049002008B504489D
:10D8400003F098FA03F09CFA024B186008BD00BF81
:10D85000096300088048002008B5F8F739FE034B3B
:10D860001860034B20221A6008BD00BF88480020C2
:10D870008448002007B5084B1B68009313460A46EE
:10D8800001460648006803F031FD10B9012004F09C
:10D89000DDFC03B05DF804FB8048002088480020D0
:10D8A000014B1A6803F092BB8048002008B5054B75
:10D8B0001B6803F069FA012802D0012004F0C6FCBD
:10D8C00008BD00BF80480020012810B50C4614BFD9
:10D8D00001460849084803F045FF10222146074841
:10D8E0001CB9BDE8104004F031BDBDE8104004F0A3
:10D8F00013BD00BF6049002000700020F0700020C0
:10D9000001461022024809B904F020BD04F004BD0C
:10D91000F07000200A460146014803F04FBF00BFE7
:10D92000007000200A460146014803F01DBF00BFF9
:10D93000007000202DE9F041069C88460021074632
:10D940001546084622461E46FFF70CFF414638465C
:10D95000FFF7FAFE28460C4D3146FFF7F5FE284644
:10D960002021FFF7F1FE002122460846FFF72AFF9B
:10D9700005F120000021FFF7A7FF20462021BDE888
:10D98000F041FFF7CFBF00BF8C48002013B5054C16
:10D990000094FFF7CFFF044B1C60044B20221A6059
:10D9A00002B010BDCC4800208848002084480020E8
:10D9B00070B59AB002AE1C460023154600961A4672
:10D9C000FFF7B8FF402200210AA804F0BFFC0F4B6C
:10D9D0000AA91A68304603F0F9FA0AAB12AA1E46E1
:10D9E00003CE964228606960334605F10805F6D1FA
:10D9F00023461AAD144603CCAC4218605960224647
:10DA000003F10803F6D11AB070BD00BF80480020B2
:10DA100070B591F8CE30FF2B88B005460C466FD11B
:10DA200001F1220630462021F8F76EFC012867D16B
:10DA30006B78D3B1FFF76CFE696CA81CFFF784FE0E
:10DA40006846FFF789FEFFF763FE10216846FFF77F
:10DA50007BFE20220021684604F078FC304620211D
:10DA6000FFF772FEA01CFFF777FE626C6B6C9A42A8
:10DA700005D0264B264A2A21264804F0C9FBFF235D
:10DA80000126636484F8CE602A7823789A4203D012
:10DA9000214B1F4A2E21EFE76A7863789A4203D020
:10DAA0001E4B1B4A2F21E7E795F9482094F948308F
:10DAB0009A4203D01A4B164A3021DDE7B5F84A20C6
:10DAC000B4F84A309A4203D0164B114A3121D3E7B9
:10DAD000022204F14C0105F14C0004F001FC18B1E4
:10DAE000114B0B4A3221C7E7802204F14E0105F1A8
:10DAF0004E0004F0F5FB30B10C4B054A3321BBE777
:10DB0000002008B070BD3046FBE700BFAB40010805
:10DB10004F400108E840010805410108464101085D
:10DB20007F410108C2410108F94101085A42010838
:10DB300010B501460446D022034804F0EDFB204610
:10DB4000BDE81040F8F7C2BA306F002010B5037876
:10DB5000E8B00446DBB134A8F8F7D0FA6846F8F725
:10DB6000CDFA94F8CE30FF2B07D1694634A8FFF7E1
:10DB70004FFF60B16846FFF7DBFF94F8CE30012B12
:10DB800005D0044B044A0548552104F041FB68B018
:10DB900010BD00BF7E40010865400108E840010853
:10DBA000172908B508DD04220449104404F098FB45
:10DBB000B0FA80F0400908BD0020FCE7BE42010831
:10DBC000034B1860034B00221A70034B1970704707
:10DBD0008049002000710020017100202DE9F043F0
:10DBE0001D4695B001238DF803302B78103B4FF084
:10DBF0000008012B16468DF8028054D84046F8F7ED
:10DC0000A1FA81464046F8F79DFA07464046F8F7E4
:10DC100099FA04464046F8F795FA3F02000E40EAAA
:10DC2000096007F47F07240A384304F47F44204343
:10DC3000019001210DF10300FCF7A4F804210DEB84
:10DC40000100FCF79FF801210DF10200FCF79AF8A2
:10DC50003246294602A800F077F848218DF80200E4
:10DC600002A8FCF78FF89DF90230C3B1FCF7A6F8C3
:10DC700001210DF10300FCF785F804210DEB0100F3
:10DC8000FCF780F80021482202A804F05FFB9DF811
:10DC900002308DF80830482102A8FCF773F80448D8
:10DCA00015B0BDE8F0834FF020630193C1E700BFDA
:10DCB0000090FFFF042238B505460C461044074982
:10DCC00004F00EFB38B946222946601C00F03CF8EF
:10DCD0002070012038BD0020FCE700BFBE420108D3
:10DCE0002DE9F0414378022B07460C461CD191F8F0
:10DCF000405001F1410630462946FFF751FFBB78FD
:10DD0000072B07D1002846F6851008BF4FF4D540F1
:10DD1000BDE8F08178B133462A4604F1200120465F
:10DD2000BDE8F041FFF75ABF032B07D14AB9BDE860
:10DD3000F041FCF7FBB84FF4D540E9E74FF4DA4087
:10DD4000E6E74FF4CE40E3E738B50D4647210446F9
:10DD5000FFF736FF2B78142B03D0152B08D00120AA
:10DD600038BD0323012223706270A3700020F7E7FF
:10DD700047212046F8F7C8FA40B201280CBF00201E
:10DD80002120EDE72DE9F04FC9B008AA01F14005C7
:10DD900014464B780E781B0443EA0663CE7833436F
:10DDA0008E78043143EA06238D4244F8043BF0D1D7
:10DDB0001024916B16464FEAF14383EA714383EADC
:10DDC0009123716A366852F8045F31440B444FEA7C
:10DDD000B54181EAF51181EAD50101340B44402CAB
:10DDE000D363E6D1D0E914E30093836D0193C36D4F
:10DDF0000293036E0393436E0493836E0593C36E85
:10DE00000693DDE9057BDDE9031CDDE901592B4BB8
:10DE1000009E079374464FF00008079B53F8042BAD
:10DE200007934FEAF12383EAB11383EA716A08ABDF
:10DE300053F828301A440AEB020327EA010A01EAE0
:10DE40000C028AEA02021A444FEA743A86EA05038F
:10DE50005A448AEAB40A06EA050B234083EA0B0314
:10DE60008AEAB45A08F101089A44B8F1400F02EB6B
:10DE70000903BB465244A94619D172440265009A6F
:10DE800022444265019A32448265029A2A44C2655C
:10DE9000039A1A44049B02660B444366059B634441
:10DEA0008366069B3B44C36649B0BDE8F08F674676
:10DEB00035468C46264619461446AEE7C44201084C
:10DEC0000023002203640023C0E912230B4B0C4AF9
:10DED0000C49DFF840C0C0E914230B4BC0E916130E
:10DEE0000A4BC0E918C30A4B836603F17453A3F5C8
:10DEF0002303A3F69243C366704700BF85AE67BB9A
:10DF000067E6096A72F36E3C3AF54FA58C68059B8B
:10DF1000ABD9831F7F520E51F8B504460D468E18BB
:10DF20000027B54200D1F8BD236C15F8012BE2544F
:10DF30000133402B2364F4D121462046FFF722FF12
:10DF4000D4E9123113F5007341F10001C4E9123133
:10DF50002764E6E7026C2DE93048372A0D464FF07A
:10DF6000800102F10103815404464FF0000246D8BB
:10DF7000382B3FD1236CD900D4E9122312EB010BCB
:10DF800043F1000C9BFA8BF2E2634FEA1C224FEA4A
:10DF90001C6384F83A204FEA1C4284F8383021464A
:10DFA000C4E912BC84F83BC084F839202046FFF74E
:10DFB000E9FE691E1823226DDA4001F8012F626D17
:10DFC000DA400A71A26DDA400A72E26DDA400A7331
:10DFD000226EDA400A74626EDA400A75A26EDA4086
:10DFE0000A76E26EDA40083B13F1080F0A77E2D1B5
:10DFF000BDE83088E2540133BAE7E25401333F2BE5
:10E00000FBD921462046FFF7BDFE3822002104F04F
:10E010009DF9AFE7000000000000000000000000D4
:10E02000C3F10803DB0070B40133002403A500BF73
:10E030005B1920C940CAAD1920C0184720C940CA81
:10E04000754120C020C940CA754120C020C940CABE
:10E05000754120C020C940CA754120C020C940CAAE
:10E06000754120C020C940CA754120C020C940CA9E
:10E07000754120C06441204670BC7047000000001C
:10E08000C3F10803DB0070B40133002403A500BF13
:10E090005B1920C940CAAD1B20C0184720C940CA1F
:10E0A000B54120C020C940CAB54120C020C940CADE
:10E0B000B54120C020C940CAB54120C020C940CACE
:10E0C000B54120C020C940CAB54120C020C940CABE
:10E0D000B54120C06441B4FA84F0400970BC704777
:10E0E000052B2DE9F04F09D0062B00F04381072BBB
:10E0F0006AD0082B00F0EA81BDE8F08F08B4F8CAB6
:10E1000004B451F8042BA3FB028940F8048B4FF0B0
:10E11000000AE4FB629A4FF0000BE5FB62AB4FF0A4
:10E12000000CE6FB62BC4FF0000EE7FB62CE51F83C
:10E13000042B4FF00008E3FB628940F8048BE4FBFA
:10E14000629AE5FB62ABE6FB62BCE7FB62CE51F88C
:10E15000042B4FF00008E3FB628940F8048BE4FBDA
:10E16000629AE5FB62ABE6FB62BCE7FB62CE51F86C
:10E17000042B4FF00008E3FB628940F8048BE4FBBA
:10E18000629AE5FB62ABE6FB62BCE7FB62CE51F84C
:10E19000042B4FF00008E3FB628940F8048BE4FB9A
:10E1A000629AE5FB62ABE6FB62BCE7FB62CE40F83D
:10E1B000049B40F804AB40F804BB40F804CB40F8A3
:10E1C00004EB0CBCBDE8F08FF0CA51F804EBA4FBE3
:10E1D0000E8940F8048B4FF0000AE5FB6E9A4FF071
:10E1E000000BE6FB6EAB4FF0000CE7FB6EBC51F88A
:10E1F00004EB4FF00008E4FB6E8940F8048BE5FB6C
:10E200006E9AE6FB6EABE7FB6EBC51F804EB4FF089
:10E210000008E4FB6E8940F8048BE5FB6E9AE6FB90
:10E220006EABE7FB6EBC51F804EB4FF00008E4FB6B
:10E230006E8940F8048BE5FB6E9AE6FB6EABE7FB5C
:10E240006EBC51F804EB4FF00008E4FB6E8940F817
:10E25000048BE5FB6E9AE6FB6EABE7FB6EBC51F8F8
:10E2600004EB4FF00008E4FB6E8940F8048BE5FBFB
:10E270006E9AE6FB6EABE7FB6EBC51F804EB4FF019
:10E280000008E4FB6E8940F8048BE5FB6E9AE6FB20
:10E290006EABE7FB6EBC40F8049B40F804AB40F863
:10E2A00004BB40F804CBA0F11C00A1F11C0170CA12
:10E2B00051F804EBD0F800804FF00009E4FB6E89C0
:10E2C00040F8048B4FF0000AE5FB6E9A4FF0000B0C
:10E2D000E6FB6EAB51F804EBD0F80080E4FB6E89EE
:10E2E00040F8048BE5FB6E9AE6FB6EAB51F804EB4D
:10E2F000D0F80080E4FB6E8940F8048BE5FB6E9A51
:10E30000E6FB6EAB51F804EBD0F80080E4FB6E89BD
:10E3100040F8048BE5FB6E9AE6FB6EAB51F804EB1C
:10E32000D0F80080E4FB6E8940F8048BE5FB6E9A20
:10E33000E6FB6EAB51F804EBD0F80080E4FB6E898D
:10E3400040F8048BE5FB6E9AE6FB6EAB51F804EBEC
:10E35000D0F80080E4FB6E8940F8048BE5FB6E9AF0
:10E36000E6FB6EAB40F8049B40F804AB40F804BBFE
:10E37000BDE8F08F70CA51F804EBA4FB0E8940F899
:10E38000048B4FF0000AE5FB6E9A4FF0000BE6FBA2
:10E390006EAB51F804EB4FF00008E4FB6E8940F8D7
:10E3A000048BE5FB6E9AE6FB6EAB51F804EB4FF085
:10E3B0000008E4FB6E8940F8048BE5FB6E9AE6FBEF
:10E3C0006EAB51F804EB4FF00008E4FB6E8940F8A7
:10E3D000048BE5FB6E9AE6FB6EAB51F804EB4FF055
:10E3E0000008E4FB6E8940F8048BE5FB6E9AE6FBBF
:10E3F0006EAB51F804EB4FF00008E4FB6E8940F877
:10E40000048BE5FB6E9AE6FB6EAB40F8049B40F88C
:10E4100004AB40F804BBA0F11800A1F1180170CAC8
:10E4200051F804EBD0F800804FF00009E4FB6E894E
:10E4300040F8048B4FF0000AE5FB6E9A4FF0000B9A
:10E44000E6FB6EAB51F804EBD0F80080E4FB6E897C
:10E4500040F8048BE5FB6E9AE6FB6EAB51F804EBDB
:10E46000D0F80080E4FB6E8940F8048BE5FB6E9ADF
:10E47000E6FB6EAB51F804EBD0F80080E4FB6E894C
:10E4800040F8048BE5FB6E9AE6FB6EAB51F804EBAB
:10E49000D0F80080E4FB6E8940F8048BE5FB6E9AAF
:10E4A000E6FB6EAB51F804EBD0F80080E4FB6E891C
:10E4B00040F8048BE5FB6E9AE6FB6EAB40F8049BDC
:10E4C00040F804AB40F804BBBDE8F08FF0CA51F847
:10E4D00004EBA4FB0E8940F8048B4FF0000AE5FB27
:10E4E0006E9A4FF0000BE6FB6EAB4FF0000CE7FBB3
:10E4F0006EBC51F804EB4FF00008E4FB6E8940F865
:10E50000048BE5FB6E9AE6FB6EABE7FB6EBC51F845
:10E5100004EB4FF00008E4FB6E8940F8048BE5FB48
:10E520006E9AE6FB6EABE7FB6EBC51F804EB4FF066
:10E530000008E4FB6E8940F8048BE5FB6E9AE6FB6D
:10E540006EABE7FB6EBC51F804EB4FF00008E4FB48
:10E550006E8940F8048BE5FB6E9AE6FB6EABE7FB39
:10E560006EBC51F804EB4FF00008E4FB6E8940F8F4
:10E57000048BE5FB6E9AE6FB6EABE7FB6EBC51F8D5
:10E5800004EB4FF00008E4FB6E8940F8048BE5FBD8
:10E590006E9AE6FB6EABE7FB6EBC51F804EB4FF0F6
:10E5A0000008E4FB6E8940F8048BE5FB6E9AE6FBFD
:10E5B0006EABE7FB6EBC40F8049B40F804AB40F840
:10E5C00004BB40F804CBA0F12000A1F12001F0CA67
:10E5D00051F804EBD0F800804FF00009E4FB6E899D
:10E5E00040F8048B4FF0000AE5FB6E9A4FF0000BE9
:10E5F000E6FB6EAB4FF0000CE7FB6EBC51F804EB92
:10E60000D0F80080E4FB6E8940F8048BE5FB6E9A3D
:10E61000E6FB6EABE7FB6EBC51F804EBD0F8008074
:10E62000E4FB6E8940F8048BE5FB6E9AE6FB6EAB6B
:10E63000E7FB6EBC51F804EBD0F80080E4FB6E8978
:10E6400040F8048BE5FB6E9AE6FB6EABE7FB6EBC15
:10E6500051F804EBD0F80080E4FB6E8940F8048B9D
:10E66000E5FB6E9AE6FB6EABE7FB6EBC51F804EB84
:10E67000D0F80080E4FB6E8940F8048BE5FB6E9ACD
:10E68000E6FB6EABE7FB6EBC51F804EBD0F8008004
:10E69000E4FB6E8940F8048BE5FB6E9AE6FB6EABFB
:10E6A000E7FB6EBC51F804EBD0F80080E4FB6E8908
:10E6B00040F8048BE5FB6E9AE6FB6EABE7FB6EBCA5
:10E6C00040F8049B40F804AB40F804BB40F804CB8E
:10E6D000BDE8F08F052A2DE9F04F09D0062A00F099
:10E6E000FD80072A5FD0082A00F06B81BDE8F08F1B
:10E6F000B1E8005E06B4AAFB09124FF00003EBFB81
:10E7000069234FF00004ECFB69344FF00005EEFB89
:10E7100069454FF00006EBFB6A63ECFB6A3449186D
:10E72000524176415B41A9FB09784FF0000949F15C
:10E73000000918EB0108A0E88001AAFB0A785741FC
:10E7400058EB0608A0E88001EEFB6A454FF0000A8E
:10E750004AF1000A4FF00001ECFB6B14EEFB6B4535
:10E760004FF00002EEFB6C255FEA59094941644114
:10E7700052416D4149F10009EBFB6B3A1AEB010A7A
:10E78000A0E80804ACFB0C6A66415AEB020AA0E858
:10E790004004AEFB0E6A6E415AEB090AA0E8400441
:10E7A00006BCBDE8F08FB1E8001E04B4AAFB09E284
:10E7B0004FF00003EBFB69234FF00004ECFB6934DE
:10E7C0004FF00005EBFB6A531EEB0E0E52416D41FC
:10E7D0004FF0000747F10007A9FB096818EB0E0886
:10E7E000A0E84001AAFB0A68564158EB0508A0E8DA
:10E7F00040014FF0000848F10008B1E8444002B47D
:10E80000E2FB69344FF00005E6FB69454FF000017B
:10E81000EEFB69514FF00009ECFB6A39E2FB6A94A8
:10E82000E6FB6A45EEFB6A514FF0000AECFB6BA970
:10E83000E2FB6B94E6FB6B45EEFB6B517F085B41A3
:10E840005AEB0A0A59EB090947F10007EBFB6B3851
:10E8500018EB0A08A0E808014FF0000848F100088A
:10E860004FF00003E2FB6C34E6FB6C45EEFB6C51B1
:10E870004FF0000AE6FB62A5EEFB62514FF0000B81
:10E88000EEFB66B17F085B4164415AEB0A0A6D41B9
:10E890005BEB0B0B494147F10007ECFB6C8919EB73
:10E8A0000309A0E80003A2FB028958EB040859EB16
:10E8B0000A09A0E80003A6FB068958EB050859EBF6
:10E8C0000B09A0E80003AEFB0E8958EB010859EBD9
:10E8D0000709A0E8000306BCBDE8F08FB1E8005FBF
:10E8E00006B4A9FB08124FF00003EAFB68234FF0BF
:10E8F0000004EBFB68344FF00005ECFB68454FF07B
:10E900000006EEFB68564FF00007EAFB6973EBFB6D
:10E910006934ECFB694530B4491852417F415B4191
:10E92000A8FB08454FF0000848F100086D1830C0FA
:10E93000A9FB094554417D4130C030BCEEFB69560E
:10E940004FF0000949F100094FF00001EBFB6A1498
:10E95000ECFB6A45EEFB6A564FF00002ECFB6B25C0
:10E96000EEFB6B564FF00007EEFB6C765FEA580843
:10E970004941644152416D417F41764148F100086F
:10E98000EAFB6A3919EB0109A0E80802ABFB0B9A14
:10E9900059EB04095AEB020AA0E80006ACFB0C9AFA
:10E9A00059EB05095AEB070AA0E80006AEFB0E9AE0
:10E9B00059EB06095AEB080AA0E8000606BCBDE8B8
:10E9C000F08FB1E8005C04B4ABFB0A234FF0000405
:10E9D000ECFB6A344FF00005EEFB6A454FF0000691
:10E9E000ECFB6B6492185B4176414FF0000747F1F6
:10E9F0000007AAFB0A8919EB0209A0E80003ABFB98
:10EA00000B8958EB030859EB0609A0E800034FF007
:10EA1000000848F100080CC902B4E2FB6A454FF057
:10EA20000006E3FB6A564FF00009EEFB6B94E2FB35
:10EA30006B454FF00001EEFB6C147F0859EB0909A0
:10EA4000494147F10007ECFB6C8919EB0109A0E88B
:10EA500000034FF0000848F1000802BC51F8049B85
:10EA6000096880B4E9FB6A564FF00007E1FB6A676A
:10EA70005DF804ABE3FB6B45E9FB6B56E1FB6B67B1
:10EA80004FF0000BE2FB6CB4E3FB6C45E9FB6C560A
:10EA9000E1FB6C674FF0000CE2FB6EC4E3FB6E45DC
:10EAA000E9FB6E56E1FB6E675FEA5A0A5BEB0B0B04
:10EAB0005CEB0C0C4AF1000AEEFB6E8B1BEB0C0BB3
:10EAC000A0E800094FF0000848F100084FF0000BE3
:10EAD000E3FB62B5E9FB6256E1FB62674FF0000CB5
:10EAE000E9FB63C6E1FB63674FF0000EE1FB69E7FA
:10EAF0005FEA5A0A64415BEB0B0B6D415CEB0C0C5B
:10EB000076415EEB0E0E7F414AF1000AE2FB62485D
:10EB100018EB0B08A0E81001A3FB03486C4158EB6D
:10EB20000C08A0E81001A9FB0948744158EB0E0835
:10EB3000A0E81001A1FB01487C4158EB0A08A0E8BD
:10EB4000100104BCBDE8F08FF0B51C4699B0164624
:10EB500007460D4693F90020314608A8FFF7BAFD95
:10EB6000D4F8AC3008A9684698476A4694F9003052
:10EB7000394608A8FFF7B4FA3846D4F8AC3008A9EB
:10EB80009847324694F90030694608A8FFF7A8FA7A
:10EB9000D4F8AC3008A9684698476A4694F9003022
:10EBA000294608A8FFF79CFAD4F8AC3008A92846F3
:10EBB000984719B0F0BD00BF000000000000000041
:10EBC00070B40123002405A5AFF30080AFF30080EB
:10EBD0005B1920C940CAAD1B20C0184720C940CAD4
:10EBE000B54120C020C940CAB54120C020C940CA93
:10EBF000B54120C020C940CAB54120C020C940CA83
:10EC0000B54120C020C940CAB54120C020C940CA72
:10EC1000B54120C06441B4FA84F0400970BC70472B
:10EC200070B40123002405A5AFF30080AFF300808A
:10EC30005B1920C940CAAD1920C0184720C940CA75
:10EC4000754120C020C940CA754120C020C940CAB2
:10EC5000754120C020C940CA754120C020C940CAA2
:10EC6000754120C020C940CA754120C020C940CA92
:10EC7000754120C06441204670BC70472DE9F04FBB
:10EC8000D4B204F1FF3A5FFA8AFA93B04FFA8AF3EA
:10EC9000002B16460694C0F2218151F82320002A49
:10ECA00040F02181A21E52B2013201EB820205E046
:10ECB00052F8047D002F40F0018123465D1E6CB2A6
:10ECC000671CF5D1002B40F0F880884AD2F800E0AC
:10ECD000BEF1000F00F08B8008910699C0F3800B05
:10ECE000A1EB0B010546CCB2C3EB461304F0FE00CA
:10ECF0004FF0FF3705EB8B021BB227FA03F30292AA
:10ED00000390069A01935844042143B24FEA5209F2
:10ED100002F0FE0C0593029A049416FB01F3009393
:10ED200064080AABCDF81CC001FB065802EBC40412
:10ED300003EBC90972469DF91C30009909932846D6
:10ED4000A8F1040840279047002850D0D8F8003098
:10ED5000019A002E03EA0203C8F800303EDDBAF142
:10ED6000030F40F2A780BBF1000F00F09080D5F8B0
:10ED700000C0029B00221146A646D3E9004008339A
:10ED8000734542EA040241EA0001F6D10A43DDE993
:10ED900003318B42744642EA0C022CD0059955F897
:10EDA0002100CBB2591C49B28E4242EA000213DD67
:10EDB00055F82100991C49B28E4242EA00020BDD4F
:10EDC00003335BB29E4255F82110C8BF55F823307B
:10EDD00042EA0102C8BF1A43002A5AD1013F06D0B5
:10EDE000424B00991A68284690470028AED100206F
:10EDF00013B0BDE8F08F002AF0D033462A460899B8
:10EE00000AA8FFF73DF910F1000C18BF4FF0010CF4
:10EE1000002211460AABA646D3E9004008339945C3
:10EE200042EA040241EA0001F6D10A43DDE9063173
:10EE30008B4274461CD0099B12A901EB8301DBB203
:10EE400051F8200C591C49B28E4242EA00020FDDF3
:10EE500012A800EB8101023351F8201C5BB29E42E4
:10EE600042EA010204DD00EB830353F8203C1A431D
:10EE70004FEA4C0C002A0CBFCCF10002CCF101028D
:10EE8000D2B2012AAAD1104613B0BDE8F08FDC46F9
:10EE90006FE733462A4608990AA8FFF7F1F810F100
:10EEA000000C18BF4FF0010CBAF1020FB0D80022CD
:10EEB0001346C1E70022114671E75D1E03F180434E
:10EEC000013B51F823302BB100225B0802F1010213
:10EED000FBD193B203EB45139BB2F6E61346002B2E
:10EEE0003FF4F3AEE9E73346751EE7E784490020B7
:10EEF0002DE9F04FB5B0B3F1000811900D9240F339
:10EF0000EC8108F1FF35EDB20135AD000DF150098E
:10EF1000164648462A460DF1700A03F0EFF924AC74
:10EF200031462A46504603F0E9F92CAE2A46002124
:10EF3000204603F00BFA01232A4630460021249391
:10EF400003F004FA5FFA88F2531EDBB24FFA83FC37
:10EF500010934FEA88034FEA8C0109EB03000690F7
:10EF600009EB010004900AEB01000AEB030705908E
:10EF7000701861181D1F0E9709913946043F0F97AD
:10EF8000771965191295069D13972F1F0A97BCF1E3
:10EF9000000F06EB0307234408900797019339DB22
:10EFA000023A53B21846069A00936FEA09050346DF
:10EFB0001544049801339B006FEA0A0725F0030506
:10EFC000551B0F4409EB0302D0F800C005980392CB
:10EFD00027F003070AEB0302CF1B0292D0F800E0F0
:10EFE000F218E3180C920B93083F083DF4451FD824
:10EFF000C0F08280DDE90212009BAB4608E052F8C7
:10F00000045D51F8040D854211D803F1FF3372D32A
:10F010001806F4D5B8F1000F06DD109A11980132E8
:10F020009200214603F06AF935B0BDE8F08F5D46E5
:10F03000149B13F0010B4FF0010263D01C9B13F0E3
:10F04000010B00F0DC80012A434640F08F805246DD
:10F0500049464846FFF714F8069B4B450AD90A9AD9
:10F060000023116843EA510342F80439AA424FEAE7
:10F07000C173F6D1099B1A68089B1B689A4213D882
:10F08000C0F0F780DDE90B21009BA44609E052F8AF
:10F09000044D51F8040D844205D803F1FF33C0F04C
:10F0A000E7801806F3D5644643463246214620469B
:10F0B000FEF7E6FF249810F0010040F0CE80019B9F
:10F0C000A3424CD9019A002352F8041D43EA51038C
:10F0D000A24213604FEAC173F6D800283FD0129ABB
:10F0E00004991368D1F800C0059943F00043D1F8A2
:10F0F00000E013607AE75D46149B13F0010B4FF0BC
:10F10000FF329BD1069B4B450AD90A9B5A46196888
:10F1100042EA510243F804299D424FEAC172F6D1F6
:10F12000249810F0010040F0AB80019BA34240F214
:10F130009080019B53F8041D4BEA5102A3421A60D0
:10F140004FEAC17BF6D8002800F08380129A049918
:10F150001368D1F800C043F00043136046E7049BF6
:10F16000D3F800C0059BD3F800E03FE74A4651467C
:10F170005046FEF785FF0E9B53450AD90F9A002390
:10F18000116843EA510342F80439BA424FEAC173A5
:10F19000F6D1089B1A68099B1B689A4213D8C0F0E5
:10F1A0009580DDE90B12009BA44609E052F8044D5E
:10F1B00051F8040D844205D803F1FF33C0F0858077
:10F1C0001C06F3D564464346224631463046FEF7D8
:10F1D00057FF2C9810F0010060D1079BB342BED9B5
:10F1E000079A002352F8041D43EA5103B242136008
:10F1F0004FEAC173F6D80028B1D0139A70E70E9B7E
:10F2000053450AD90F9B5A46196842EA510243F8FE
:10F2100004299F424FEAC172F6D12C9810F00100E8
:10F2200046D1079BB3429DD9079B53F8041D4BEA77
:10F230005102B3421A604FEAC17BF6D8002891D040
:10F24000139A05991368D1F800E043F00043136066
:10F25000CCE6049BD3F800C0C8E643460D9A21468D
:10F260002046FEF7DDFE019BA3423FF62BAF34E7BD
:10F27000644643460D9A21462046FEF7D1FE13E729
:10F2800043460D9A21462046FEF7CAFE019BA34243
:10F29000059BD3F800E03FF64CAF54E743460D9A88
:10F2A00031463046FEF7BCFE079BB34298D8A2E732
:10F2B00043460D9A31463046FEF7B2FE079BB342F5
:10F2C000049BD3F800C0AFD8B8E7644643460D9A14
:10F2D00031463046FEF7A4FE75E7012324930DF175
:10F2E00050090DF1700A24AC2CAE2BE62DE9F04F3D
:10F2F000ABB0DFB21C4604937B1EDBB2A6B20C4659
:10F3000059B206934FEA86181AAB00290797099459
:10F31000059015461FFA88F80893C0F2268252F825
:10F320002130002B40F01F82BA1E52B2013205EB91
:10F33000820205E052F8040D002840F0D4811946FD
:10F340004B1E5BB2581CF5D1002940F0CC810FFA5E
:10F3500088F8B8F1000F4346B8BF08F11F035B11EE
:10F36000D8F1000202F01F025FB208F01F0658BF7A
:10F370005642002F07DD5A1ED2B201329200002100
:10F380000AA802F0E3FF002E40F3CB81049B002B80
:10F3900000F0E4812A682AA800EB870102FA06F04F
:10F3A00041F8800C0499C6F12003012922FA03F2E6
:10F3B00040F2DC8069682AA801FA06FC00EB8700AD
:10F3C0004CEA020240F87C2C049A022A21FA03F14A
:10F3D00000F0CC80AA682AA802FA06FC00EB87009D
:10F3E0004CEA010140F8781C0499032922FA03F23F
:10F3F00000F0BC80E9682AA801FA06FC00EB87004F
:10F400004CEA020240F8742C049A042A21FA03F10F
:10F4100000F0AC802A692AA802FA06FC00EB8700FB
:10F420004CEA010140F8701C0499052922FA03F204
:10F4300000F09C8069692AA801FA06FC00EB8700AD
:10F440004CEA020240F86C2C049A062A21FA03F1D5
:10F4500000F08C80AA692AA802FA06FC00EB87005B
:10F460004CEA010140F8681C0499072922FA03F2CA
:10F470007CD0E9692AA801FA06FC00EB87004CEA77
:10F48000020240F8642C049A082A21FA03F16DD094
:10F490002A6A2AA802FA06FC00EB87004CEA01015E
:10F4A00040F8601C0499092922FA03F25ED0696AC7
:10F4B0002AA801FA06FC00EB87004CEA020240F899
:10F4C0005C2C049A0A2A21FA03F14FD0AA6A2AA8CE
:10F4D00002FA06FC00EB87004CEA010140F8581CD8
:10F4E00004990B2922FA03F240D0E96A2AA801FA0A
:10F4F00006FC00EB87004CEA020240F8542C049A08
:10F500000C2A21FA03F131D02A6B2AA802FA06FC50
:10F5100000EB87004CEA010140F8501C04990D29CA
:10F5200022FA03F222D0696B2AA801FA06FC00EB4A
:10F5300087004CEA020240F84C2C049A0E2A21FA69
:10F5400003F113D0AA6B2AA802FA06FC00EB87008D
:10F550004CEA010140F8481C04990F2922FA03F2F1
:10F5600004D0EB6BB340134340F8443CB8F1000FB8
:10F57000C0F2848004990FFA81FC4FEA8C020AAB36
:10F580009F18BA186FEA030E00923A1FBE444B1E32
:10F5900003922AAA02EB83032EF0030EA7EB0E0EB2
:10F5A000019302EB81034FEA4C0CAEF1080E4FF0D1
:10F5B000010B0293BCF1000FD8BF002426DD2AAA5C
:10F5C000CBF1010302EB830353F888AC02EB8B030E
:10F5D000002253F8889C144613462AA901EB8303A2
:10F5E00010B253F8803C59F820102344CB1A34BF92
:10F5F000012600268B4202F1010500F089806AB2E3
:10F6000094454AF8203034461346E6DCABEB040B55
:10F610000AABBBFA8BFB9F424FEA5B1B0AD9039AEA
:10F620000023116843EA510342F8043972454FEA56
:10F63000C173F6D1029B019953F8802C51F8803C9C
:10F6400043EAC27341F8803C009BBB420AD91A4688
:10F65000002352F8041D43EA5103974213604FEA16
:10F66000C173F6D308F1FF380FFA88F8B8F1FF3FFD
:10F67000A0D12AAB03EB8B0B5BF8884C049B002BCF
:10F680002EDD05990A4604F108030832944238BF7A
:10F690009942069A2CBF01230023052A94BF002318
:10F6A00003F00103002B4AD00B4623435B0746D1EE
:10F6B000079B5D0801EBC505A4F108020B46F2E9C2
:10F6C0000201E3E80201AB42F9D1079A02F0FE031E
:10F6D0009A4205D01BB2059954F8232041F8232003
:10F6E0002BB0BDE8F08F8EB201F18041013955F8A1
:10F6F00021302BB100225B0802F10102FBD193B251
:10F70000013EA8EB4618A8EB03031FFA83F81EE698
:10F71000013252B262454AF820301346FFF65DAF1F
:10F7200074E7049B002B4FEA870017DD069B5A1CE9
:10F730000AAB29461844920002F0E0FD16E7059B4B
:10F74000069A043B04EB8201043C54F8042F43F86E
:10F75000042FA142F9D12BB0BDE8F08FB8F1000F12
:10F76000BFF608AFBCE70499BEE7049900293FF44F
:10F77000EEADB8E72DE9F04192F9006098B015467A
:10F7800000230446324608A80327CDE90133CDE91A
:10F790000333CDE90533079300978846FEF79AFFB8
:10F7A000D5F8AC3008A92046984733462146204674
:10F7B0006A462F1DFEF764FC00283BD1424695F9AE
:10F7C0000030214608A8FEF78BFC08A9D5F8AC301C
:10F7D00020469847334605F1840221462046FEF72D
:10F7E0001FFCF0B9F3B25A1E52B2002A19DB12B252
:10F7F00057F8221054F822208A4218D311D8023B1D
:10F800005BB25A1C92001544224408E055F80409E2
:10F8100052F8041D88420AD803F1FF3301D31906B8
:10F82000F4D533463A4621462046FEF729FC18B067
:10F83000BDE8F08133463A4621462046FEF7F0FB0C
:10F84000BCE700BF2DE9F04798B01646209DA946B9
:10F85000804619F9044B8A461F4602462346314624
:10F860006846FEF70DFC002840F0818095F90020E5
:10F8700008A86946FEF72EFF08A9D5F8AC306846FF
:10F8800098476A4608A895F900304146FEF728FCDB
:10F8900008A9D5F8AC30404698476A4608A895F9BB
:10F8A00000303146FEF71CFC08A9D5F8AC303046D4
:10F8B00098472346524639463846FEF7E1FB002872
:10F8C0007FD195F90020394608A8FEF703FFD5F847
:10F8D000AC3008A9684698472346424669466846C0
:10F8E000FEF7CEFB002865D12346324669466846BE
:10F8F000FEF7C6FB002856D1234642463146304625
:10F90000FEF7BEFB002847D1324695F9003051463C
:10F9100008A8FEF7E5FBD5F8AC3008A95046984793
:10F9200023466A4641463046FEF7AAFB68BB32468C
:10F9300095F90030394608A8FEF7D2FBD5F8AC306F
:10F9400008A9384698472346524639463846FEF7B6
:10F9500097FB98B9002C07DD621ED2B201329200EB
:10F960006946304602F0CAFC18B0BDE8F08723466D
:10F970004A4669466846FEF753FB77E74A46234600
:10F9800039463846FEF74CFBE4E723464A46314603
:10F990003046FEF745FBCAE723464A463146304625
:10F9A000FEF73EFBB0E723464A4669466846FEF747
:10F9B00037FBA1E723464A4669466846FEF730FB17
:10F9C00092E723464A4639463846FEF729FB78E750
:10F9D0002DE9F047B3F902A01AF11F0448BF0AF15C
:10F9E0003E041F461AF1070348BF0AF10E03DE105A
:10F9F000641196424FFA84F928BF1646B9F1000FF8
:10FA00000546884606DD621ED2B201329200002110
:10FA100002F09CFCF31C48BFB31D9B105AB2002A95
:10FA200007DD5A1ED2B2013292000021284602F0B0
:10FA30008DFC002E16DD00221146701E411A21F0A9
:10FA4000030C18F802E055F80C3001F00301C9006E
:10FA500001320EFA01F152B20B43964245F80C30D6
:10FA60001146EBDCF600564539D905EB84039D427F
:10FA7000A6EB0A0A0CD2CAF12006002053F8041D96
:10FA800021FA0AF202439D421A6001FA06F0F5D308
:10FA9000E4B2631E5BB2002B07F1240218DB1BB239
:10FAA00052F8231055F823308B4218D310D8023C5B
:10FAB00064B207EB8407243708E057F8041955F8B7
:10FAC000243099420BD804F1FF3401D32306F4D536
:10FAD0004B4629462846BDE8F047FEF7D1BABDE8B7
:10FAE000F08700BF000000000000000000000000E0
:10FAF0002DE9F04500F1080201F10803984238BFF2
:10FB000091428BB080468A46C0F03C8140EA0103B6
:10FB10005B0740F03781D1E90023C0E90023D1E938
:10FB20000223C0E90223D1E90423C0E90423D1E977
:10FB30000623C0E90623DAE90B370593DAF83830F3
:10FB40000193DAF83430069702AADAF83C7007938A
:10FB5000019B00260024002511461046CDE90837F8
:10FB6000CDE902450496FFF75BF802AA0746414635
:10FB70004046FFF755F8DAF830300593DAF83830B8
:10FB80000193DAF83430069302AA019B07931146D9
:10FB9000DAF83C300893074410460996FFF740F81E
:10FBA00002AA074441464046FFF73AF8DAE908134B
:10FBB0000744CDE90213DAF82800DAF83830049067
:10FBC00002AA414608934046DAF83C300993CDE951
:10FBD00006450596FFF724F8DAF83430DAF82010F5
:10FBE00009910744DAF82810DAF82C0005930893F5
:10FBF000DAF838300693DAF83C300793CDE9031091
:10FC0000DAF82430029302AA41464046FFF708F88A
:10FC1000DAE90B130744CDE90213DAF83400DAF815
:10FC20002030049002AA414608934046DAF8283072
:10FC30000993CDE906450596FEF7C2FFDAE90C13F4
:10FC4000CDE90645DAF83C400594CDE90213DAF82F
:10FC50002440DAF82C303F1ADAF83800049002AA6F
:10FC600041464046CDE90843FEF7AAFFDAE90D41D7
:10FC7000DAE908353F1ADAF83C000294CDE9053597
:10FC8000DAF83040DAF82830039102AA41460490AD
:10FC90004046079309940896FEF792FFDAE9095166
:10FCA000DAE90E430691DAF82C100791DAF83410ED
:10FCB00009913F1A02AA4146404604960896CDE9AA
:10FCC00002430595FEF77CFF3F1A50D4DFF8F8C0D9
:10FCD0004FF0010EF7B9D8F81C3001334FD1D8F8E6
:10FCE0001830002B4BD0012B14D8D8F814308BB916
:10FCF000D8F8103073B9D8F80C305BB9D8F80830A0
:10FD000001333CD1D8F80430013338D1D8F8003071
:10FD1000013334D14346624671464646002003A46F
:10FD2000091910CE20CA641B10C3084710CE20CA80
:10FD3000AC4110C310CE20CAAC4110C310CE20CAB3
:10FD4000AC4110C310CE20CAAC4110C310CE20CAA3
:10FD5000AC4110C310CE20CAAC4110C310CE20CA93
:10FD6000AC4110C34041002808BF013FB2E7164C28
:10FD7000224641464046FEF753FF3F18F8D40BB0E9
:10FD8000BDE8F085DAF80030C8F80030DAF8043061
:10FD9000C8F80430DAF80830C8F80830DAF80C305F
:10FDA000C8F80C30DAF81030C8F81030DAF814302F
:10FDB000C8F81430DAF81830C8F81830DAF81C30FF
:10FDC000C8F81C30B7E600BFC84301082DE9F0476A
:10FDD000A8B01646309DA946074619F9044B8A4635
:10FDE00098460246234631466846FEF749F9002800
:10FDF00040F0098195F9002018A86946FEF76AFCD1
:10FE000018A9D5F8AC30684698476A4618A895F9FD
:10FE100000303946FEF764F918A9D5F8AC303846F9
:10FE200098476A4618A895F900303146FEF758F908
:10FE300018A9D5F8AC30304698472346524641467B
:10FE40006846FEF7EDF808BBE3B25A1E52B2002A2C
:10FE50001CDB12B228A901EB820059F8221050F8DD
:10FE6000A02C914218D811D3023B5BB25A1C9200CD
:10FE7000A9186A4408E051F804C952F8040D8445F1
:10FE80000AD803F1FF3301D31806F4D523464A46B6
:10FE900069466846FEF7F4F8234652464146404616
:10FEA000FEF7EEF8002840F0E68008A823463A4620
:10FEB0003146FEF7E5F8002840F0D68008AA95F90B
:10FEC0000030514618A8FEF70BF9D5F8AC3018A948
:10FED0005046984723463246394608A8FEF7A0F810
:10FEE00010BBE3B25A1E52B2002A1DDB12B228A97F
:10FEF00001EB820159F8222051F8801C914219D35C
:10FF000012D8023B5BB25A1C920008A8A9180244FE
:10FF100008E051F804C952F8040D84450AD803F1E9
:10FF2000FF3301D31806F4D508A923464A460846EC
:10FF3000FEF7A6F895F90020414618A8FEF7CAFB7F
:10FF4000D5F8AC3018A930469847234608AA314660
:10FF50003046FEF795F800287FD1324610A8234698
:10FF60003946FEF78DF8002870D110AA95F90030B7
:10FF7000414618A8FEF7B4F8D5F8AC3018A94046A9
:10FF800098472346524641464046FEF779F80028F6
:10FF900055D195F90020694618A8FEF79BFBD5F8C6
:10FFA000AC3018A910A8984710A9234608AA0846FB
:10FFB000FEF766F800283BD123463A4610A908A868
:10FFC000FEF75EF868BB6A4695F9003008A918A8E4
:10FFD000FEF786F8D5F8AC3018A908A8984723464C
:10FFE000524608A95046FEF74BF898B9002C07DD99
:10FFF000621ED2B20132920010A9384602F07EF998
:020000040801F1
:1000000028B0BDE8F08723464A4669466846FEF7B1
:1000100007F8EFE64A46234651465046FEF700F8F9
:10002000E4E708A923464A460846FDF7F9FFCAE770
:1000300010A923464A460846FDF7F2FFBCE72346CF
:100040004A4641464046FDF7EBFFA2E710A923468A
:100050004A460846FDF7E4FF87E723464A4631460D
:100060003046FDF7DDFF78E708A923464A460846F3
:10007000FDF7D6FF22E723464A4641464046FDF7B4
:10008000CFFF12E72DE9F04FC3B098464D9FBDF961
:10009000309197F900400394A5000B462B44002CA7
:1000A0000791CDE908500292069340F33281651E14
:1000B000EEB201361AABB600184632462AAC0593AA
:1000C00002F01CF932460699204602F017F932ABCD
:1000D0000493324641461846B8F1000F00F02D81D6
:1000E00002F00CF9039B0599EDB2002B05F1010517
:1000F0004FEA85050DF1480BD8BF04252A4658461E
:100100000DF1880A02F008F92A465046214602F00D
:1001100003F9049D059E21463B462A463046FEF7DC
:1001200013FD21463B46D7F8A4402A463046A04757
:10013000A9F102043B462A465146584624B2FEF72E
:1001400003FD002C28DD6311029AA4B252F823208B
:10015000009704F01F03012101FA03F3134213BFB8
:1001600020260026202500250BEB06090BEB0508B1
:1001700056445544314648462B464246FFF726FE34
:10018000013C33464A46294640460097FFF75AFB52
:10019000A3B21CB2002BD6D1029B1B6800976FEA5A
:1001A000030903F0010809F001094FEA49194FEA70
:1001B00048180BEB09020BEB0804D144D0444B4622
:1001C0004146204602923D1DFFF700FE0599039B24
:1001D00005950AA85A46FDF753FF002840F0A6806F
:1001E000049D97F9003042460AA92846FDF778FF9A
:1001F000D7F8AC3029460AA89847079A97F90030F3
:100200000AA92846FDF76CFFD7F8AC3029460AA8A2
:100210009847039B002B40F39B805FFA83FE0EF10F
:10022000FF35EDB2022D40F2BC804FEA5E0C002299
:100230000AAB03EBCC0C1146D3E9006008336345ED
:1002400042EA060241EA0001F6D10EF0FE007045D6
:1002500041EA020143B21BD042AA02EB8302DBB2A5
:1002600052F8E00C5A1C0143039852B290420FDD41
:1002700042AE06EB8202023352F8E02C5BB29842A7
:1002800041EA020104DD06EB830353F8E03C194325
:10029000002957D00AA9039B059A0846FEF728FEB5
:1002A0000135049E069A97F900300AA93046FDF7F9
:1002B00017FFD7F8AC3031460AA89847224697F97D
:1002C00000300AA93046FDF70BFF3146D7F8AC30B5
:1002D0000AA8984743462246494602980097FFF7E6
:1002E000B1FA3B460AAA51465846FEF72DFC099C36
:1002F000AD0059462A46204602F000F82346089CE5
:1003000023442A465146184601F0F8FF43B0BDE8A1
:10031000F08FB8F1000F47D01AAB059332AB2AAC7F
:1003200004930DF1480B0DF1880AF2E60AA9039B2C
:100330003A1D0846FDF774FE52E702F007F8012364
:100340003293CFE60135AA000AA801F0FFFFA8E723
:10035000049D069A97F900300AA92846FDF7C0FEC9
:10036000D7F8AC3029460AA89847224697F90030BA
:100370000AA92846FDF7B4FE2946D7F8AC300AA8EA
:10038000984743462246494602980097FFF75AFA93
:100390003B460AAA51465846FEF7D6FB43B0BDE895
:1003A000F08F00210B4657E701233293B4E700BFDB
:1003B000F0B59DF914E0CEF10804E40001349C4648
:1003C00023460446002705A5AFF30080AFF3008065
:1003D0005B1920C940CAAD1920C4184720C940CABA
:1003E000754120C420C940CA754120C420C940CAF3
:1003F000754120C420C940CA754120C420C940CAE3
:10040000754120C420C940CA754120C420C940CAD2
:10041000754120C47F41DFB95FFA8EF35A1E52B294
:10042000002A15DB12B25CF8221050F8222091420B
:1004300015D80DD3023B5BB208E05CF8231050F8EE
:10044000232091420BD803F1FF3301D31A06F4D5D0
:10045000734662460146BDE8F040FDF711BEF0BDAF
:100460002DE9F04F93F90070002FA5B040F36F8194
:100470005FFA87FA0AF1FF34E4B2032C0294C2F364
:10048000800640F2B281002E00F06481146803946B
:100490004FF0010BAAEB06095FFA89F902EB860619
:1004A0004FEA59084FF0000E06EBC808F446D6E9AB
:1004B00000540836464545EA0E0E44EA0C0CF6D1C7
:1004C00009F0FE05039C4CEA0E0CAB44A9454CEA2E
:1004D00004044FFA8BFB1DD05FFA8BF56E1C52F8AB
:1004E0002BC076B2B74244EA0C0413DD52F826C0A2
:1004F000AE1C76B2B74244EA0C040BDD03356DB294
:10050000AF4252F82660C8BF52F8255044EA0604AC
:10051000C8BF2C43002C00F01A81984614460546AB
:100520003A4614A88946FEF7D5F814A904A8D8F8C5
:10053000AC30984704AA14A898F900302946FDF772
:10054000CFFDD8F8AC3014A90CA8984798F9002032
:1005500004A914A8FEF7BEF814A904A8D8F8AC3072
:100560009847224614A898F900304946FDF7B8FD8F
:10057000D8F8AC3014A94846984798F9002014A838
:100580002146FEF7A7F808F1040B14A9D8F8AC30FF
:10059000204698475B462246294628460097FFF7A3
:1005A00007FF5B462246214620460097FFF700FFE3
:1005B0003B46224629462046FDF762FD002840F0D2
:1005C000CC80224698F90030294614A8FDF788FD12
:1005D000D8F8AC3014A9284698475B462A462946E5
:1005E00020460097FFF7E4FE5B4622460097294627
:1005F0002846FFF7DDFE2B68BA00AE1813F00103A2
:10060000A2F10402039206D0CAE056F8042D43EA90
:1006100052033360D307B542F7D398F90020294637
:1006200014A8FEF757F8D8F8AC3014A9204698471C
:100630003B460CAA21462046FDF722FD002840F04B
:10064000A8803B460CAA21462046FDF719FD00284C
:1006500040F098800CA93B4622460846FDF710FD65
:10066000002840F088800CAA98F90030294614A888
:10067000FDF736FDD8F8AC3014A92846984704AAEF
:100680003B4629461046FDF7FBFC00286CD105F1DE
:10069000080304F108060299B54238BF9C422CBFFA
:1006A0000123002345EA0402052994BF00270127FE
:1006B00012F0070F18BF0023002B00F08A80002FD4
:1006C00000F087804FEA5A0C05EBCC0CA4F108022D
:1006D0002B46F2E90201E3E802016345F9D10AF091
:1006E000FE03534504D01BB254F8232045F82320C1
:1006F00009F10803B14538BF9C4249EA04022CBF06
:100700000126002612F0070F18BF0026002E6FD01A
:10071000002F6DD04FEA5A0504EBC505A9F1080278
:100720002346F2E90201E3E80201AB42F9D10AF003
:10073000FE03534504D01BB259F8232044F823206C
:10074000029A0132920004A9484601F0D7FD25B073
:10075000BDE8F08F0396B3469CE63B465A462146D9
:100760002046FDF75DFC2CE704A93B465A460846A7
:10077000FDF756FC8BE70CA93B465A460846FDF7A9
:100780004FFC70E73B465A4621462046FDF748FCA1
:1007900060E73B465A4621462046FDF741FC50E7BC
:1007A0003B465A4629462846FDF73AFCB54238BF33
:1007B000002308D256F8042D43EA5203B5423360B1
:1007C0004FEAC273F6D3039AAB5843EAC073AB50F7
:1007D00023E7029A043D231F04EB820153F8042F00
:1007E00045F8042F8B42F9D182E70024A34673E633
:1007F000029A043CA9F1040309EB820153F8042F87
:1008000044F8042F8B42F9D19AE700BF2DE9F04F4D
:10081000BDB00DF1300B479CCDF828B094F90040E5
:1008200002949E46002C14AB0B9340F3B7809DF8C6
:1008300008300393013BDBB2032B0593CEF3800812
:1008400040F2DD80B8F1000F00F0AC80DEF800303F
:1008500004934FF00109039BA3EB080A5FFA8AFA9D
:100860004FEA5A0C0EEB8804002604EBCC0C3546FC
:10087000D4E900730834A44546EA070645EA0305AF
:10088000F6D10AF0FE03049C35439944534545EAEA
:1008900004054FFA89F91ED05FFA89F35C1C029FA8
:1008A0005EF8296064B2A74245EA060513DD5EF8EA
:1008B00024609C1C64B2A74245EA06050BDD0333A5
:1008C0005BB29F425EF82440C8BF5EF8233045EA21
:1008D0000405C8BF1D43002D60D0479B0990B3F9A4
:1008E0000240479B14F11F0648BF04F13E067611F3
:1008F000243375B2CDE90712049319462CA82B4670
:100900007246F246FDF7BCFB003018BF0120002DF7
:1009100044DD5FFA86F909F1FF33DBB2022B06935F
:1009200040F20F824FEA590C00222CAB03EBCC0CA7
:100930001146D3E9007608339C4542EA070241EAB2
:100940000601F6D109F0FE034B4542EA01025EB210
:100950001BD03CAB03EB8603F6B253F8401C731C70
:100960005BB29D4242EA01020FDD3CA901EB830329
:10097000023653F8403C76B2B54242EA030204DD47
:1009800001EB860656F8403C1A434300002A0CBF90
:100990005B42C3F10103DBB2012B07D000203DB065
:1009A000BDE8F08FCDF81080C14654E7479B049A0C
:1009B000B3F9027017F11F0648BF07F13E0646F370
:1009C0004716334651465846FDF72AFBD0B9B7EBD8
:1009D000461F80F2AB817B113CAA02EB830307F038
:1009E0001F0753F8C02C012303FA07F717420CBF67
:1009F000042300233CAA134453F8C87C03E00025D9
:100A0000A94649E75F463346049A594614A8FDF7BC
:100A100007FB01344799479B019324B200230094BC
:100A20003A461CA84431FFF72DFB059B022B40F2F0
:100A30009581039B00215E081CAB03EBC6060A46AA
:100A4000D3E9004008339E4241EA040142EA000231
:100A5000F6D1039800F0FE03984242EA010259B22F
:100A60001BD03CAB03EB8100CBB250F8800C591C7F
:100A70000243029849B288420FDD3CAC04EB81018D
:100A8000023351F8801C5BB2984242EA010204DD55
:100A900004EB830353F8803C1A43002A3FF47EAFF3
:100AA000B34B1968002900F043812A46049958463F
:100AB000FEF7E4F800283FF471AF2B465A46514642
:100AC0002CA8FDF70DFB049A2CA95046FEF70EFC4E
:100AD000069B032B40F24781B8F1000F00F03481F0
:100AE000DAF800C00127A9EB0804E4B20AEB880891
:100AF0006608002308EBC6061A46D8E9000108F18B
:100B00000808464543EA000342EA0102F5D104F031
:100B1000FE0013430744844243EA0C017BB21CD01D
:100B2000DAB25AF82300531C5BB29D4241EA00013D
:100B300013DD5AF82300931C5BB29D4241EA000189
:100B40000BDD5AF82300D31C5BB29D42C8BF5AF894
:100B5000233041EA0001C8BF1943002900F0F780A3
:100B60002B46049A51465046FEF7C2F92B465A4688
:100B700051462CA8FDF7B4FA049A2CA95046FEF76A
:100B8000B5FB479B93F90140002C16DD469A0027E0
:100B90003B46661E501EF31A23F003023CA90A448A
:100BA00003F00303013752F8802CD900FBB2CA408E
:100BB0009C4200F8012F5FB2EDDC479BB3F9026065
:100BC000F41D48BF06F10E04E410E31C48BFA31D4A
:100BD0009B105AB2002A07DD5A1ED2B2013292008F
:100BE0000021584601F0B2FB002E17DD00220998C3
:100BF0001346671EFB1A23F0030610F802C05BF8C9
:100C0000061003F00303DB0001320CFA03F352B2C7
:100C1000194394424BF806101346EBDC029B059AED
:100C2000002B05F1FF343CAB03EB840302F101021E
:100C30004FEA82021CA9D8BF0422002614A843F858
:100C4000A06C01F05BFB2B4614AA59462CA8FDF7BB
:100C500047FA049E2CA9324614A8FEF747FBDDE9AB
:100C60000712479B5846FEF7B3FE14AA1046594692
:100C700033460095FFF79CFB2B46524614A92CA83F
:100C8000FDF72EFA32462CA914A8FEF72FFB9DF98A
:100C90001820002A65DB13B23CA901EB830353F84B
:100CA000A03C002B5DD1A9F102035BB2013314A972
:100CB00001EB830303E053F8040D28B90A46541EE0
:100CC00061B2481CF7D17AB13CAB03EB820252F817
:100CD000A43C002B4AD000225B0802F10102FBD1A8
:100CE00092B202EB441212B2479B93F90150B2EB5D
:100CF000C50F3FF753AE002D16DD469A00210B4677
:100D00006E1E5419F31A23F003023CA8024403F0A8
:100D10000303013152F8A02CD800CBB2C2409D424F
:100D200004F8012B59B2EDDC012038E614AF6AE675
:100D3000069B5A1C9200584601F008FB01230C93B5
:100D4000BBE60022164604E6C4464746CBE6069BB1
:100D50005A1C9200504601F0F9FA07E700221146AA
:100D60007FE62A46B0E700210B46D9E61A46B8E7E7
:100D700084490020014B1860704700BF844900205F
:100D800000487047C44301082DE9F04FB3F90290C1
:100D9000A9B019F107049A4648BF09F10E0493F966
:100DA00000300293E41010AB0793E31C48BFA31D6F
:100DB0009B1005925AB208AE002A9AF90150069685
:100DC00083460F4607DD5A1ED2B20132920000213F
:100DD000304601F0BBFAB9F1000F16DD00221346D0
:100DE00004F1FF3EAEEB030323F0030017F802C04B
:100DF000315803F00303DB0001320CFA03F352B263
:100E00001943944231501346ECDCEB1C48BFAB1D38
:100E10009B105AB2002D03924EDD013BDAB218ACA2
:100E20000132920020460021049301F08FFA029BC8
:100E30004FF0000C04EB830705F1FF3863460BF11C
:100E4000FF3EA8EB030323F003011EF8010F6258D5
:100E500003F00303DB000CF1010C98405FFA8CF304
:100E600002439D4262504FFA83FCEADC002D0DDD07
:100E70009DF81020039B0132002B4FEA82024FF0B5
:100E80000001D8BF0422384601F060FA0022134660
:100E90000BEB0201A8EB030323F003004C5D395870
:100EA00003F00303DB00013204FA03F352B21943E7
:100EB000954239501346EBDC19F11F0748BF09F181
:100EC0003E0747F347170AF124083B46424631469E
:100ED0003046FDF7A5F80446002873D1B9EB471F4B
:100EE00010DA4FEA691328AA02EB830309F01F09FD
:100EF00053F8802C012303FA09F919EA020F14BFF1
:100F00001C4600243B463146424610A8FDF788F8AF
:100F10002D4B1E6866B128AB03EB8403029A53F88D
:100F2000886C0AF104013046FDF7A8FE002846D07F
:100F3000BAF80230CDF804A084F0010428AA02EB2C
:100F4000840201331BB218AC52F8882C009321465E
:100F500033462046FFF796F8002D16DD059B00214D
:100F60005E1E6F1E0B46FB1A23F0030228A80244E4
:100F700003F00303013152F8402CD800CBB2C24039
:100F80009D4206F8012F59B2EDDC9AF8002052007C
:100F9000D2B253B2002BD8BF002010DD002304EBE7
:100FA00082021946D4E900500834A24243EA0503FC
:100FB00041EA0001F6D10B4314BF0120002029B003
:100FC000BDE8F08F01249DE7844900202DE9F04F12
:100FD000B2F90270FD1D48BF07F10E05ED10EB1CC4
:100FE00048BFAB1D9B10AFB093465AB2002A0646CD
:100FF000029107DD5A1ED2B201329200002106A8EA
:1010000001F0A4F9002F17DD00210B46681E06AC85
:10101000C31A23F0030C16F801E054F80C2003F077
:101020000303DB0001310EFA03F349B21A438D4288
:1010300044F80C200B46EBDC17F11F0548BF07F105
:101040003E056D114FFA85F8B8F1000F40F394801A
:10105000EDB205F1FF395FFA89F9B9F1020F40F2FB
:10106000CF8006AC6F08002204EBC70C2346114664
:10107000D3E9006008339C4542EA060241EA0001D8
:10108000F6D125F0010A5FFA8AF0A84242EA01028D
:1010900043B275D02EA901EB8301DBB2581C51F885
:1010A000A01C40B2804542EA010210DD2EA901EBEE
:1010B0008000023350F8A01C5BB2984542EA01025E
:1010C00005DD2EA901EB830353F8A03C1A43002A47
:1010D00052D00BF1240306AC1EAE039319462246F0
:1010E00030464346FCF7CCFF10F1000E18BF4FF01E
:1010F000010EB9F1020F40F2F6806F0825F0010AE7
:10110000002206EBC70C11463346D3E900700833C2
:101110009C4542EA070241EA0001F6D15FFA8AFAE9
:10112000554542EA01024FFA8AF31BD02EA901EB82
:101130008301DBB251F8400C591C49B2884542EAA0
:1011400000020FDD2EA800EB8101023351F8401C94
:101150005BB2984542EA010204DD00EB830353F8D9
:10116000403C1A434FEA4E03002A0CBF5B42C3F1D6
:101170000103DBB2012B15D000202FB0BDE8F08FAA
:10118000002AF9D00BF124031EAE03931946304612
:1011900043462246FCF774FF10F1000E18BF4FF0D3
:1011A000010EADE7BBF90270039A17F11F0548BFA6
:1011B00007F13E050DF1380845F347150DF15809C3
:1011C00021462B464046CDE90489FCF729FFD0B9DA
:1011D000B7EB451F80F285807B112EAA02EB8303BB
:1011E00007F01F0753F8802C012303FA07F7174273
:1011F0000CBF042300232EAA134453F8A84C03E089
:101200000022134646E744462B46039A4146484689
:10121000FCF706FFBBF80230CDF804B001331BB277
:10122000224600930BF1440100233046FEF72AFFCB
:101230009BF800205200D2B253B2002B9CDD002359
:1012400006EB82021946D6E900400836964243EA88
:10125000040341EA0001F6D10B438DD09BF9015004
:10126000002D3ADD029A00210B466E1E541EF31A21
:1012700023F003022EA8024403F00303013152F8C5
:10128000402CD800CBB2C2409D4204F8012F59B285
:10129000EDDC9BF901409BF90060002C1DDD029BF9
:1012A000002123441846671E0B460425FB1A23F031
:1012B00003020DF1B80C16FB0522624403F0030390
:1012C000013152F8402C4FEAC30CCBB222FA0CF297
:1012D0009C4200F8012B59B2E8DC01202FB0BDE898
:1012E000F08F4C4690E7002213461FE72DE9F047A8
:1012F0008AB08246129D88461746994605F1240613
:10130000402407E0CDE900955046FFF77FFAB8B9D1
:10131000013C11D0B5F9023013F11F0248BF03F1AF
:101320003E02314642F3471202A8FDF7A7FC02AB8A
:101330003A4641460028E5D100200AB0BDE8F087D2
:1013400001200AB0BDE8F087F0B501F120020346A4
:101350000C781C704C785C708C789C70CC78DC704D
:101360000431914203F10403F2D1194A194F0826BE
:1013700016F0070C037F457F847FC17F20D112F8D0
:1013800005C0155D545CD15CF308FB5C8CEA03037B
:1013900090F800C083EA0C0380F8203043785D4069
:1013A000837880F821505C40C37880F82240013671
:1013B00059403C2E80F8231000F10400D8D1F0BD34
:1013C000BCF1040F01BFD35C555D145D515CDFE7D8
:1013D0007F4501087444010870B502EB00120C1D32
:1013E0001431231F1546187815F8016B704003F867
:1013F000010BA342F7D11C1D8C4202F10402F0D173
:1014000070BDC3095A00134403EBC30383EA4000D1
:10141000C0B270472DE9F04F0A4685B004468A46AF
:1014200001460020FFF7D8FF231D009304F11003AD
:1014300001270193A14623460CE013F822104848E7
:10144000415C03F822100132042AF6D1009A0133DC
:10145000934201D00022F0E7627963786270627A89
:101460006271627B6272A27A6373A378A270A27BBC
:10147000A372A379A271E27BA373E378E270E27AAC
:10148000E273E279E272E37121460B784E788D784F
:1014900091F803B0029385EA0B0283EA060080EA22
:1014A00002080392FFF7ADFF029B584088EA000054
:1014B000087086EA0500FFF7A4FF039A704088EAE7
:1014C000000048701046FFF79CFF029B684088EAC6
:1014D0000000887083EA0B00FFF793FF8BEA00009F
:1014E00088EA0008019B81F8038004319942CCD13D
:1014F0003846013752462146FFB2FFF76DFF0E2FE7
:1015000098D1174A002319F82310515C09F82310C9
:101510000133042BF7D1009B09F101099945F1D161
:10152000627963786270627A6271627B6272A27AB7
:101530006373A378A270A27BA372A379A271E27BEA
:10154000A373E378E270E27AE273E279E272214611
:1015500052460E20E37105B0BDE8F04FFFF73CBFE7
:101560007F4501082DE9F04F8FB0044603910A46EC
:1015700001460E20FFF730FF0D230293231D049335
:1015800004F110030B93627A637B62736279627277
:1015900062786271A27A6370A378A270A27BA37250
:1015A000A379A271E279A373E378E270E27AE2713F
:1015B000E27BE272E373A3462246002312F8231073
:1015C0006748415C02F823100133042BF6D1049BD9
:1015D00001329342F1D1039A02982146FFF7FCFEB3
:1015E00026463778737801933846FFF70AFF05904F
:1015F000FFF707FF0690FFF704FF0D900198B578FD
:1016000096F803A0FFF7FDFE0146FFF7FAFE0790EC
:10161000FFF7F7FE81462846FFF7F3FE0C90FFF731
:10162000F0FE0890FFF7EDFE80465046FFF7E9FE1A
:101630000990FFF7E6FE0A90FFF7E3FEDDE90532C9
:1016400083EA020C0D9B089A83EA0C0C81EA0C0CCD
:1016500089EA0C0C82EA0C0C88EA0C0C019A80EAEC
:101660000C0C82EA0C0C85EA0C0C079A8AEA0C0C2A
:10167000594086F800C05140DDF830C00A9A89EA26
:10168000010181EA0C0188EA0101514041407940A1
:10169000069A69408AEA0101717082EA030189EAC7
:1016A00001018CEA010208994A40099988EA02027C
:1016B0004A40424001997A404A408AEA020A86F842
:1016C00002A0059A5340079A534089EA0309099BEF
:1016D00088EA090883EA08080A9B83EA080880EA7E
:1016E000080047404F406F400B9BF7700436B342F1
:1016F0007FF477AF029B013B13F0FF0302937FF46B
:1017000042AF627A637B62736279627262786271FD
:10171000A27A6370A378A270A27BA372A379A2714C
:10172000E279A373E378E270E27AE271E27BE2723B
:101730000B4AE37300231BF82310515C0BF82310B2
:101740000133042BF7D1049B0BF1010B5B45F1D165
:10175000039A214600200FB0BDE8F04FFFF73CBED2
:101760007F440108FFF7F0BD2DE9F04100F1F005DD
:1017700007460E4690462B460C46A21B904509D8BC
:1017800003F1100253F8041B45F8041B9342F9D1EE
:10179000BDE8F081611E013B04F10F0211F8010F59
:1017A00013F801CF914280EA0C000870F6D1204670
:1017B0003946FFF72FFE23461034DEE72DE9FF47B9
:1017C0006FF00E068046914601F10F04761A0DF176
:1017D000100A33199945A4F10F0C02D804B0BDE8E2
:1017E000F0876A46634604F1010E15461868596889
:1017F000174603C7083373453A46F7D1414660465A
:10180000FFF7B0FEA4F1100308F1EF0113F8012F68
:1018100011F8010FA34282EA00021A70F6D108F112
:10182000F0072B4603CB5345386079601D4607F11E
:101830000807F6D11034CCE703680BB1013B036015
:101840007047F8B50446D0E90006331A9F1A002FF6
:1018500015460ADA1EB1D51A0023C4E900332368FD
:101860001D4425604FF0004005E000F047FD23686F
:101870001D4425600020F8BDDFB51F461646002F29
:1018800013BA08BF182E3ABA9DF82040CDE90223BA
:101890000DF10F0109D204EB13648DF80F4004AB76
:1018A0005A1AFFF7CEFF04B0D0BD002F08BFB6F51F
:1018B000807F2CBF01230023002F08BFB6F5803F97
:1018C00028BF0133012F08BF002E24BF0133DBB234
:1018D00001229A40891A183423440B70DFE71FB5A0
:1018E0000C46194603682360436863600830FFF7BD
:1018F000A3FF501C01F02003B2F1FF3FA060E360A2
:101900000DD11F3143F004038DF80F10E360012265
:101910000DF10F012046FFF794FF04B010BD0BB18D
:101920001044A060009100232046FFF7A5FFF4E7D4
:101930000A44426002220160C0E90223704737B5C1
:10194000014608301D46FFF777FF00230093084645
:101950002B46FFF791FF03B030BD37B5D9170546C9
:1019600008304A4083EA0104FFF766FF01F02001D6
:10197000009123462846FFF77FFF03B030BDA1F159
:101980001903062B13B504460BD90830FFF754FF93
:10199000E02300930A4600232046FFF76DFF02B0C4
:1019A00010BD4FF48370FAE773B5044608300E4655
:1019B0001546FFF741FF4023009320460023FFF721
:1019C0005BFF2A463146204602B0BDE87040FFF773
:1019D00038BF73B5044608300E461546FFF72CFF96
:1019E0006023009320460023FFF746FF2A46314636
:1019F000204602B0BDE87040FFF723BF8023FFF709
:101A00006EBF0000074B10B402F100449C4204D9A1
:101A1000A0235DF8044BFFF762BF4FF480605DF8D0
:101A2000044B7047FEFFFF7F0B6807B50360CB6870
:101A30004A68426013F004030CD0FF2301220DF129
:101A400007018DF80730FFF7FCFE0346184603B088
:101A50005DF804FB8968012906D0002940F20133B2
:101A600008BF4FF44073F1E7002A08BF4FF000436E
:101A7000ECE700F0DF00402803D0803818BF0120D9
:101A80007047002070470120704700F037BC0268A3
:101A9000FF2170B5817344681568AC42034602D1DA
:101AA00040F2011070BD227802F0E00102F01F0246
:101AB00081731B2A4FF00000D8739A8117D91F2A0F
:101AC00007D040F2051040F20313E02908BF184682
:101AD000E8E70846FFF7CDFF10B90422DA73E1E723
:101AE000E02940F2051008BF4FF48170DAE7172AA9
:101AF00007D9A2F118060120B04001302D1BA842E1
:101B0000CED84809012809D14FF40071D981172A8C
:101B100018D9182A21D162789A8113E00728F6D1C2
:101B2000143A072A0ED8DFE802F0040B0B0B0F0B58
:101B300009090020F52298819A73B3E70122DA732C
:101B400022789A730020ADE762789A811F2AF9D82B
:101B5000FF229A734FF48370A4E7192A03D1B4F8D3
:101B6000012052BAD8E7DA7B42F00102DA73E9E7E2
:101B70008268531C07D1D0E9001309688B4202D058
:101B80001978FF2901D0FFF782BF0133436000239A
:101B9000827383601846704783685A1C05D0827B25
:101BA000C02A02D0013B83600BB1FFF7E1BFFF22E7
:101BB00082731846704708B500F092FBB0FA80F0C7
:101BC000400908BD73B506683346054613F8010B96
:101BD0002B6000F01F00172806D8C0B20021C2E910
:101BE0000001002002B070BD1B2827D8183801243E
:101BF0008440C91AA14224D3012C06D17078002157
:101C0000C2E9000123442B60EBE7022C04D1B6F8B3
:101C1000010040BA80B2F2E7042C06D1D6F80110D8
:101C200009BA116000215160ECE7186859686E46E6
:101C300003C601BA019800BA1060F4E740F205103B
:101C4000D0E740F20110CDE72DE9D748044650F81F
:101C5000043B6A461968FFF7B5FF30B1134B144ACD
:101C60004FF4A571134800F0D3FAA37B03F0DF0310
:101C7000402B15D1DDE900BC844508BFDB4504D00D
:101C80000D4B0B4A40F24D11ECE7E17B4B0704D5BD
:101C90000A4B074A4FF4A771E4E763685B4463604B
:101CA0002046FFF779FF03B0BDE8D088324801082D
:101CB0007F46010845480108564801086F48010859
:101CC0002DE9774BC37B0D4699071646044603F072
:101CD000040207D56AB900232B6020463360FFF762
:101CE0005BFF0DE02AB1426843F00203013242601B
:101CF000C373D4E9002311688B4204D140F2011070
:101D000003B0BDE8708B1A78FF2A02D101336360FB
:101D1000E1E7A37B02F0E002934222D16A46201D54
:101D2000FFF750FF10B100233360E9E7DDE90089D8
:101D3000484508BFC045C6F800800FD1D4E9001659
:101D40000968891B4145D9D32E60636808EB0302FB
:101D5000E37B626043F00203E373D1E74FF48060FA
:101D6000CEE74FF48270CBE72DE9F04F1E46837B20
:101D700003F0DF0387B0402B8A469046DDE9105917
:101D800006D0244B244A25484FF4886100F040FADD
:101D900005B902AD0FC8002485E80F000123337098
:101DA000A34601AA69462846FFF78AFF0746A8B955
:101DB0000099D1B1019AA7180ED2337893B1D8F80F
:101DC0000030BB420ED30AEB0400C847003018BFF6
:101DD000012030703C46E4E74FF48067384607B096
:101DE000BDE8F08F86F800B0F4E7337873B1D8F827
:101DF0000030A3420AD98DF80400012201A90AEBA0
:101E00000400C847003018BF01203070C8F80040F7
:101E1000E4E700BF074001082F47010845480108D3
:101E200007B5C37BDB070BD4837B0633DBB2012B07
:101E300006D9164B164A4FF4B171164800F0E8F96E
:101E400043681A7802F01E011A2904D0124B104A76
:101E50004FF4B371F1E712F0010105D1D3F801009D
:101E600000BA03B05DF804FB02F01F021B2A04D085
:101E70000A4B074A4FF4B571DFE753F8010F596871
:101E80006A4603C208BA009909BAEAE75F4701083F
:101E90009046010845480108D54701080548010852
:101EA00010B4044601982144C3E90012C0E900348B
:101EB000012383605DF8044BFFF7E9BD08B50346D5
:101EC000807BFF2806D10C4B0C4A4FF4ED710C4877
:101ED00000F09EF9FFF7CDFD20B90A4B074A40F20A
:101EE000DB11F4E79A6822B11846BDE80840FFF715
:101EF000ABBE032008BD00BFA1480108B2460108DF
:101F000045480108BD48010810B50446A37BC02B15
:101F100001D0002004E02046FFF7D0FF0028F5D0D4
:101F200010BD0000F7B5837B03F0DF03802B05466F
:101F30000C4606D01F4B204A40F24D211F4800F0AE
:101F400067F90FC884E80F00EB7B5B0708D54FF0FB
:101F5000FF330131A36061602046FFF709FE1AE0FC
:101F600001686A46201DFFF72DFE20B1144B124A6E
:101F700040F25621E2E7DDE90023834208BF9242A6
:101F8000A26004D1002B08BFB2F1FF3F05D16B68FE
:101F900063604FF4806003B0F0BDA17BA02903D142
:101FA000002AF4DB5100A1601343D5D1FF23A373B2
:101FB000F1E700BFD5480108DE46010845480108A1
:101FC0003248010808B5837B03F0DF03802B06D07D
:101FD0000A4B0B4A40F27E210A4800F019F98B7B2C
:101FE000FF2B04D0084B064A40F27F21F4E74B68F0
:101FF0004360BDE80840FFF7CFBD00BFD5480108EA
:10200000F9460108454801080E490108F8B5837BE7
:1020100004460D4633B1134B134A144840F25D3168
:1020200000F0F6F8C37BDB0711D5FFF7F9FEE37B81
:1020300013F002036FF000464FF000070AD08F4202
:1020400008BF86420AD3C04328600020F8BD8089BB
:102050000021ECE78F4208BF8642F5D24FF4806042
:10206000F4E700BFF148010814470108454801089A
:1020700030B50A4C0A4D85B0002908BF2C46CDE981
:1020800000340DF10F03FFF76FFE28B99DF80F30F4
:10209000002B08BF4FF0004005B030BD8B1A01087F
:1020A000871A010830B5837B85B0044618460D4673
:1020B000FFF7DFFC014620B12046FFF7C5FD05B064
:1020C00030BD03F0DF03802B08D04FF0FF330093C7
:1020D0006A4623462046FFF7CBFFF0E7A5B16946E5
:1020E0002046FFF71FFF0028E9D1013D029B23B9DD
:1020F00069462046FFF766FFE1E729466846FFF795
:10210000D1FF0028F2D0DAE740F20140D7E7000023
:1021100008B5827BFF2A06D1074B084A084840F2DF
:102120000E2100F075F8836823B10321BDE8084053
:10213000FFF7B8BF032008BDA1480108CB4601083E
:10214000454801084FF0FF330B6000230A4619464B
:10215000FFF78EBF2DE9FF41054608460E4614469F
:1021600000F0AAFDAB7BA02B074606D0204B214AEE
:10217000214840F21F5100F04BF828462146FFF756
:10218000D1FE054680BBDFF87480A3682BB9FF231E
:10219000A373284604B0BDE8F0812046FFF7B4FEE3
:1021A00010BBA37B602B12D1CDE900480DF10B03CE
:1021B00003AA314620460397FFF7D6FDA0B99DF844
:1021C0000B3043B12046FFF762FC0546E1E72046AD
:1021D000FFF79EFF40B92046FFF796FE20B9204644
:1021E000FFF796FF0028D0D0FF23A373EDE700BFD1
:1021F000304901084547010845480108B71B010857
:1022000008B5062000F032FD012001F05FFA000061
:102210001FB51C46094B1B680546D86852B1084BD0
:102220000091CDE9013207492B46224600F022F801
:10223000FFF7E6FF044B1A46F2E700BFE801002073
:102240004749010854490108013E010808B5074BF8
:10225000044613B10021AFF30080054B1868836A70
:1022600003B19847204601F031FA00BF000000009A
:10227000844901080EB403B5014603AB054853F881
:10228000042B0068019300F093F802B05DF804EBB2
:1022900003B07047E801002070B50D4D0D4C641B74
:1022A000A4100026A64209D10B4D0C4C02F0AEFB47
:1022B000641BA4100026A64205D170BD55F8043B4E
:1022C00098470136EEE755F8043B98470136F2E7A8
:1022D00000000000000000000000000000000000FE
:1022E00030B501390024A24201D1002005E0035D90
:1022F00001340D5DAB42F6D0581B30BD0A4491420B
:1023000000F1FF3300D1704710B511F8014B03F80D
:10231000014F9142F9D110BD884210B501EB020383
:1023200002D983421C4607D8421E994208D011F8B0
:10233000014B02F8014FF8E783189A1A9A4200D12C
:1023400010BD14F8011D03F8011DF7E70244034610
:10235000934200D1704703F8011BF9E79368013BF2
:10236000002B10B4936008DA9469A34201DB0A29B8
:1023700003D15DF8044B00F0B9BC1368581C106021
:10238000197008465DF8044B7047F8B506460F46CD
:102390001446D518AC4201D1002007E03A4614F8A3
:1023A000011B3046FFF7DAFF431CF3D1F8BD0000F4
:1023B0002DE9F04F0D469DB014461E46074618B154
:1023C00083690BB900F06CFE854B9D421BD17D6883
:1023D0006B6ED90705D4AB899A0502D4A86D00F0BD
:1023E000FCFEAB891B0701D52B69EBB929463846A2
:1023F00000F0CEFCC0B16B6ED8070ED54FF0FF30A9
:102400001DB0BDE8F08F774B9D4201D1BD68DFE77D
:10241000754B9D4208BFFD68DAE7AB899905EDD49D
:10242000A86D00F0DBFEE9E70023099320238DF877
:102430002930DFF8B891039630238DF82A304FF019
:10244000010A23461E4613F8012B0AB1252AF9D1A9
:10245000B6EB040B0BD05B46224629463846FFF705
:1024600094FF013000F0A380099B5B44099333780B
:10247000002B00F09C8000234FF0FF32CDE90523B4
:102480000136049307938DF853301A93344605228E
:1024900014F8011B554800F00BFF049BC0B9DA0685
:1024A00044BF20228DF85320180744BF2B228DF8FB
:1024B000532032782A2A13D0079A344600200A265D
:1024C000214611F8013B303B092B4BD970B914E080
:1024D000A0EB09000AFA00F0184304902646D5E75D
:1024E000039A111D12680391002A01DB079204E090
:1024F000524243F002030792049323782E2B0CD10F
:1025000063782A2B33D1039B1A1D1B680392002B7F
:10251000B8BF4FF0FF3302340593354E21780322C4
:10252000304600F0C5FE38B14023801B03FA00F0AE
:10253000049B03430134049314F8011B2D488DF8C8
:102540002810062200F0B4FE00283FD02A4B13BB0F
:10255000039B073323F0070308330393099B43448A
:1025600009936EE706FB023201200C46A8E7002320
:102570000134059319460A26204610F8012B303AFB
:10258000092A03D9002BC8D00591C6E706FB012113
:1025900001230446F0E703AB00932A46174B04A936
:1025A0003846AFF30080B0F1FF3F8046D6D16B6E66
:1025B000D90705D4AB899A0502D4A86D00F00EFEA8
:1025C000AB895B063FF51AAF099819E703AB009397
:1025D0002A460A4B04A9384600F088F8E3E700BF12
:1025E000CC490108EC490108AC49010888490108B7
:1025F0008E49010892490108000000008B23010860
:102600002DE9F04791461F468A680B69DDF8208066
:102610009342B8BF1346C9F8003091F843200646EC
:102620000C4612B10133C9F800302368990642BF45
:10263000D9F800300233C9F80030256815F00605D6
:1026400007D104F1190AE368D9F800209B1AAB42BC
:1026500028DC94F843302268003318BF0123920627
:102660002DD404F1430239463046C047013020D012
:102670002368E568D9F8002003F00603042B08BF9F
:10268000AD1AA36822690CBF25EAE57500259342BF
:10269000C4BF9B1AED184FF000091A344D451AD1EA
:1026A000002008E00123524639463046C047013039
:1026B00003D14FF0FF30BDE8F0870135C3E7E118E3
:1026C0005A1C302081F84300224494F8451082F8C7
:1026D00043100233C5E70123224639463046C0473E
:1026E0000130E6D009F10109D8E700002DE9F043F7
:1026F00006460C4601F14300097E85B06E299846D6
:1027000017460C9B00F0BA8024D8632939D00AD828
:10271000002900F0C380582900F0918004F142059F
:1027200084F8421035E0642901D06929F6D1256882
:102730001A6815F0800F02F104012CD0126819609C
:10274000002A03DA2D23524284F84330DFF8BCC15B
:102750000A233FE0732900F0A58008D86F2921D013
:102760007029DBD1226842F02002226003E0752943
:1027700018D07829D2D1782284F84520DFF890C18A
:1027800061E01A68111D1960136884F8423004F181
:102790004205012393E01268196015F0400F18BF3D
:1027A00012B2CDE7D4F800C01A681CF0800F02F115
:1027B00004051D6001D0126803E01CF0400FFAD040
:1027C0001288DFF848C16F290CBF08230A230021B3
:1027D00084F843106568A560002DA2BF216821F030
:1027E000040121600AB9002D46D00546B2FBF3F181
:1027F00003FB112E93421CF80EE005F801ED39D9C8
:10280000082B0BD12368DA0708D5236962689A423E
:10281000DEBF302305F8013C05F1FF35401B206188
:10282000CDF800803B4603AA21463046FFF7E8FE7C
:10283000013049D14FF0FF3005B0BDE8F083DFF83B
:10284000CCC084F845101D68216855F8042B1D6024
:102850000D060BD5CD0744BF41F0200121601AB908
:10286000236823F0200323601023B0E74B0648BF02
:1028700092B2EFE70A46B9E70546C1E71A68D4F80D
:1028800000C06169151D1D601CF0800F136801D028
:10289000196003E01CF0400FFAD019800023236177
:1028A0000546BDE71A68111D1960156862680021A8
:1028B000284600F0FDFC08B1401B6060636823619E
:1028C000002384F84330ABE723692A463946304673
:1028D000C0470130AED023689B0713D4E068039B48
:1028E0009842B8BF1846A7E701234A463946304602
:1028F000C04701309ED00135E368039A9B1AAB4272
:10290000F2DCEBE7002504F11909F5E74B3E01087D
:1029100099490108022B10B50AD09208013A0368C0
:102920000C6840F8044B002A41F8043BF6DC10BD6B
:1029300002440C78037800F8014B01F8013B131AAC
:10294000002BF6DCF3E7F8B50F46144606461D46A5
:1029500098470028214638460CDAA847002802DAB2
:102960003C462046F8BD21463046A8470028F8DB03
:102970003446F6E7A8470028F2DC21463046A8474F
:102980000028EEDAF4E72DE9F04F97B007460193FF
:1029900040EA02039B07144618D1B2F1040818BF9D
:1029A0004FF001080023029304FB01F6BB1906292E
:1029B00007EB0409039328D8039B4B4510D8029BCF
:1029C000002B40F01A8117B0BDE8F08F4FF00208DD
:1029D000E8E74346224631462846FFF79BFF0FE0D3
:1029E0004D460EE02E1B29463046019B9847002895
:1029F00009DDB8F1000FECD12B6832682A60336032
:102A00003546AF42EED3A144D6E74FEA510A361B12
:102A1000072904FB0A7A3E4421D0282944D9C90851
:102A200004FB01F579194A19019B3846FFF78BFF22
:102A300051460AEB0502019B8346481BFFF783FFC3
:102A40008246A6EB45003246019B4119FFF77BFF0A
:102A500002465146019B5846FFF775FF8246B8F182
:102A6000000F24D13B68DAF800203A60CAF8003041
:102A7000CB46B2464D460023B34536D8049339467B
:102A8000019B584698470028049B3DDC0AD1B8F1C9
:102A9000000F13D12B68DBF800202A60CBF8003040
:102AA00025440123A344E7E73246BB46D1E743462A
:102AB000224651463846FFF72DFFD9E743462246C6
:102AC00059462846FFF726FFEAE70BD1B8F1000F79
:102AD00013D13368DAF800203260CAF80030AAEB6C
:102AE000040A0123049EB3450ED9002B42D1039B57
:102AF0004B457FF664AF4D4638E04346224651468B
:102B00003046FFF707FFEAE705933946019B304659
:102B10009847331B00280493059BD6DAB8F1000FC1
:102B200006D04346224631465846FFF7F3FE05E0FD
:102B3000DBF800303268CBF800203360049EB0E749
:102B40004346224631462846FFF7E4FE0DE02E1BA1
:102B500029463046019B9847002809DDB8F1000F4F
:102B6000EED12B6832682A6033603546AF42EED32F
:102B7000A144BCE7ABEB0509EA1B4A45A8BF4A469E
:102B80002AB14346ABEB02013846FFF7C3FE039B75
:102B9000A3EB0A02AAEB0606121BB24228BF32467A
:102BA0002AB103994346891A5846FFF7B3FE039B9F
:102BB0004E45CA46A3EB060004D93B46B24607463B
:102BC0004E461846A64221D9B6FBF4F1029B072BCC
:102BD0000DD816AA02EBC303BAFBF4F243F8407C0B
:102BE00043F83C2C029B013302930746DCE6019B31
:102BF0002246FFF7C8FEA2450BD8029B16AA013B4E
:102C0000029302EBC30353E91001EEE7A2457FF6FE
:102C1000D6AEBAFBF4F13846E7E71F2938B50446CB
:102C20000D4604D9162303604FF0FF3038BD426CC7
:102C300012B152F821304BB9204600F031F82A4643
:102C400001462046BDE8384000F018B8012B0AD0F4
:102C5000591C03D1162303600120E7E7002442F842
:102C60002540284698470020E0E70000024B014637
:102C70001868FFF7D2BF00BFE801002038B5074C45
:102C80000023054608461146236000F0F1FC431C72
:102C900002D1236803B12B6038BD00BF0C71002046
:102CA00000F0D6BC10F8012B11F8013B012A28BF17
:102CB0009A42F7D0D01A7047034613F8012B002A26
:102CC000FBD1181A0138704710B56AB10139841860
:102CD00010F8013B11F8012F934203D1A04201D01B
:102CE000002BF5D1981A10BD1046FCE7F8B50E463A
:102CF0001446054618B183690BB900F0D1F9214B90
:102D00009C422BD16C68A369A360A3891A072FD5B5
:102D100023696BB323692068C01A6369F6B28342E2
:102D2000374604DC2146284600F026F930BBA3686C
:102D3000013BA36023685A1C22601E706369013046
:102D4000834204D0A389DB0706D50A2E04D121468D
:102D5000284600F011F988B93846F8BD0A4B9C4264
:102D600001D1AC68CFE7094B9C4208BFEC68CAE7C9
:102D70002146284600F00CF80028CBD04FF0FF3752
:102D8000EAE700BFCC490108EC490108AC49010859
:102D9000324B70B51D6806460C4625B1AB6913B9B8
:102DA000284600F07DF92E4B9C420FD16C68B4F997
:102DB0000C309AB215072CD4D00611D409223260F7
:102DC00043F04003A3814FF0FF303EE0254B9C428F
:102DD00001D1AC68EBE7244B9C4208BFEC68E6E706
:102DE000510712D5616B41B104F14403994202D0FD
:102DF000304600F0ADFA00236363A38923F0240377
:102E0000A3810023636023692360A38943F008033F
:102E1000A38123694BB9A38903F42073B3F5007F21
:102E200003D02146304600F0FFF9A28912F00103D9
:102E30000CD00023A36063695B42A361236953B98B
:102E4000B4F90C3013F08000BAD170BD920758BFAE
:102E50006369A360F2E70020F7E700BFE801002004
:102E6000CC490108EC490108AC4901088A892DE9DF
:102E7000F041054610070C4658D44B68002B05DC82
:102E80000B6C002B02DC0020BDE8F081E66A002E0E
:102E9000F9D0002312F480522F682B6032D0606D7D
:102EA000A3895A0705D56368C01A636B0BB1236CFD
:102EB000C01A00230246E66A216A2846B047431C2E
:102EC000A38906D129681D292CD82A4ACA40D607C9
:102ED00028D500226260D9042269226004D5421CF0
:102EE00001D12B6803B96065616B2F600029CAD0DE
:102EF00004F14403994202D0284600F029FA002048
:102F00006063C1E7216A01232846B047411CC7D14D
:102F10002B68002BC4D01D2B01D0162B01D12F60A4
:102F2000B1E7A38943F04003A381ADE70F69002F08
:102F3000A9D093070E6808BF4B690F6018BF002324
:102F4000A6EB07088B60B8F1000F9CDD43463A46BC
:102F5000216AA66A2846B047002806DCA38943F008
:102F60004003A3814FF0FF308EE70744A8EB000831
:102F7000E9E700BF0100402038B50B6905460C4663
:102F800013B90025284638BD18B183690BB900F084
:102F900087F8144B9C421BD16C68B4F90C30002BA1
:102FA000EFD0626ED00704D4990502D4A06D00F072
:102FB00014F928462146FFF759FF636EDA070546E4
:102FC000E0D4A3899B05DDD4A06D00F007F9D9E713
:102FD000054B9C4201D1AC68DFE7044B9C4208BF23
:102FE000EC68DAE7CC490108EC490108AC49010872
:102FF000002310B50446C0E9003383608181436635
:10300000C281C0E904338361194608225C30FFF7AE
:103010009DF9054B6362054BA362054BE362054BCB
:103020002462236310BD00BFC1340108E3340108EA
:103030001B3501083F350108014900F0AFB800BF5A
:10304000792F010870B54A1E682555430E4605F1D3
:10305000740100F0CBF9044640B10021C0E900162C
:103060000C30A06005F16802FFF770F9204670BDD2
:10307000014800F0B2B800BF0A710020014800F01A
:10308000ADB800BF0A710020014800F0A6B800BF2B
:1030900005710020014800F0A1B800BF05710020B3
:1030A00010B50446FFF7F0FFA3691BB1BDE810405F
:1030B000FFF7F0BFC4E912332365134B134A1B68B3
:1030C000A262A34204BF0123A361204600F020F8BE
:1030D0006060204600F01CF8A060204600F018F860
:1030E0000022E06004216068FFF782FF01220921CD
:1030F000A068FFF77DFF02221221E068FFF778FF4A
:103100000123A361D2E700BF8449010839300108D7
:10311000F8B50746FFF7ACFF1E4B1E68B36913B93D
:103120003046FFF7BDFF4836D6E90134013B03D5F1
:1031300033680BB33668F7E7B4F90C50D5B9164BC2
:10314000E36004F15800656600F046F8FFF796FF6B
:103150002560C4E90155C4E90455A5610822294642
:1031600004F15C00FFF7F2F8C4E90D55C4E912550B
:103170002046F8BD6834D9E704213846FFF762FFDE
:10318000044630600028D5D1FFF778FF0C233B6060
:10319000EEE700BF844901080100FFFF2DE9F84375
:1031A0008046894600F14804002614B93046BDE83F
:1031B000F883D4E90175013F01D52468F5E7AB89AF
:1031C000012B07D9B5F90E30013303D0294640460B
:1031D000C84706436835EEE770477047704770B5DB
:1031E0000E46B1F90E10002996B014461D4607DAB6
:1031F00000232B60B3891A0610D44FF480630EE0CD
:103200006A4600F0C3F90028F2DB019A02F470422A
:10321000A2F500535A425A412A60EEE740230020AB
:10322000236016B070BD00008B8973B59D070646FC
:103230000C4607D504F14703236023610123636132
:1032400002B070BD01AB6A46FFF7C9FF00990546A1
:10325000304600F0CBF848B9B4F90C309A05EFD4F9
:1032600023F0030343F00203A381E3E70D4BB362B2
:10327000A389206043F08003A381009B6361019BCD
:1032800020615BB1B4F90E10304600F091F928B11D
:10329000A38923F0030343F00103A381A3891D4302
:1032A000A581CDE7393001080000000000000000D2
:1032B00001F0FF01102A2BDB10F0070F08D010F8E7
:1032C000013B013A8B422DD010F0070F42B3F6D1EB
:1032D000F0B441EA012141EA014122F007047FF004
:1032E00000070023F0E80256083C85EA010586EA5B
:1032F000010685FA47F5A3FA87F586FA47F6A5FA97
:1033000087F68EB9EED1F0BC01F0FF0102F00702A2
:1033100032B110F8013B013A83EA010313B1F8D14D
:103320000020704701387047002D06BF354603382E
:10333000073815F0010F07D1013015F4807F02BF67
:10334000013015F4C03F0130F0BC0138704700BFB8
:1033500038B50546002945D051F8043C0C1F002B18
:10336000B8BFE41800F046F91F4A1368104633B995
:10337000636014602846BDE8384000F041B9A342BC
:103380000CD921686218934204BF1A685B686360B5
:1033900004BF521822600460ECE713465A680AB171
:1033A000A242FAD919685818A0420BD120680144EA
:1033B000581882421960DDD1106852685A60014481
:1033C0001960D7E702D90C232B60D3E720682118B6
:1033D0008A4204BF11685268626004BF0918216004
:1033E0005C60C7E738BD00BF88490020F8B5CD1C38
:1033F00025F0030508350C2D38BF0C25002D064699
:1034000001DBA94203D90C2333600020F8BD00F092
:10341000F1F821490A6814469CB9204F3B6823B94A
:103420002146304600F03CF838602946304600F02E
:1034300037F8431C23D10C233360304600F0E0F80A
:10344000E3E723685B1B17D40B2B03D923601C44D1
:10345000256004E06368A2420CBF0B6053603046F5
:1034600000F0CEF804F10B00231D20F00700C21A73
:10347000CCD01B1AA350C9E722466468CCE7C41C11
:1034800024F00304A042E3D0211A304600F008F8EB
:103490000130DDD1CFE700BF884900208C490020F2
:1034A00038B5064C002305460846236000F0F8F8BE
:1034B000431C02D1236803B12B6038BD0C7100207E
:1034C00010B50C46B1F90E1000F0A0F80028ABBF03
:1034D000636DA3891B1823F48053ACBF6365A3817C
:1034E00010BD2DE9F0411F468B89DB0505460C46D2
:1034F000164605D502230022B1F90E1000F068F837
:10350000A389B4F90E1023F48053A38132463B46BD
:103510002846BDE8F04100F017B810B50C46B1F9E7
:103520000E1000F055F8431CA38915BF606523F405
:10353000805343F48053A38118BFA38110BDB1F918
:103540000E1000F013B8000038B5074C05460846C9
:103550001146002222601A4600F0B0F8431C02D146
:10356000236803B12B6038BD0C71002038B5064CC0
:10357000002305460846236000F05AF8431C02D198
:10358000236803B12B6038BD0C71002038B5074C9F
:103590000023054608461146236000F051F8431CFD
:1035A00002D1236803B12B6038BD00BF0C7100202D
:1035B00038B5064C002305460846236000F050F855
:1035C000431C02D1236803B12B6038BD0C7100206D
:1035D00038B5074C054608461146002222601A46B7
:1035E00000F04EF8431C02D1236803B12B6038BDB4
:1035F0000C7100200148FFF7F0BD00BF06710020EC
:103600000148FFF7EBBD00BF0671002038B5074C3D
:10361000054608461146002222601A4600F038F896
:10362000431C02D1236803B12B6038BD0C7100200C
:10363000024B58221A604FF0FF3070470C71002087
:10364000024B58221A604FF0FF3070470C71002077
:10365000024B58221A604FF0FF3070470C71002067
:10366000024B58221A600020704700BF0C710020E6
:10367000024B58221A604FF0FF3070470C71002047
:10368000024B58221A604FF0FF3070470C71002037
:10369000024B58221A604FF0FF3070470C71002027
:1036A000044A05491368002B08BF0B4618441060F4
:1036B000184670479049002010710020024B582294
:1036C0001A604FF0FF3070470C710020FEE700BF1A
:1036D0007372632F696E69742E63001B2626ECC813
:1036E000F69B0F69E34FB236D76466BA12AC16C3C5
:1036F000AB5750BA064E8B90E02448008876631B87
:10370000D4A0427F57730EC71C9E027900308202FC
:10371000E93082028EA003020102020101300A0692
:10372000082A8648CE3D040302308182310B3009DD
:103730000603550406130255533111300F06035585
:1037400004080C084D6172796C616E64311430129A
:10375000060355040A0C0B534F4C4F204841434B72
:1037600045523110300E060355040B0C07526F6F93
:10377000742043413115301306035504030C0C73B8
:103780006F6C6F6B6579732E636F6D3121301F061F
:10379000092A864886F70D010901161268656C6CC6
:1037A0006F40736F6C6F6B6579732E636F6D302034
:1037B000170D3138313231313032323031325A181E
:1037C0000F32303638313132383032323031325ACD
:1037D000308194310B30090603550406130255530A
:1037E0003111300F06035504080C084D6172796CD5
:1037F000616E6431143012060355040A0C0B534FEA
:103800004C4F204841434B4552312230200603554E
:10381000040B0C1941757468656E74696361746F8B
:1038200072204174746573746174696F6E31153000
:103830001306035504030C0C736F6C6F6B6579737F
:103840002E636F6D3121301F06092A864886F70DD9
:10385000010901161268656C6C6F40736F6C6F6BB9
:103860006579732E636F6D3059301306072A8648C9
:10387000CE3D020106082A8648CE3D0301070342D9
:1038800000047D78F6BECA40763BC75CE3ACF42703
:1038900012C394981337A6410E92F69A3B15478DA2
:1038A000B6CED9D34F3913ED127B81143BE8F94CD6
:1038B0009638FEE3D6CB1B5393A274F7139A0F9D51
:1038C0005EA6A381DE3081DB301D0603551D0E048C
:1038D0001604149AFBA2210923B5E47A2A1D7A6CF6
:1038E0004E038992A30EC23081A10603551D230405
:1038F0008199308196A18188A48185308182310BA4
:1039000030090603550406130255533111300F06D2
:10391000035504080C084D6172796C616E643114B2
:103920003012060355040A0C0B534F4C4F204841EC
:10393000434B45523110300E060355040B0C075211
:103940006F6F742043413115301306035504030C87
:103950000C736F6C6F6B6579732E636F6D312130F3
:103960001F06092A864886F70D01090116126865A7
:103970006C6C6F40736F6C6F6B6579732E636F6DDA
:10398000820900EBD4845014ABD15730090603559B
:103990001D1304023000300B0603551D0F040403F1
:1039A0000204F0300A06082A8648CE3D04030203CA
:1039B00049003046022100A17B2A1D4E42A8686DB5
:1039C00065611EF5FE6DC699AE7C208316BAD6E5FC
:1039D0000FD70D7E05DAC90221009249F30B57D1AA
:1039E0001972F2755AA2E0B6BD0F0738D0E5A24FA2
:1039F000A0F3876182D8CD48FC570000ED023082E9
:103A00000303308202AAA003020102020101300A6C
:103A100006082A8648CE3D040302308180310B30EF
:103A2000090603550406130255533111300F0603DE
:103A30005504080C084D6172796C616E6431123066
:103A400010060355040A0C09536F6C6F204B6579FF
:103A5000733110300E060355040B0C07526F6F7450
:103A60002043413115301306035504030C0C736FCA
:103A70006C6F6B6579732E636F6D3121301F060992
:103A80002A864886F70D010901161268656C6C6F6D
:103A900040736F6C6F6B6579732E636F6D30201799
:103AA0000D3139313230313139323334395A180F1E
:103AB00032303639313131383139323334395A30A4
:103AC0008191310B30090603550406130255533119
:103AD00011300F06035504080C084D6172796C61B2
:103AE0006E643111300F060355040A0C08536F6CD5
:103AF0006F4B65797331223020060355040B0C1986
:103B000041757468656E74696361746F7220417485
:103B1000746573746174696F6E31153013060355E3
:103B200004030C0C736F6C6F6B6579732E636F6D90
:103B30003121301F06092A864886F70D0109011632
:103B40001268656C6C6F40736F6C6F6B6579732E68
:103B5000636F6D3059301306072A8648CE3D020147
:103B600006082A8648CE3D0301070342000422FED0
:103B70000FB52A78BEC645371A28A7574349A46F00
:103B8000854DCA4E251C9F75303DBF10D5D2D20B36
:103B9000B9692CDDB25C14D8398512F623EE91BADE
:103BA000C6ACFF4A1A27EFE0C1543FD4D9C5A38160
:103BB000FF3081FC301D0603551D0E041604143B16
:103BC000E6D2C06FF2E7B07C9D9E28C020B00D0702
:103BD000C815C830819F0603551D23048197308185
:103BE00094A18186A48183308180310B3009060342
:103BF000550406130255533111300F0603550408BE
:103C00000C084D6172796C616E64311230100603DC
:103C100055040A0C09536F6C6F204B657973311092
:103C2000300E060355040B0C07526F6F742043418E
:103C30003115301306035504030C0C736F6C6F6B56
:103C40006579732E636F6D3121301F06092A86480E
:103C500086F70D010901161268656C6C6F40736F71
:103C60006C6F6B6579732E636F6D820900C4476357
:103C7000928FF4BE8C30090603551D1304023000E8
:103C8000300B0603551D0F0404030204F030210617
:103C90000B2B0601040182E51C010104041204102F
:103CA0008876631BD4A0427F57730EC71C9E02798F
:103CB000300A06082A8648CE3D0403020347003036
:103CC0004402204DEA09156C8648572AA88D87C3FF
:103CD000FAB66B299BFB8B4D4D29775BA1044C7F7A
:103CE000128D710220474C3DB2A174E39CFEE1238A
:103CF000BFEC4796F4E59B6576ACC8691DE274FF9E
:103D00004EA4CF026D000703EA09156C8648572AB6
:103D1000A88D003433385A180F32303639313131EA
:103D200038313932343338006D7B412BFF57F00383
:103D3000BD5B394AF7A92D6DCB9E2D88BFB393C5C6
:103D4000663BD1BC34FA5C4C0220590149391BB79F
:103D5000A91CED49784F92A96114A56E963F2902DE
:103D600093E05DE275D060D974C2003530325A18E4
:103D70000F32303639313131383139323530320065
:103D80004D08C89DC4504970484DD012D97C625E20
:103D90006BD384D53642FE868E7A2359A020F0C597
:103DA00002205F7093615AE420CFB98AF5DD87D095
:103DB000486D7D59EF9E0E11A38EF7E3E2F535377E
:103DC000991A00F201A0000006472F000100D276E8
:103DD0000000850101000000000F20007F007F042B
:103DE00006E104007F0000536F6C6F4B657920740F
:103DF0006170005532465F5632001256ABF000E15A
:103E00000300E104006C69622F757362642F75739F
:103E100062645F636F6E662E630012010002000031
:103E200000408304CAA2000101020301536F6C6FBA
:103E30004B65797300536F6C6F20332E312E332D09
:103E4000322D6764643137383534003031323334E1
:103E500035363738394142434445460004030904A6
:103E6000616C670073696700783563006964006995
:103E7000636F6E006E616D6500646973706C61796B
:103E80004E616D650074797065007075626C696370
:103E90002D6B6579004649444F5F325F3000726B8D
:103EA00000757000706C617400636C69656E7450AD
:103EB000696E007061636B6564002E2E2F2E2E2FAD
:103EC0006669646F322F637461702E6300686D6180
:103ED000632D7365637265740063626F725F7661F0
:103EE0006C75655F6765745F626F6F6C65616E00AE
:103EF00063626F725F76616C75655F6765745F732F
:103F00007472696E675F6C656E6774680063626F78
:103F1000725F76616C75655F636F70795F746578E9
:103F2000745F737472696E670063626F725F76614B
:103F30006C75655F636F70795F627974655F7374C8
:103F400072696E670063626F725F76616C75655F40
:103F50006765745F61727261795F6C656E677468C2
:103F60000063626F725F76616C75655F6765745F31
:103F70006D61705F6C656E6774680063626F725F1D
:103F800076616C75655F69735F627974655F737480
:103F900072696E672876616C7565290063626F725D
:103FA0005F76616C75655F69735F617272617928B4
:103FB00076616C7565290063626F725F76616C75FE
:103FC000655F69735F626F6F6C65616E2876616CA7
:103FD000756529002E2E2F2E2E2F74696E7963623F
:103FE0006F722F7372632F63626F722E6800636249
:103FF0006F725F76616C75655F69735F6D61702864
:1040000076616C7565290063626F725F76616C75AD
:10401000655F69735F627974655F737472696E67F7
:104020002876616C756529207C7C2063626F725FE5
:1040300076616C75655F69735F746578745F7374BE
:1040400072696E672876616C756529007576006DFA
:104050006967726174655F66726F6D5F46465F7413
:104060006F5F303100646F5F6D6967726174696F93
:104070006E5F69665F7265717569726564007374FD
:104080006174655F63757272656E742D3E646174F0
:10409000615F76657273696F6E203D3D20535441B8
:1040A00054455F56455253494F4E007374617465D1
:1040B0005F746D705F7074722D3E5F7265736572B0
:1040C000766564203D3D2073746174655F70726530
:1040D000765F307866662D3E70696E5F636F6465EB
:1040E0005F6C656E677468002E2E2F2E2E2F66690A
:1040F000646F322F646174615F6D696772617469A6
:104100006F6E2E630073746174655F707265765FA5
:10411000307866662D3E69735F696E697469616C9B
:10412000697A6564203D3D2073746174655F746DC8
:10413000705F7074722D3E69735F696E6974696136
:104140006C697A65640073746174655F707265761A
:104150005F307866662D3E69735F70696E5F736568
:1041600074203D3D2073746174655F746D705F7081
:1041700074722D3E69735F70696E5F73657400734E
:10418000746174655F707265765F307866662D3E27
:1041900072656D61696E696E675F747269657320BF
:1041A0003D3D2073746174655F746D705F707472EF
:1041B0002D3E72656D61696E696E675F74726965C7
:1041C000730073746174655F707265765F307866D2
:1041D000662D3E726B5F73746F726564203D3D2087
:1041E00073746174655F746D705F7074722D3E726C
:1041F0006B5F73746F726564006D656D636D7028BD
:1042000073746174655F707265765F307866662D71
:104210003E6B65795F6C656E732C20737461746599
:104220005F746D705F7074722D3E6B65795F6C6545
:104230006E732C2073697A656F6628737461746578
:104240005F746D705F7074722D3E6B65795F6C6525
:104250006E732929203D3D2030006D656D636D70C2
:104260002873746174655F707265765F3078666616
:104270002D3E6B65795F73706163652C207374618B
:1042800074655F746D705F7074722D3E6B65795FDD
:1042900073706163652C2073697A656F6628737427
:1042A0006174655F746D705F7074722D3E6B6579BB
:1042B0005F73706163652929203D3D2030008C27A4
:1042C00090F60000982F8A4291443771CFFBC0B519
:1042D000A5DBB5E95BC25639F111F159A4823F92D1
:1042E000D55E1CAB98AA07D8015B8312BE8531242A
:1042F000C37D0C55745DBE72FEB1DE80A706DC9BEB
:1043000074F19BC1C1699BE48647BEEFC69DC10F96
:10431000CCA10C246F2CE92DAA84744ADCA9B05CD2
:10432000DA88F97652513E986DC631A8C82703B095
:10433000C77F59BFF30BE0C64791A7D55163CA06A3
:1043400067292914850AB72738211B2EFC6D2C4DAF
:10435000130D385354730A65BB0A6A762EC9C2819D
:10436000852C7292A1E8BFA24B661AA8708B4BC233
:10437000A3516CC719E892D1240699D685350EF45D
:1043800070A06A1016C1A419086C371E4C77482714
:10439000B5BCB034B30C1C394AAAD84E4FCA9C5B8A
:1043A000F36F2E68EE828F746F63A5781478C884DB
:1043B0000802C78CFAFFBE90EB6C50A4F7A3F9BEBD
:1043C000F27871C608200001FFFFFFFFFFFFFFFF2B
:1043D000FFFFFFFF000000000000000000000000E1
:1043E00001000000FFFFFFFF512563FCC2CAB9F3C3
:1043F000849E17A7ADFAE6BCFFFFFFFFFFFFFFFF9C
:1044000000000000FFFFFFFF96C298D84539A1F4D5
:10441000A033EB2D817D0377F240A463E5E6BCF881
:1044200047422CE1F2D1176BF551BF376840B6CB4C
:10443000CE5E316B5733CE2B169E0F7C4AEBE78E48
:104440009B7F1AFEE242E34F4B60D2273E3CCE3BBD
:10445000F6B053CCB0061D65BC86987655BDEBB35F
:10446000E7933AAAD835C65A6104010875F70008DF
:10447000F1FA00088D01020408102040801B36521A
:10448000096AD53036A538BF40A39E81F3D7FB7C9F
:10449000E339829B2FFF87348E4344C4DEE9CB543B
:1044A0007B9432A6C2233DEE4C950B42FAC34E08D4
:1044B0002EA16628D924B2765BA2496D8BD12572D4
:1044C000F8F66486689816D4A45CCC5D65B6926CE8
:1044D000704850FDEDB9DA5E154657A78D9D849062
:1044E000D8AB008CBCD30AF7E45805B8B34506D066
:1044F0002C1E8FCA3F0F02C1AFBD0301138A6B3A56
:104500009111414F67DCEA97F2CFCEF0B4E6739693
:10451000AC7422E7AD3585E2F937E81C75DF6E47EC
:10452000F11A711D29C5896FB7620EAA18BE1BFC4E
:10453000563E4BC6D279209ADBC0FE78CD5AF41F86
:10454000DDA8338807C731B11210592780EC5F60AE
:10455000517FA919B54A0D2DE57A9F93C99CEFA00B
:10456000E03B4DAE2AF5B0C8EBBB3C8353996117D5
:104570002B047EBA77D626E169146355210C7D633E
:104580007C777BF26B6FC53001672BFED7AB76CAA9
:1045900082C97DFA5947F0ADD4A2AF9CA472C0B7CE
:1045A000FD9326363FF7CC34A5E5F171D8311504DB
:1045B000C723C31896059A071280E2EB27B2750944
:1045C000832C1A1B6E5AA0523BD6B329E32F845377
:1045D000D100ED20FCB15B6ACBBE394A4C58CFD03C
:1045E000EFAAFB434D338545F9027F503C9FA8510C
:1045F000A3408F929D38F5BCB6DA2110FFF3D2CDDF
:104600000C13EC5F974417C4A77E3D645D1973607B
:10461000814FDC222A908846EEB814DE5E0BDBE088
:10462000323A0A4906245CC2D3AC629195E479E738
:10463000C8376D8DD54EA96C56F4EA657AAE08BAC6
:1046400078252E1CA6B4C6E8DD741F4BBD8B8A707E
:104650003EB5664803F60E613557B986C11D9EE129
:10466000F8981169D98E949B1E87E9CE5528DF8C66
:10467000A1890DBFE6426841992D0FB054BB166168
:104680006476616E63655F696E7465726E616C00FD
:104690005F63626F725F76616C75655F6465636F9F
:1046A00064655F696E7436345F696E7465726E61DD
:1046B0006C0063626F725F76616C75655F616476D2
:1046C000616E63655F66697865640063626F725FDF
:1046D00076616C75655F616476616E6365006362C7
:1046E0006F725F76616C75655F656E7465725F632E
:1046F0006F6E7461696E65720063626F725F76617E
:104700006C75655F6C656176655F636F6E7461691A
:104710006E65720063626F725F76616C75655F676C
:1047200065745F696E745F636865636B6564006977
:104730007465726174655F737472696E675F6368D4
:10474000756E6B730063626F725F76616C75655F27
:104750006D61705F66696E645F76616C7565007629
:10476000616C75652D3E666C61677320262043621F
:104770006F724974657261746F72466C61675F49EC
:104780006E746567657256616C7565546F6F4C61C8
:10479000726765207C7C2076616C75652D3E74792E
:1047A0007065203D3D2043626F72466C6F617454AA
:1047B000797065207C7C2076616C75652D3E7479FE
:1047C0007065203D3D2043626F72446F75626C6579
:1047D0005479706500282A76616C75652D3E707479
:1047E00072202620536D616C6C56616C75654D614D
:1047F000736B29203D3D2056616C756533324269EB
:1048000074207C7C20282A76616C75652D3E70743E
:1048100072202620536D616C6C56616C75654D611C
:10482000736B29203D3D2056616C756536344269B5
:104830007400657272203D3D2043626F724E6F4579
:1048400072726F72007372632F63626F7270617243
:104850007365722E63006C656E677468203D3D2041
:104860002873697A655F74296C656E6774680028BF
:1048700069742D3E666C61677320262043626F72F7
:104880004974657261746F72466C61675F556E6BD7
:104890006E6F776E4C656E67746829203D3D2030E1
:1048A0000069742D3E7479706520213D2043626F4C
:1048B00072496E76616C6964547970650069735FE2
:1048C00066697865645F747970652869742D3E74D3
:1048D000797065290063626F725F76616C75655FE0
:1048E00069735F636F6E7461696E6572286974299C
:1048F0000063626F725F76616C75655F69735F6993
:104900006E74656765722876616C756529007265DD
:104910006375727365642D3E74797065203D3D202A
:1049200043626F72496E76616C6964547970650098
:1049300063626F725F76616C75655F69735F6D61ED
:1049400070286D617029002C2066756E6374696F24
:104950006E3A2000617373657274696F6E20222550
:104960007322206661696C65643A2066696C652013
:10497000222573222C206C696E6520256425732501
:10498000730A0000EC010020232D302B2000686CFE
:104990004C00656667454647003031323334353662
:1049A000373839616263646566000000000000000A
:1049B00000000000000000000000000000000000F7
:1049C00000000000000000000000000000000000E7
:1049D00000000000000000000000000000000000D7
:1049E00000000000000000000000000000000000C7
:1049F00000000000000000000000000000000000B7
:104A0000000000000000000000000000F8B500BF3A
:084A1000F8BC08BC9E4670478B
:044A1800F8B500BF2E
:104A1C00005065737F8991999FA6ACB1B6BBC0C499
:104A2C00C8CDD0D4D8DBDFE2E5E8EBEEF1F5000041
:104A3C00F35B0008070000000014D1010E5504734D
:104A4C006F6C6F6B6579732E636F6D2F00000000B8
:104A5C0000093D00998C00085D8C00086D8B0008E6
:104A6C0000000000DD8A00082F8B0008058B000871
:104A7C00000000000000000000000000000000002A
:104A8C0000000000000000000000000009022900E6
:104A9C000101008032090400000203000002092118
:104AAC0011010001222200070581034000050705C2
:104ABC000103400005000000F18C0008218D000866
:104ACC00518D000800000000018E0008C18D000807
:104ADC00E18D000800000000000000000000000054
:104AEC00558E0008318E0008498E00083D8E000856
:104AFC000A0600020000004001000000BD970008FB
:104B0C00C9970008F1970008D59700080D98000880
:104B1C00000000000000000006D0F10901A101090D
:104B2C0020150026FF00750895408102092115000B
:104B3C0026FF00750895409102C00000D599000829
:104B4C00B9990008E198000800000000000000007E
:104B5C00C99800081D9A0008000000000000000021
:104B6C0000000000BD980008BD980008BD98000822
:104B7C00D598000809211100000122220000000034
:104B8C000A06000200000040010000000902290092
:104B9C000101008032090400000203000002092117
:104BAC0011010001222200070581034000050705C1
:104BBC000103400005000000619B00082D9B0008CC
:104BCC006D9A000800000000679A00085D9A0008C2
:104BDC00599A0008000000000000000000000000CE
:104BEC0000000000000000000000000000000000B9
:104BFC000100000003000000EC0100200000000098
:104C0C00CC490108EC490108AC490108000000003E
:104C1C000000000000000000000000000000000088
:104C2C000000000000000000000000000000000078
:104C3C000000000000000000000000000000000068
:104C4C000000000000000000000000000000000058
:104C5C000000000000000000000000000000000048
:084C6C00000000000301030039
:0400000508007491EA
:00000001FF
